:020000040800F2
:100000000000012011240008B5160008B7160008EA
:10001000B9160008BB160008BD1600080000000055
:10002000000000000000000000000000BF160008F3
:10003000C116000800000000C3160008C51600081D
:100040006124000861240008C91600086124000822
:100050006124000861240008D5160008DB1600089A
:10006000612400086124000861240008612400085C
:10007000612400086124000861240008E1160008DA
:10008000612400086124000861240008612400083C
:100090000000000061240008ED160008612400083B
:1000A000612400086124000861240008612400081C
:1000B000612400086124000861240008612400080C
:1000C00061240008612400086124000861240008FC
:1000D00061240008F5160008612400086124000866
:1000E0006124000861240008011700086124000849
:1000F00061240008000000000000000061240008E6
:1001000061240008612400080D170008612400081C
:1001100061240008612400086124000861240008AB
:10012000612400086124000861240008612400089B
:080130006124000861240008AD
:1001380010B5054C237833B9044B13B10448AFF319
:1001480000800123237010BD08010020000000007A
:10015800D0F0000808B5034B1BB103490348AFF3BF
:10016800008008BD000000000C010020D0F000084D
:10017800034613F8012B002AFBD1181A01387047DF
:1001880081F0004102E000BF83F0004330B54FEA40
:1001980041044FEA430594EA050F08BF90EA020FAD
:1001A8001FBF54EA000C55EA020C7FEA645C7FEA40
:1001B800655C00F0E2804FEA5454D4EB5555B8BF63
:1001C8006D420CDD2C4480EA020281EA030382EAD4
:1001D800000083EA010180EA020281EA0303362D66
:1001E80088BF30BD11F0004F4FEA01314FF4801C39
:1001F8004CEA113102D0404261EB410113F0004F4B
:100208004FEA03334CEA133302D0524263EB430301
:1002180094EA050F00F0A780A4F10104D5F1200E9F
:100228000DDB02FA0EFC22FA05F2801841F10001FA
:1002380003FA0EF2801843FA05F359410EE0A5F1CE
:1002480020050EF1200E012A03FA0EFC28BF4CF0FF
:10025800020C43FA05F3C01851EBE37101F00045B5
:1002680007D54FF0000EDCF1000C7EEB00006EEBC2
:100278000101B1F5801F1BD3B1F5001F0CD349084C
:100288005FEA30004FEA3C0C04F101044FEA4452A3
:1002980012F5800F80F09A80BCF1004F08BF5FEA2A
:1002A800500C50F1000041EB045141EA050130BD0A
:1002B8005FEA4C0C404141EB0101013C28BFB1F51C
:1002C800801FE9D291F0000F04BF01460020B1FA67
:1002D80081F308BF2033A3F10B03B3F120020CDA3A
:1002E8000C3208DD02F1140CC2F10C0201FA0CF018
:1002F80021FA02F10CE002F11402D8BFC2F1200C7D
:1003080001FA02F120FA0CFCDCBF41EA0C01904032
:10031800E41AA2BF01EB0451294330BD6FEA04047B
:100328001F3C1CDA0C340EDC04F11404C4F1200266
:1003380020FA04F001FA02F340EA030021FA04F378
:1003480045EA030130BDC4F10C04C4F1200220FACF
:1003580002F001FA04F340EA0300294630BD21FA0D
:1003680004F0294630BD94F0000F83F4801306BFD3
:1003780081F480110134013D4EE77FEA645C18BFC7
:100388007FEA655C29D094EA050F08BF90EA020F5E
:1003980005D054EA000C04BF1946104630BD91EA56
:1003A800030F1EBF0021002030BD5FEA545C05D159
:1003B8004000494128BF41F0004130BD14F5800498
:1003C8003CBF01F5801130BD01F0004545F0FE410C
:1003D80041F470014FF0000030BD7FEA645C1ABF41
:1003E800194610467FEA655C1CBF0B46024650EA78
:1003F800013406BF52EA033591EA030F41F40021A4
:1004080030BD00BF90F0000F04BF0021704730B529
:100418004FF4806404F132044FF000054FF00001FE
:1004280050E700BF90F0000F04BF0021704730B5BF
:100438004FF4806404F1320410F0004548BF404294
:100448004FF000013EE700BF42004FEAE2014FEAE9
:1004580031014FEA02701FBF12F07F4393F07F4FC4
:1004680081F06051704732F07F4208BF704793F0C7
:100478007F4F04BF41F40021704730B54FF46074DA
:1004880001F0004521F000411CE700BF50EA0102DD
:1004980008BF704730B54FF000050AE050EA010286
:1004A80008BF704730B511F0004502D5404261EBF6
:1004B80041014FF4806404F132045FEA915C3FF437
:1004C800D8AE4FF003025FEADC0C18BF03325FEAD4
:1004D800DC0C18BF033202EBDC02C2F1200300FA85
:1004E80003FC20FA02F001FA03FE40EA0E0021FAAA
:1004F80002F11444BDE600BF4FF0FF3C06E000BF28
:100508004FF0010C02E000BF4FF0010C4DF804CD94
:100518004FEA410C7FEA6C5C4FEA430C18BF7FEA54
:100528006C5C1BD001B050EA410C0CBF52EA430C82
:1005380091EA030F02BF90EA020F0020704710F102
:10054800000F91EA030F58BF994208BF90422CBF91
:10055800D8176FEAE37040F0010070474FEA410C8A
:100568007FEA6C5C02D150EA013C07D14FEA430CA8
:100578007FEA6C5CD6D152EA033CD3D05DF8040B19
:10058800704700BF8446104662468C46194663464B
:1005980000E000BF01B5FFF7B7FF002848BF10F122
:1005A800000F01BD4DF808EDFFF7F4FF0CBF012067
:1005B80000205DF808FB00BF4DF808EDFFF7EAFFE3
:1005C80034BF012000205DF808FB00BF4DF808ED9E
:1005D800FFF7E0FF94BF012000205DF808FB00BF93
:1005E8004DF808EDFFF7CEFF94BF012000205DF81D
:1005F80008FB00BF4DF808EDFFF7C4FF34BF01202A
:1006080000205DF808FB00BF4FEA410212F5001216
:1006180015D211D56FF47873B3EB625212D94FEA41
:10062800C12343F0004343EA505311F0004F23FA2B
:1006380002F018BF404270474FF00000704750EA80
:10064800013005D111F0004008BF6FF0004070473D
:100658004FF00000704700BF80F0004002E000BF8C
:1006680081F0004142001FBF5FEA410392EA030F95
:100678007FEA226C7FEA236C6AD04FEA1262D2EBDF
:100688001363C1BFD218414048404140B8BF5B42E4
:10069800192B88BF704710F0004F40F4000020F07D
:1006A8007F4018BF404211F0004F41F4000121F093
:1006B8007F4118BF494292EA030F3FD0A2F10102DD
:1006C80041FA03FC10EB0C00C3F1200301FA03F11B
:1006D80000F0004302D5494260EB4000B0F5000F3E
:1006E80013D3B0F1807F06D340084FEA310102F1FD
:1006F8000102FE2A51D2B1F1004F40EBC25008BFAF
:1007080020F0010040EA03007047490040EB000078
:10071800013A28BFB0F5000FEDD2B0FA80FCACF179
:10072800080CB2EB0C0200FA0CF0AABF00EBC250A6
:1007380052421843BCBFD0401843704792F0000F94
:1007480081F4000106BF80F400000132013BB5E7E7
:100758004FEA41037FEA226C18BF7FEA236C21D05D
:1007680092EA030F04D092F0000F08BF08467047C2
:1007780090EA010F1CBF0020704712F07F4F04D190
:10078800400028BF40F00040704712F100723CBFA3
:1007980000F50000704700F0004343F0FE4040F4CD
:1007A800000070477FEA226216BF08467FEA23638B
:1007B8000146420206BF5FEA412390EA010F40F476
:1007C800800070474FF0000304E000BF10F00043C2
:1007D80048BF40425FEA000C08BF704743F09643A9
:1007E80001464FF000001CE050EA010208BF7047C4
:1007F8004FF000030AE000BF50EA010208BF70474B
:1008080011F0004302D5404261EB41015FEA010C5F
:1008180002BF84460146002043F0B64308BFA3F157
:100828008053A3F50003BCFA8CF2083AA3EBC25339
:1008380010DB01FA02FC634400FA02FCC2F1200258
:10084800BCF1004F20FA02F243EB020008BF20F08F
:100858000100704702F1200201FA02FCC2F12002F5
:1008680050EA4C0021FA02F243EB020008BF20EAEA
:10087800DC7070474FF0FF0C1CEAD0521EBF1CEA18
:10088800D15392EA0C0F93EA0C0F6FD01A4480EA06
:10089800010C400218BF5FEA41211ED04FF00063EF
:1008A80043EA501043EA5111A0FB01310CF000401B
:1008B800B1F5000F3EBF490041EAD3715B0040EA41
:1008C800010062F17F02FD2A1DD8B3F1004F40EB11
:1008D800C25008BF20F00100704790F0000F0CF0E4
:1008E800004C08BF49024CEA502040EA51207F3AA8
:1008F800C2BFD2F1FF0340EAC250704740F4000083
:100908004FF00003013A5DDC12F1190FDCBF00F073
:1009180000407047C2F10002410021FA02F1C2F121
:10092800200200FA02FC5FEA310040F1000053EABD
:100938004C0308BF20EADC70704792F0000F00F00B
:10094800004C02BF400010F4000F013AF9D040EA11
:100958000C0093F0000F01F0004C02BF490011F4A5
:10096800000F013BF9D041EA0C018FE70CEAD153A3
:1009780092EA0C0F18BF93EA0C0F0AD030F0004C23
:1009880018BF31F0004CD8D180EA010000F00040D7
:10099800704790F0000F17BF90F0004F084691F095
:1009A800000F91F0004F14D092EA0C0F01D14202CF
:1009B8000FD193EA0C0F03D14B0218BF084608D198
:1009C80080EA010000F0004040F0FE4040F40000E2
:1009D800704740F0FE4040F4400070474FF0FF0C75
:1009E8001CEAD0521EBF1CEAD15392EA0C0F93EABC
:1009F8000C0F69D0A2EB030280EA010C49024FEA0E
:100A0800402037D04FF0805343EA111143EA1013C6
:100A18000CF000408B4238BF5B0042F17D024FF47E
:100A2800000C8B4224BF5B1A40EA0C00B3EB510F59
:100A380024BFA3EB510340EA5C00B3EB910F24BF42
:100A4800A3EB910340EA9C00B3EBD10F24BFA3EBC7
:100A5800D10340EADC001B0118BF5FEA1C1CE0D18F
:100A6800FD2A3FF650AF8B4240EBC25008BF20F042
:100A7800010070470CF0004C4CEA50207F32C2BF96
:100A8800D2F1FF0340EAC250704740F400004FF033
:100A98000003013A37E792F0000F00F0004C02BF64
:100AA800400010F4000F013AF9D040EA0C0093F02E
:100AB800000F01F0004C02BF490011F4000F013B88
:100AC800F9D041EA0C0195E70CEAD15392EA0C0FF0
:100AD80008D142027FF47DAF93EA0C0F7FF470AF28
:100AE800084676E793EA0C0F04D14B023FF44CAF6B
:100AF80008466EE730F0004C18BF31F0004CCAD100
:100B080030F000427FF45CAF31F000437FF43CAF3B
:100B18005FE700BF4FEA4002B2F1FE4F0FD34FF03C
:100B28009E03B3EB12620DD94FEA002343F0004352
:100B380010F0004F23FA02F018BF404270474FF000
:100B48000000704712F1610F01D1420205D110F087
:100B5800004008BF6FF0004070474FF0000070473A
:100B680042000ED2B2F1FE4F0BD34FF09E03B3EB0F
:100B7800126209D44FEA002343F0004323FA02F03B
:100B880070474FF00000704712F1610F01D1420227
:100B980002D14FF0FF3070474FF00000704700BFA0
:100BA80053B94AB9002908BF00281CBF4FF0FF31CC
:100BB8004FF0FF3000F070B9ADF1080C6DE904CECC
:100BC80000F006F8DDF804E0DDE9022304B0704720
:100BD8002DE9F047089E0D4604460F46002B4AD1E2
:100BE8008A42944665D9B2FA82F343B102FA03FC09
:100BF800C3F120029F4020FA02F217439C404FEABB
:100C08001C4E1FFA8CF5B7FBFEF1220C0EFB117778
:100C180042EA074201FB05F090420AD91CEB0202A6
:100C280001F1FF3780F01B81904240F218810239B0
:100C38006244121AA4B2B2FBFEF00EFB102244EA80
:100C4800024400FB05F5A5420AD91CEB040400F197
:100C5800FF3280F00681A54240F2038164440238E5
:100C680040EA0140641B00211EB1DC400023C6E9B4
:100C78000043BDE8F0878B4208D9002E00F0EC80D5
:100C88000021C6E900050846BDE8F087B3FA83F1FC
:100C9800002949D1AB4202D3824200F2F780841A7C
:100CA80065EB030201201746002EE2D0C6E9004793
:100CB800DFE702B9FFDEB2FA82F3002B40F08F8043
:100CC8008A1A4FEA1C471FFA8CFE0121B2FBF7F57E
:100CD80007FB1520220C42EA00420EFB05F0904269
:100CE80008D91CEB020205F1FF3802D2904200F24B
:100CF800CA804546121AA4B2B2FBF7F007FB1022CD
:100D080044EA02440EFB00FEA64508D91CEB040485
:100D180000F1FF3202D2A64500F2BA801046A4EBD9
:100D28000E0440EA05409FE7C1F120078B4022FAF4
:100D380007FC4CEA030C05FA01F420FA07F3FD401E
:100D4800234300FA01F94FEA1C401FFA8CFEB5FB59
:100D5800F0F81C0C00FB185544EA054408FB0EF596
:100D6800A54202FA01F20BD91CEB040408F1FF3A80
:100D780080F08780A54240F28480A8F1020864448C
:100D8800641B9DB2B4FBF0F300FB134445EA044432
:100D980003FB0EFEA64508D91CEB040403F1FF3043
:100DA8006BD2A64569D9023B644443EA0840A0FBDC
:100DB8000283A4EB0E049C42C6461D4655D352D06E
:100DC80056B1B9EB0E0364EB050404FA07F7CB4000
:100DD800CC401F43C6E900740021BDE8F087C3F189
:100DE800200102FA03FC20FA01F225FA01F19D40E4
:100DF8002A434FEA1C471FFA8CFEB1FBF7F007FBAA
:100E08001015110C41EA054100FB0EF58D4204FA5C
:100E180003F408D91CEB010100F1FF382FD28D42F1
:100E28002DD902386144491B92B2B1FBF7F507FB93
:100E3800151142EA014205FB0EF1914208D91CEB5B
:100E4800020205F1FF3816D2914214D9023D6244DC
:100E5800521A45EA004139E73146304609E7394632
:100E6800E7E61046FCE6C145AAD2B8EB020E63EBF2
:100E78000C050138A4E74546EAE7034695E74046EE
:100E8800D1E7D0467CE7023D624433E708460BE7EA
:100E98006444023843E700BF704700BF1348144A50
:100EA80008B54FF00043C0E9002304220023426143
:100EB8000122C2614FF4805107220383C0E9023343
:100EC800C0E90933C0E90C120361837680F8203049
:100ED80080F82C30826380F83C30C36401F0F8FA63
:100EE80018B1BDE8084000F023BB08BD240100206C
:100EF800002401400268084B9A4282B00AD14FF0A0
:100F0800B0431A6E42F400721A661B6E03F4007343
:100F18000193019B02B07047002401400268054B11
:100F28009A4201BF4FF0B042136E23F40073136668
:100F3800704700BF0024014030B585B00024054645
:100F4800CDE901440394FFF7A9FF144801F058FEC6
:100F580008B100F0EDFA1148039401A9CDE9015454
:100F680001F014FC08B100F0E3FA0C4801F072FD3E
:100F780008B100F0DDFA4FF0FF31084801F0A8FB96
:100F8800064801F01FFE054801F0FCFB0446034833
:100F980001F0C2FD204605B030BD00BF240100208D
:100FA800014B024A1A6070472401002000240140C6
:100FB80008B50948FFF7C0FF68B1084BB3F8AA3075
:100FC8004FF6FF72934216BF40F6E442044B534378
:100FD800B3FBF0F398B208BD002000B40075FF1F02
:100FE800D8084C0013B50023ADF80630FFF7E0FF32
:100FF80004461948FFF7A0FF184BB3F8C820B3F808
:10100800A8108A4204FB00F018D040F6E443B0FB75
:10101800F3F364205B1A4343521A93FBF2F31E3333
:101028001BB2ADF80630BDF806305BB21B02ADF856
:101038000630BDF8060000B202B010BD4FF47A7257
:1010480040F6FF73B0FBF3F35343A3F53923A3F53D
:101058000C6340F6C412E0E7001000B00075FF1FF3
:101068004FF0B04307B59A6C42F004029A649A6C48
:1010780002F004020192019A9A6C42F001029A6409
:101088009B6C03F001030093002202210F20009BB8
:1010980001F054FE0F2003B05DF804EB01F080BEB0
:1010A80008B502F0C5F810B16FF0040008BD064B92
:1010B8009A6942F040429A614CF2FA321A6102F09F
:1010C800C9F80028F2D0EFE700400058F0B585B025
:1010D80000230C4600930646A8B3FFF7E1FF054638
:1010E80070BB02F0A5F888BB1A481B4A022301937B
:1010F800D0F8E01506F1784302EA8121B3FBF1F755
:1011080001FB1733DB0A0293D0F8E00504F17841BC
:101118000139314402EA8022B1FBF2F002FB1011DE
:10112800C3EBD1230133694601A8039302F012F9F6
:1011380020B102280CBF01256FF0010502F08AF8E2
:10114800284605B0F0BD6FF00505F9E76FF0040516
:10115800F6E700BF0070FF1F00FCFF03014B18609B
:1011680000207047880100202DE9F04F89B0B0F1C8
:10117800006F06460F460092C0F0C580DFF89881E0
:10118800664DD8F8E03505EA832303F10063013B97
:10119800984200F2B880002800F0B880002900F0DA
:1011A800B58040EA02035B0740F0B080FFF778FFA4
:1011B8000446A0BB02F03CF8002840F0AA80D8F80A
:1011C800E01506F1784205EA8121B2FBF1F301FB53
:1011D8001322009B03F17843013B3344B3FBF1F046
:1011E80001FB1033DB0A01334FEAD22AA3EBD222E8
:1011F800012A039388BFC6F30A050AF58038C6F1A9
:10120800080398BF009D069388BFC5F500654FEA9F
:10121800C828B346039B9A4505D302F01BF820461D
:1012280009B0BDE8F08FA6F10803069A1A44954262
:1012380019D804950197CDF814B04FF00009059B13
:1012480009EB0301049B99453ED3009BAB442F4413
:101258005D1BB5F5006F28BF4FF400650AF1010A60
:1012680008F50068D6E753F8081F5A68B2F1FF3F3F
:1012780008BFB1F1FF3FD8D0294B186810B96FF0FB
:101288000504CAE7B8F1000F04D04FF400624146E4
:101298000DF044FADFF88890D9F80030CBF30A0053
:1012A80039461844AAB20DF039FA4FF400614046A5
:1012B800FFF70CFF08BBD9F8003001934FF4006327
:1012C800CDF814800493B8E7019B07914B4402932F
:1012D8000120D3E9002301F0F7FF88B90799019BA2
:1012E800D1E9000259F80310029B5B689A4208BFD3
:1012F800884205D109F10809A1E76FF001048CE7DC
:101308006FF0030489E74FF0FF3488E76FF00504B6
:1013180085E76FF0040482E70070FF1F00FCFF03FD
:1013280088010020B1F1006F70B511D30B4BD3F8D1
:10133800E0650B4B03EA862303F10063013B994206
:1013480006D840B139B192B20DF0E8F9002070BD6D
:101358004FF0FF30FBE76FF00500F8E70070FF1F64
:1013680000FCFF03B0F1006F10B40DD3084BD3F8A5
:10137800E045084B03EA842303F10063013B9842EC
:1013880002D810BCFFF7A2BE4FF0FF3010BC704768
:101398000070FF1F00FCFF034FF0B04382B0DA6C0F
:1013A8000243DA64DB6C03400193019B02B070478F
:1013B80030B5022087B000242C4DCDE90444FFF756
:1013C800EBFF0420FFF7E8FF0120FFF7E5FF01A985
:1013D8004FF6FF7203232846CDE90123039402F058
:1013E80007F801A9224802F003F801A94FF090403C
:1013F80001F0FEFF4FF0B0432846DA6C22F00102FC
:10140800DA64DA6C22F00202DA64DA6C22F004029E
:10141800DA644FF43A41224602F00AF90220FFF753
:10142800BBFF14210123CDE90113CDE9030001A974
:10143800284601F0DDFF22462146062001F07EFC09
:10144800062001F0ADFC22462146072001F076FC7B
:10145800072001F0A5FC22462146162001F06EFC6B
:10146800162001F09DFC07B030BD00BF0004004805
:101478000008004800B59BB04822002108A80DF0DC
:1014880075FD1822002102A80DF070FD02F0EAF89F
:101498004FF0B0420120D2F8903023F01803C2F880
:1014A8009030D2F8003423F4C06343F40073C2F8D8
:1014B8000034D2F8003403F4C0630193019B242361
:1014C800089381230B930023CDE91003B02208A8C9
:1014D800CDE9122302F050FA08B172B6FEE74F23A5
:1014E800CDE90230CDE90400CDE90600022102A8C9
:1014F80002F0DCFC08B172B6FEE71BB05DF804FB35
:1015080008B500F0ABFFFFF7B5FFFFF751FF06483E
:1015180003F0F0FB00F058FC04480122102102F00F
:1015280087F800F058FCFCE7380200200004004867
:1015380072B6FEE700B58DB02C22002101A80DF08F
:1015480015FD1748174B03601F2383604FF0804237
:101558000023C0E90433C0E9072383614FF4807393
:10156800436202F04DFF08B1FFF7E2FF0C4803F0B9
:1015780073F808B1FFF7DCFF4FF000530022079320
:10158800074808924FF4807301A9029206920B93C0
:1015980002F096FF08B1FFF7CBFF0DB05DF804FB32
:1015A8008C0100200028004010B5044690B0382275
:1015B800002102A80DF0DAFC2268194B9A422CD1BE
:1015C8004FF48033029302A84FF480730F9302F014
:1015D80091FD08B1FFF7ACFF4FF0B0430220D3F8FC
:1015E800902042F40042C3F890209A6D42F4806241
:1015F8009A659B6D002203F4806311460193019B59
:1016080001F09CFB022001F0CBFB00222A201146AE
:1016180001F094FB2A2001F0C3FB10B010BD00BFFD
:101628000028004008B500F02FFF034B07229A61FD
:10163800BDE8084002F03EB80004005800F02BBF97
:1016480008B50F4803F056FB00F07CFB4FF6FF711E
:101658004FF0904001F078FF0A484FF6FF7101F013
:1016680073FF09484FF6FF7101F06EFF00F00CFFA1
:10167800064B0120C3F88800BDE8084002F05CB8BA
:101688003802002000040048000800480004005800
:1016980008B500F0F9FEBDE808400121002001F07E
:1016A800E9BF00F0F8BE00F0F6BE7047FEE7FEE7BF
:1016B800FEE7FEE7FEE77047704770477047000097
:1016C800014802F0EFBF00BF8C010020012001F0AB
:1016D800BDBF022001F0BABF014801F03BBD00BF09
:1016E800D8010020402001F0B1BF0000014803F0FC
:1016F800BDBB00BF38020020014802F005BE00BF94
:101708008C010020014803F0F8B900BFC401002093
:10171800054808B50823036003F00AF818B1BDE8C6
:101728000840FFF705BF08BDC40100204FF0B043D3
:1017380007B55A6E42F001025A665B6E002203F04A
:101748000103019311463220019B01F0F7FA322080
:1017580003B05DF804EB01F023BB00000CB407B53F
:10176800054A05AB102101930DF0E2FA03B05DF8CC
:1017780004EB02B0704700BF74F1000830B585B0C3
:10178800044602A80D460DF0FFF8BDF90C30064AD4
:1017980000931021029B2046FFF7E0FF2046FEF74A
:1017A800E7FC288005B030BD74F100084FF0B04266
:1017B80010B5936823F4004393600DF06DF90D4B59
:1017C80001241C700CF038FE0B480CF04FFE0B4B3C
:1017D8004FF400421A6100200CF04EFEFFF7E0FBC8
:1017E80000F0B4F80CF044FF21462046BDE8104054
:1017F8000CF05EBFD001002085170008004000589B
:101808000CF06CBF08B5FFF7D3FB40F6B83398422D
:101818000CD8B0F5E16F0BD3FE23A0F5E160584377
:101828004FF49663B0FBF3F0C0B208BDFE20FCE7AE
:101838000020FAE77FB5684600F06CF80198FFF7DA
:1018480069F900B207B05DF804FB0000194A38B521
:10185800D2F88035591C044619D100F023FE0546FC
:1018680000F02CFE054400F023FE2B0EE3712B0C38
:10187800A3712B0A6371030EE370C0F30742C0F330
:1018880007232571C0B2A2706370207038BD190A91
:10189800C3718171190C1B0E41710371D2F8843523
:1018A800C370D2F88405C0F30722C0F30743000EC3
:1018B800E9E700BF0070FF1F38B5094BD3F8803542
:1018C80003600133054609D100F0ECFD044600F041
:1018D800EFFD444000F0F2FD44402C6038BD00BFED
:1018E8000070FF1F012102200CF0CCBE0021022055
:1018F8000CF0C8BE00207047024B187808B100F001
:101908005DB87047D001002082B00190019802B004
:1019180000F0F0B810B50446FFF764FB074BA3606E
:1019280040F30F20FEF752FF054B064A2360064B93
:101938006060C4E90323002010BD00BF00004842D6
:1019480000007A440D093E00AB03050000207047F3
:10195800014B1868704700BFD4010020032070476E
:1019680008B501464FF47A7200238002890DFFF70B
:1019780017F908BD4FF47A73A0FB0303800A40EA05
:1019880083507047034B98689A689042FBD1C043D4
:10199800704700BF0028004008B5FFF7F3FF014B70
:1019A800186008BDD401002008B5FFF7EBFF024B13
:1019B8001B68C01A08BD00BFD4010020024B18786C
:1019C80008B1FFF7DFBF7047D101002010B5074B02
:1019D800074C0122DA654FF48071204602F05AFC68
:1019E8004FF0FF332363002010BD00BF00280040E4
:1019F8008C01002002460021014802F064BE00BFAD
:101A08008C01002002460121014802F05CBE00BFA3
:101A18008C01002010B58CB02C220021044601A8AE
:101A28000DF0A4FAFFF7D2FF0C4B0D481B681C44BD
:101A38000023089306934FF00053E44307930122D1
:101A48004FF4807301A902940B9302F039FD08B199
:101A5800FFF76EFD00200CB010BD00BFD4010020C0
:101A68008C01002038B50546FFF78CFF022104469B
:101A7800074802F02FFEC4F309024FF47A71A2FB63
:101A88000121920AA30A2A8043EA805038BD00BF88
:101A98008C0100200148002102F01CBE8C010020AE
:101AA8000148012102F016BE8C010020F8B50F4D47
:101AB8002E78CEB90E4C4FF0FF372763FFF73AFD6B
:101AC800FFF784FF4FF48071204602F0E3FB2046C5
:101AD800276302F0A3FD32462046022102F0F3FDFF
:101AE800FFF75AFF01232B700020F8BDD101002019
:101AF8008C010020014610B54FF47A720023800251
:101B0800890DFFF74DF80146FFF73CFF0446FFF744
:101B180039FF031B8B4200D310BD00BFF7E70DF060
:101B2800C3B8000010B5064C0221204602F0D2FDD1
:101B38000221421C2046BDE8104002F0C4BD00BF8F
:101B48008C0100201348144A08B54FF4E133C0E96A
:101B5800002300230C22C0E90233C0E90523C0E9B1
:101B68000733C0E90933036103F061FF08B1FFF7E8
:101B7800DFFC0848002104F0D6F808B1FFF7D8FCCC
:101B8800044804F0B0F818B1BDE80840FFF7D0BC2D
:101B980008BD00BF380200200044004070B596B070
:101BA80006461422002103A80DF0E0F9382200218E
:101BB80008A80DF0DBF932682C4B9A4254D1022365
:101BC800089308A82A4B0A9302F094FA08B1FFF781
:101BD800AFFC4FF0B04300259A6D42F400329A658D
:101BE8009A6D02F400320292029ADA6C42F0010213
:101BF800DA64DB6C03F0010301930422019B0223E6
:101C0800CDE903230324072303A94FF09040CDE92E
:101C18000554079301F0ECFB082303A94FF090400B
:101C2800CDE90334CDE90555124C01F0E1FB124929
:101C380025621423C4E900131023C4E902352046A1
:101C48008023C4E90435C4E9065501F009F908B14F
:101C5800FFF76EFC2520F46700220221A66201F03E
:101C68006DF8252001F09CF816B070BD00440040C6
:101C780004000C00D80100205800024002680C4BF8
:101C88009A4210B5044612D14FF0B0420C21936D20
:101C980023F4003393654FF0904001F055FCE06F5A
:101CA80001F052F9BDE81040252001F087B810BDB9
:101CB8000044004008B50A460146024803F03AF8D5
:101CC800002008BD3802002013B5114B114C1860D4
:101CD8004FF40013009302AB13E90600204603F00B
:101CE800A6FF2368DA69D103FCD4DA695202FCD56D
:101CF8009A68084842F480029A6003F0DEFF0649B9
:101D08000448012203F04CFF002002B010BD00BFC0
:101D1800CC02002038020020D402002008B5074B6E
:101D28001860FFF79DF9FFF70DFF054AD2F88030DC
:101D380043F00063C2F88030002008BDD0020020C4
:101D48000008005808B54FF0B04308489A6B42F4B1
:101D580000329A639A6B22F400329A63FFF78EFF7F
:101D68000F2001F02BF8002008BD00BF380200202A
:101D78000268044B9A4203D1034B00201B681847A2
:101D8800704700BF00440040D002002002680B4B9F
:101D98009A4210B504460FD1094B1B682BB1D0F8F5
:101DA800902012B907480121984720460549BDE807
:101DB8001040012203F0F4BE10BD00BF00440040F3
:101DC800CC020020D402002008B5FFF7EFFCBDE8E4
:101DD800084000F007BA4FF0FF300CF0E3BC704742
:101DE80070477047014BD870704700BF58000020FB
:101DF800014B1874704700BF5800002008B5022036
:101E080000210CF097FCBDE8084001480CF0FABE30
:101E180028040020002101200CF08CBC10B5094CCE
:101E280060B1206008480CF09FFE216806480CF05D
:101E380023FFBDE8104004480CF0E4BE47F23053DD
:101E48002360EFE7700000202804002008B50E4B3F
:101E58001B78022B03D1002108200CF06BFC0B48E7
:101E680000224FF4004101F0E3FB084800224FF440
:101E7800007101F0DDFBBDE80840044800224FF482
:101E8800006101F0D5BB00BF00000020000400483D
:101E9800024800224FF4004101F0CABB0004004888
:101EA800024800224FF4007101F0C2BB0004004850
:101EB80038B504460D4607484FF40061FFF752FA5B
:101EC80030B92A4621460348BDE83840FFF74CB9E7
:101ED80038BD00BF00F003080A460149FFF722BADF
:101EE80000F0030838B5154801224FF4004101F00D
:101EF8009FFB124801224FF4007101F099FB0F4833
:101F080001224FF4006101F093FB0D480CF02CFE08
:101F180004F06EFB60B90B4C0B480125257004F0EA
:101F2800F9F92078294603F04BFF05480CF06AFEC2
:101F3800BDE8384005480CF065BE00BF0004004805
:101F4800280400200000002058000020F80300208A
:101F580004F0EABB2DE9F04387B0FFF753FC0122F8
:101F680010210546514801F063FB50480122042125
:101F780001F05EFB04F01AF80746D8B100244C487B
:101F88000CF0F2FD4B4B4A481968A14238BF214674
:101F98000CF072FE46480CF035FE4448002204213D
:101FA80001F046FB41480022102101F041FB07B037
:101FB800BDE8F083404C6846FFF7ACFC022302986A
:101FC80023703E49FEF756FCFEF7CAFD86B201981B
:101FD800FEF7A0FD3A490FFA80F80098FEF74AFC90
:101FE8003649FEF7FBFCFEF7BBFD364A63681278FC
:101FF8001A706368C0F307225A7063689870636840
:1020080083F803806368320A1A7163685E712E4E22
:102018003378082B01D0012B2DD8626800239371E7
:102028006268D371626828B200EB40001372537281
:1020380000EB4010FE23B0FBF3F00B2390726370AB
:10204800224C637A63B103F09DFF012808D1204632
:102058000CF08AFD154800224FF4006101F0E8FAFF
:10206800F1781548002203F0B7FF063086D103F057
:1020780083FF044683E7DDE90385D4F80490FFF77E
:10208800C1FB89F8060063684FEA2842DA71636881
:102098004FEA28221A722A149A722A1283F809809F
:1020A800DA721D735F739F730F23C8E7000400483B
:1020B80028040020700000200400002000002041B7
:1020C8000000C842C703002058000020C8030020B1
:1020D80002484FF4006101F0B0BA00BF00040048A4
:1020E80008B504F08EFA80B903F04CFF01280CD132
:1020F800BFF34F8F0549064BCA6802F4E0621343E9
:10210800CB60BFF34F8F00BFFDE708BD00ED00E0D7
:102118000400FA0508B560B1037853B105480122F7
:102128004FF4007101F084FABDE8084002480CF051
:1021380069BD08BD000400481004002010B568B14E
:1021480090F9064054B906480CF00EFD22460548A1
:10215800BDE810404FF4006101F06ABA10BD00BF3D
:10216800C80300200004004838B504460D4681B372
:10217800184801224FF4004101F05AFA16480CF0B1
:1021880041FD2B782BB324B3636822780BB3022A62
:102198000ED0032A1DD16278012A1AD11878012895
:1021A80002D0022800D0A0B9BDE8384003F0E0BF53
:1021B8006278012A0DD11B78084903F001030B70DE
:1021C80003B91A46BDE8384002484FF4006101F0EF
:1021D8002FBA38BD00040048E0030020C7030020E0
:1021E800704700001FB5002403A92046039404F09B
:1021F800EBF903A9012004F0E7F92C4B2C480094D3
:1022080022464FF4FA710CF051FC2A4B2A480094EC
:1022180022464FF4FA710CF049FC284B28480094E8
:1022280001224FF4FA710CF041FC2046FEF796FFAC
:1022380008B1FFF77DF9234B009400224FF4FA61AF
:1022480021480CF033FC214A002101200CF02EFB20
:102258001F4A002102200CF029FB1E4A00210420FD
:102268000CF024FB1C4A002108200CF01FFB00F096
:102278004FF81A491A4804F05DF91A4804F04AF868
:102288000F480CF0BFFC184B0021187803F098FD9C
:1022980016490094164B0968164800220CF006FCF3
:1022A80014480CF0AFFC04B010BD00BFA91E000814
:1022B80010040020991E0008E0030020D92000081F
:1022C800C8030020551E0008F80300201561000807
:1022D8005D1F0008591F0008ED1E000800000301DB
:1022E8000C00002058000020000000207000002092
:1022F800051E000828040020022804D0402806D122
:102308000021042001E0002108200CF013BA7047D6
:10231800034B0022C3E902220122C3E900227047CD
:102328004004002000487047400400204FF0B043AC
:1023380082B0DA6C0243DA64DB6C03400193019BE0
:1023480002B070472DE9F04186B000240220154DF7
:102358000594FFF7EBFF0420FFF7E8FF124F039403
:102368004FF4807601230DEB0001CDE90163284687
:10237800032304934FF4005801F03AF801A93846B2
:10238800CDF8048001F034F822464146384601F081
:102398004FF928462246314601F04AF9204606B050
:1023A800BDE8F0810004004800080048032810B583
:1023B8000ED8012810D868B902460B484FF480712E
:1023C80001F036F9002209484FF4005101F030F9C4
:1023D800002010BD0122F0E7002203484FF480716D
:1023E80001F026F90122EEE7000400480008004841
:1023F80002207047002070470120704700280CBF5A
:102408000F201620704700000D48854600F025F87B
:102418000C480D490D4A002302E0D458C450043337
:10242800C4188C42F9D30A4A0A4C002301E013600D
:102438000432A242FBD30CF0A1FDFFF761F8FEE7DE
:10244800000001200000002008010020B4FC000862
:1024580008010020B4210020FEE7704710B50320D2
:1024680000F05AFC01F078FA064B18600F20FFF7CD
:1024780041FA044618B9FFF718F9204610BD01249F
:10248800FBE700BF740000204FF0E022136923F03F
:102498000203136170474FF0E022136943F002030F
:1024A80013617047014BD3F8900570470070FF1F08
:1024B800014BD3F8940570470070FF1F014BD3F808
:1024C800980570470070FF1F8068C0F38000704750
:1024D800F7B5002301930446002800F0E980856DD4
:1024E80025B9FEF707FDE56584F8545023689A6816
:1024F800D00040F1A1809A68D10000F1B480A26DAB
:1025080042F01002A265E26D42F00102E265012587
:102518001846FFF7D9FFA26D02F01002024340F0FF
:10252800C980A26D206922F4817242F00202A2657C
:102538009A68D2075DD4226BA67E94F82CC0003A24
:1025480018BF01221703D4E902120A43217E42EA86
:102558008132617E42EAC13242EA4632002842EACA
:102568004C02B4BF20F000414FF400113A430A4333
:1025780094F82010012903D1002E76D142F480323C
:10258800616A21B1A66A01F4E07131430A43D9684E
:10259800E66C21F4FE3121F4FF711143D96094F8FF
:1025A8003C206168012A01F0404C4CEA060609D13A
:1025B800D4E910273A433243A66C324342EA0C026C
:1025C80042F001061F693E4A3A4032431A6121F03F
:1025D8000042B2F1804F0CD0B1F1004F09D0394E12
:1025E800D6F8082701F4701122F470120A43C6F8CD
:1025F80008275A69666BA16B22F0070232435A61B9
:102608005A6922F0700242EA01125A61002835D153
:102618009A6A62F00F029A625B6903F007039E42AE
:102628003CD10023E365A36D23F0030343F00103CA
:10263800A365284603B0F0BD9A68234922F01042EA
:1026480022F0170242F080529A60204A1268B2FBC8
:10265800F1F2013252000192019A002A3FF44BAF85
:10266800019A013AF7E7002552E7A16D41F02001F0
:10267800A165E16D41F00101E16581E7B0F5001F59
:10268800CAD19A6AE269013A92006FF00F0102F02A
:102698001C0201FA02F2216E0A43BCE7A36D23F083
:1026A800120343F01003A365E36D43F00103E365F0
:1026B8000125BEE7A36D43F01003A365F8E700BF4B
:1026C80002FCFF1F00200140400D030074000020A1
:1026D800F8B54569082D04460E460AD00368DB683C
:1026E800D80705D5A36D43F02003A3650120F8BDE5
:1026F8000425FFF701F9074623681A682A4221D002
:10270800A26D42F40072A265DA6812F4406F14D127
:10271800A27E92B91A6812070FD51846FFF7D4FEA1
:1027280028BB5A6822F00C025A60A26D22F480720B
:1027380022F0010242F00102A265207E00BB0C22B9
:102748001A60D4E7711CD8D0FFF7D6F8C01BB04286
:1027580001D8002ED0D123681B682B40CCD1A26DA4
:1027680084F8543042F00402A2650320BFE7A26D4A
:1027780042F02002A265E26D42F00102E265DCE768
:102788000020B4E70368186C70470000F7B5002311
:10279800019390F85430012B044600F0C580056879
:1027A8000669012380F854302846FFF78DFE00287B
:1027B80040F0B480D1E90020022826F0040300F09C
:1027C8008280B3F1004FC2F3110E13D1AB6A43EA12
:1027D8000E03AB628B68686903EA022323F07C432B
:1027E80023F0FF0320EA02210B43002A6B6126DB5A
:1027F800002055E0236E00F01F074FF00F0C0CFA75
:1028080007FC6FEA0C0623EA0C0CBEF1000F11D18D
:10281800C2F38463BB4043EA0C0323668008E36980
:1028280001309842D6D8A86AC2F38363BB400640F9
:102838003343CEE792FAA2F3B3FA83F3EAE73B49CC
:102848003B48D1F80837824203F0E07519D11B02E2
:10285800CED4D1F8083723F0E0732B4343F40003B8
:10286800C1F80837334B1A68334BB2FBF3F20C2329
:1028780002FB03330193019B002BB9D0019B013B61
:10288800F8E72E48824210D113F08070B0D1D1F809
:10289800083723F0E0732B4343F08073C1F80837FF
:1028A800002384F8543003B0F0BD254882429FD1FC
:1028B80013F480009CD1D1F8083723F0E0732B4340
:1028C80043F48003EAE7B3F1004F01BFAB6AC2F3F8
:1028D80011018B43AB62002A8ADA154813498242F8
:1028E800D1F8083709D1D1F8082703F0A07322F0EE
:1028F800E0721343C1F808377AE71048824204D1DE
:10290800D1F8082703F44003F1E70D4882427FF429
:102918006FAFD1F8082703F0C073E8E7A26D42F063
:102928002002A2651846BBE70220BCE70020014050
:10293800001000B074000020400D0300004000B8F3
:10294800002000B4026838B504461046FFF7BCFD05
:1029580008B9002038BD9368990707D4936823F015
:10296800004323F0170343F010039360FEF7C4FFFE
:10297800054623689B685B07EBD5FEF7BDFF401B48
:102988000228F6D923689B685A07F2D5A36D43F04D
:102998001003A365E36D43F00103E3650120D9E764
:1029A80073B50023026801939368DD07044602D5D6
:1029B800002002B070BD9168214B194209D0A36D67
:1029C80043F01003A365E36D43F00103E3650120C1
:1029D800EFE7936823F0004323F0170343F0010364
:1029E8009360184BD3F8083718021CD4637E012B68
:1029F800DED0FEF781FF144E054622681368DB0718
:102A0800D6D49368D9075FBF9368334043F0010376
:102A18009360FEF771FF401B0228EED923681B68FC
:102A2800DA07EAD4CBE7094B094A1B68B3FBF2F390
:102A380001330193019B002BD8D0019B013BF8E7A0
:102A48001700008000200140E8FFFF7F740000208D
:102A5800400D030038B504460068FFF735FD05460C
:102A680020BB94F85430012B20D0012384F8543033
:102A78002046FFF795FFB0B9A36D226823F4706371
:102A880023F0010343F48073A3651C23E0651360FE
:102A980084F85400936823F0004323F0170343F0AD
:102AA8000403936038BD84F85450FBE70220F9E72B
:102AB800026838B5936891680446C80701D40020B5
:102AC80038BD9907FBD4936803F00503012B19D18E
:102AD800936823F0004323F0170343F00203936045
:102AE80003231360FEF708FF054623689B68DB078E
:102AF800E5D5FEF701FF401B0228F6D923689B683D
:102B0800DA07F2D5A36D43F01003A365E36D43F034
:102B18000103E3650120D3E770B5044600284BD0D4
:102B2800836D43F002038365FFF70CFF054668B920
:102B38002046FFF7BDFF054608B90123A3652268B3
:102B4800936823F0104323F01703936023685A68AF
:102B580022F4677222F003025A6040F29F321A6030
:102B6800D968164A0A40DA601A6922F040421A61A6
:102B78005A6922F007025A611A6A02F0F0221A62B0
:102B88005A6A02F0F0225A62DA6A02F0F022DA6235
:102B98009A6A0B4A00269E62D2F8083723F0FE7321
:102BA800C2F808372046FEF7B9F9E6652666A66535
:102BB80084F85460284670BD0125FBE700023E8377
:102BC8000020014010B590F85430012B044615D070
:102BD800012380F85430FFF7B5FE58B92046FFF7B7
:102BE80067FF38B9A36D23F4807323F0010343F022
:102BF8000103A365002384F8543010BD0220FCE7CC
:102C0800F7B50023019390F85430012B04467FD088
:102C1800012380F85430FFF74BFF23689A6812F0BD
:102C28000102054607D0A36D43F01003A3650023F6
:102C380084F854302DE0A16D364F21F4817141F0B4
:102C48000201A165DE68D96826F4FF4626F07C06F5
:102C580021F40041360421F00301360CD960082024
:102C68009968394041F0004199609968002913DA60
:102C78000199013101910199B1F52E3FF5D3A36D69
:102C880023F0120343F01003A365002384F85430A3
:102C98000125284603B0F0BDD3F8B410013801F07F
:102CA8007F010A44DCD199681A48014041F00101CA
:102CB8009960D3F8B41021F07F0141EAD202C3F839
:102CC800B4209A68024042F002029A60FEF714FEAD
:102CD800074623689A68D20708D4DA683243DA606C
:102CE800A36D23F0030343F001039FE7FEF704FEFF
:102CF800C01B0228EDD923689B68D907E9D5A36DC5
:102D080043F01003A365E36D43F00103E365BFE7F8
:102D18000225BEE7E8FFFF7F0749CA6822F4E062A0
:102D28000302120403F4E063120C134343F0BF637D
:102D380043F40033CB60704700ED00E0164B30B52C
:102D4800DC68C4F30224C4F10703251D042B28BF43
:102D58000423062D4FF0FF358CBF033C002405FAF1
:102D680003F321EA0303A54022EA0502A340002851
:102D780043EA0203ACBF00F16040084A4FEA03137C
:102D8800B8BF00F00F00DBB2AABF00F561401354D2
:102D980080F8003330BD00BF00ED00E014ED00E026
:102DA800002807DB044A4109012300F01F00834083
:102DB80042F82130704700BF00E100E000280CDB3A
:102DC8004309064900F01F0020330122824041F8E0
:102DD8002320BFF34F8FBFF36F8F704700E100E0F0
:102DE80070B5D0E913456560446D14B1D0E9164556
:102DF8006560D0E9105404F01C060124B4406C60EE
:102E0800046863608368102B0BBFA260A160E16057
:102E1800E26070BD0268416CD3B210B5083B14245F
:102E2800B3FBF4F30B4CA24288BF0B4A21F0030119
:102E380099BF01F1804202F50232521807338264C9
:102E4800064AC26403F01F03012202FA03F3036572
:102E580010BD00BF070402401C0802408008024061
:102E680038B500285ED002682F4B9A424FF0140103
:102E78004CD82E4B1344B3FBF1F32D499B00C0E90A
:102E88001013022380F825301368056923F4FF43E3
:102E980023F070031360D0E9024323432B434569B1
:102EA80011682B4385692B43C5692B43056A2B435E
:102EB8000B431360FFF7AEFFB4F5804F04BF002348
:102EC80043604268816C02F07F030B60D0E9131401
:102ED800013A032A4C6020D8164A174981651A44DA
:102EE800013B9200012103F0030301FA03F30021DF
:102EF8004265C3651160114A536400230122C3630C
:102F080080F8243080F82520184638BD0C4B13442F
:102F1800B3FBF1F30B499B00B1E70023C0E915337C
:102F2800C365EAE70120F0E707040240F8FFFDBFA8
:102F3800000002403F8200104009024000090240A0
:102F4800F8FBFDBF0004024038B5002841D00268F4
:102F5800136823F0010313601F4B9A424FF01401CA
:102F680030D81E4B1344B3FBF1F31D499B00C0E955
:102F78001013012403F01C0304FA03F30025156061
:102F88004B60FFF747FF836C41681D60D0E913323F
:102F98005A604A1E032A06D8124B0B449B009440E1
:102FA8001D60114B5C640023C363C0E91533C0E99D
:102FB8000B33C0E90D33C36580F8253080F8243021
:102FC800184638BD094B1344B3FBF1F308499B007D
:102FD800CDE70120F5E700BF07040240F8FFFDBF79
:102FE800000002403F82001000090240F8FBFDBFCC
:102FF8000004024070B590F82450012D04463BD0DF
:1030080090F825600125AE4280F824504FF0000664
:103018002CD1022580F825500568C6632E6826F055
:1030280001062E60FFF7DCFE036BBBB12B6843F093
:103038000E032B60A36C1A68D20342BF1A6842F4CD
:1030480080721A60636D1BB11A6842F480721A604C
:103058002B6843F001032B60002070BD2B6823F020
:1030680004032B602B6843F00A03E2E78023C36361
:1030780080F824602846F0E70220EEE7034640B1D6
:1030880090F82520022A06D00422C263002280F884
:103098002420012070470268806C116821F00E011D
:1030A8001160016821F480710160116821F001014B
:1030B8001160D3E9100202F01C0101228A4042602B
:1030C800D3E9132151605A6D32B1116821F480712E
:1030D8001160D3E9162151600122002083F82520D0
:1030E80083F82400704710B590F82530022B03D0E0
:1030F8000423C363012010BD03681A6822F00E027E
:103108001A601A6822F001021A60826C136823F4AC
:1031180080731360D0E9101303F01C02012393405D
:103128004B60D0E913325A60436D33B11A6822F408
:1031380080721A60D0E916325A60012380F825306F
:10314800836B002480F8244013B198472046D2E7C7
:103158001846D0E770B4426C046C036826681D6892
:1031680002F01C020421914031420FD015F0040FE7
:103178000CD01A6892065EBF1A6822F004021A6020
:10318800036B6160002B33D070BC1847022191405B
:10319800314217D015F0020F14D01A68940606D4DD
:1031A8001A6822F00A021A60012280F82520114AC2
:1031B80093428CBF104B114B5960002380F8243088
:1031C800C36ADFE708219140314211D029070FD5A2
:1031D800196821F00E011960012303FA02F26260F6
:1031E800C36380F82530002380F82430436BC9E797
:1031F80070BC70478000024000040240000002409A
:103208000A4A536943F4802330B55361EFF31084BD
:1032180072B60023CD58C5500433B3F5807FF9D179
:103228001369DB03FCD484F3108830BD00400058D8
:10323800064B5A69002ABFBF054A9A6002F18832D4
:103248009A60BABF5869C00F002070470040005804
:1032580023016745044B5A6942F000425A61586994
:10326800C043C00F704700BF0040005870B5054606
:10327800FEF742FB124E04463369D90313D433696F
:10328800DA0744BF012232614CF2FA32134011D1FD
:103298000B4E306910F480200BD0FEF72DFB001B7D
:1032A800A842F6D304E0FEF727FB001BA842E3D3AD
:1032B800032070BD024A1361024A01205360F8E7F7
:1032C80000400058500400202DE9F041184D984660
:1032D8002B78012B06460C46174626D001232B7067
:1032E8004FF47A7000236B60FFF7C0FFA0B9012E7E
:1032F80016D1104A536943F0010353612760BFF3A5
:103308006F8FC4F804804FF47A70FFF7AFFF094A53
:10331800536923EA0603536100232B70BDE8F0814B
:1033280039462046FFF76CFFEDE70220F6E700BFBD
:103338005004002000400058054A536923F47E7366
:1033480043EAC00040F4803040F00200506170470A
:10335800004000582DE9F041234F3B78012B0546EA
:1033680088463FD001233B704FF47A7000237B607E
:10337800FFF77CFF044688B92B68042B13D11B4A3E
:10338800536943F4803343F0040353614FF47A7074
:10339800FFF76CFF0446154B1A681B6800233B7047
:1033A8002046BDE8F0814FF0FF33C8F800306E6862
:1033B800D5E901321344B3420AD93046FFF7BCFFBE
:1033C8004FF47A70FFF752FF50B1C8F80060044616
:1033D800064A536923F47E7323F002035361DAE744
:1033E8000136E5E70224DBE75004002000400058DE
:1033F8002DE9F04F524C00234FF00F090A6832FABA
:1034080003F501D1BDE8F08F012505FA03F818EAA4
:10341800020200F08E804E68032706F003054FEA8B
:10342800430E07FA0EFC6F1E012F6FEA0C0C32D800
:10343800876807EA0C0ACF6807FA0EF747EA0A070F
:103448008760476827EA0808C6F300179F4047EADD
:1034580008074760C76807EA0C088F6807FA0EF77D
:1034680047EA0807022DC76017D14FEAD30800EBD7
:10347800880803F0070AD8F820704FEA8A0A09FA80
:103488000AFB27EA0B0B0F6907FA0AF747EA0B074B
:10349800C8F8207001E0032DDCD1076805FA0EF5A5
:1034A80007EA0C073D4316F4403F056041D023F07E
:1034B800030707F1804707F5803703F0030CBD6861
:1034C8004FEA8C0C4FF0070E0EFA0CFEB0F1904F3D
:1034D80025EA0E0E2FD01B4DA8422ED005F580658B
:1034E800A8420CBF0225072505FA0CF545EA0E058A
:1034F800BD602568D74316F4801F0CBF3D401543B7
:103508002560656816F4001F0CBF3D4015436560D3
:10351800D4F8805016F4803F0CBF3D401543C4F8E2
:103528008050D4F88450B60354BF3D401543C4F8C6
:103538008450013362E70025D6E70125D4E700BFB0
:103548000008005800040048374A2DE9F04F0023CE
:103558004FF0010A4FF0070B4FF00F0931FA03F44F
:1035680001D1BDE8F08F0AFA03FC1CEA010654D029
:1035780023F0030404F1804404F5803403F00307C6
:10358800A568BF000BFA07F8B0F1904F08EA050EDE
:1035980045D0264DA84244D005F58065A8420CBF09
:1035A80002250725BD40754517D1D2F8805025EA78
:1035B8000605C2F88050D2F8845025EA0605C2F8FC
:1035C8008450156825EA06051560556825EA06053C
:1035D8005560A56825EA0805A560056803265C000E
:1035E80006FA04F423FA06F6254300EB860605607E
:1035F80003F00705376AAD0009FA05F527EA05075C
:103608003762856825EA04058560456825EA0C0562
:103618004560C56825EA0404C46001339EE70025B7
:10362800C0E70125BEE700BF0008005800040048B5
:103638000AB18161704781627047436901EA0302F8
:1036480021EA030141EA024181617047044AD168D5
:10365800014208B502D0D060FEF74EFE08BD00BF9B
:1036680000080058024A136843F4807313607047D7
:10367800000400580D4B10B55B690C4628B99A0533
:1036880007D500F039F820B110BD9B0501D400F032
:103698002BF8074A1369012C23F00403136101D1A5
:1036A80030BFF1E740BF20BF20BFEDE7000400585E
:1036B80000ED00E0064A136823F0070343F0030314
:1036C8001360044A136943F00403136130BF704761
:1036D8000004005800ED00E0024B186800F4C060D8
:1036E800704700BF00040058024A136843F480433F
:1036F80013607047000400580C4A136823F4804391
:1037080013600B4B1B6832214B430A49B3FBF1F39F
:103718005169890500D533B9536913F4007F14BF83
:10372800032000207047013BF2E700BF0004005867
:103738007400002040420F000B4A136823F007036F
:1037480043F002031360094B1A69012842F004028E
:103758001A6105D130BF1A6922F004021A61704754
:1037680040BF20BF20BFF6E70004005800ED00E08E
:103778004FF0B0431868C0F3404070474FF0B04373
:103788001868C0F3400070474FF0B042536823F404
:103798007F4343EA0023536070474FF0B0431868F3
:1037A800C0F34060704700007FB54FF0B0432C4A2B
:1037B800D3F80831C0F3031003F00F0352F8204088
:1037C800284A52F82330B4FBF3F4FFF785FF264B61
:1037D800054693E80700B5F5007F04AB03E9070049
:1037E80010D0224B9C4218D303F5B70303F67F533E
:1037F8009C4229D903F5741303F510639C4225D81C
:1038080002230BE01A4B9C4207D91A4B9C421BD946
:1038180003F5370303F5D853F0E7002304AA02EBB6
:10382800830353F80C4C144D2B6823F007032343F0
:103838002B60FEF761F806462B6803F007039C42ED
:1038480006D1002004B070BD0123E7E70024EAE7B1
:10385800FEF752F8801B0228EED90320F2E700BFDA
:1038680030F20008D0F10008E8F00008C0CF6A0084
:10387800BFEA21013F933402004000584FF0B043A3
:1038880010B59A68D96812F00C0205D00C2A4AD1F2
:1038980001F00303012B50D14FF0B0412B480B68C6
:1038A80013F0080306D00B6813F0080337D1D1F8DA
:1038B800941007E00C68240756BFD1F894300968C3
:1038C800C3F3032350F82330002A0CBF1846002006
:1038D8004FF0B0418A6802F00C020C2A1ED1CA6867
:1038E80002F00302022A2ED0032A06D10B68184AD6
:1038F80013F4801F174B18BF13464FF0B042D0681F
:10390800D168D268C0F306205843C1F302130133CB
:10391800B0FBF3F0530F0133B0FBF3F010BD0B68AD
:10392800C3F30313CEE7042A0AD0082A05D11B687B
:1039380013F4801304D10748CAE700231846C7E7E1
:1039480003480023C4E7024BD7E700BF30F2000862
:103958000024F4000048E80108B5FFF78FFF4FF096
:10396800B043044A9B68C3F3031352F82330B0FBF7
:10397800F3F008BDD0F100082DE9F0410446002815
:1039880053D04FF0B0439D68DE6803689B0605F08E
:103998000C0506F0030668D5026A1DB10C2D46D148
:1039A800012E44D1002A40D04FF0B043A16A1A68D2
:1039B800170756BFD3F894301B681B0903F0F003B0
:1039C80099421FD90846FFF7EFFE00282DD14FF086
:1039D800B042136843F0080313601368A16A23F028
:1039E800F0030B431360606AFFF7CEFEFFF7B4FFE6
:1039F800AB4B1860AB4B1868FDF77CFF002834D040
:103A0800BDE8F0814FF0B042136843F0080313603B
:103A1800136823F0F0030B431360606AFFF7B4FEEA
:103A28000846FFF7C1FE0028E0D00120E8E74FF084
:103A3800B043002A54D01A6842F001021A60FDF718
:103A48005BFF0746FFF79AFE002842D04FF0B042CE
:103A5800136843F0080313601368A16A23F0F003A6
:103A68000B431360606AFFF78FFE2368D80748D4BA
:103A78002368990700F18C8023681E0740F1FA80BB
:103A8800A3694FF0B046002B00F0E180D6F89430DF
:103A9800E16903F01002914200F0C48003F00302D0
:103AA800022AC2D0D80740F1B380D6F8943023F068
:103AB8000103C6F89430FDF71FFF0746D6F8943087
:103AC800990740F1A580FDF717FFC31B112BF5D906
:103AD80004E0FDF711FFC01B0228B3D903208FE7CC
:103AE8001A6822F001021A60FDF706FF0746FFF781
:103AF80045FE0028B9D0FDF7FFFEC01B0228F6D905
:103B0800ECE7082D03D00C2D05D1032E03D16368F3
:103B1800002BADD189E74FF0B043A1681A6822F4B1
:103B280080120A431A606268B2F5803F10D11A68A1
:103B380042F480321A60FDF7DFFE0746FFF718FEF1
:103B4800002895D1FDF7D8FEC01B6428F6D9C5E733
:103B5800B2F5041F04D11A6842F400121A60E6E7AD
:103B6800196821F480311960196821F4001119606D
:103B7800002AE0D1FDF7C0FE0746FFF7F9FD00284F
:103B88003FF476AFFDF7B8FEC01B6428F5D9A5E76A
:103B9800042D236903D00C2D0ED1022E0CD1002B3D
:103BA8003FF443AF4FF0B0426169536823F0FE43DE
:103BB80043EA016353605FE74FF0B046BBB1336837
:103BC80043F480733360FDF797FE074633685A0560
:103BD80007D57368626923F0FE4343EA02637360A2
:103BE8004AE7FDF789FEC31B022BEFD976E7336856
:103BF80023F480733360FDF77FFE074633685B0567
:103C08007FF53AAFFDF778FEC31B022BF6D965E7BF
:103C18004FF0B042E169D2F8943023F010030B431F
:103C2800C2F894304FF0B047D7F8943043F001030E
:103C3800C7F89430FDF760FE0646D7F894309A0727
:103C480018D4FDF759FE831B112BF6D946E7D6F891
:103C5800943023F00103C6F89430FDF74DFE074673
:103C6800D6F894309B0705D5FDF746FEC31B112BEC
:103C7800F6D933E72368580754D50B4F3B68D90565
:103C880014D4FFF7EFFCFDF737FE06463B68DA056C
:103C98000CD4FDF731FE831B022BF7D91EE700BFBA
:103CA800740000207800002000040058E3684FF0FA
:103CB800B046002B58D023F08003052B02BFD6F85E
:103CC800903043F00403C6F890304FF0B046FDF74B
:103CD80013FED6F8903043F001030746C6F890303B
:103CE80041F28838D6F890309B0705D4FDF704FEDA
:103CF800C31B4345F6D9F1E6E36823F00403812B9F
:103D08001BD1FDF7F9FDD6F8903043F08003C6F8D3
:103D1800903007464FF0B04641F28838D6F89030D8
:103D2800180504D5E06A00284AD1002068E6FDF7A6
:103D3800E3FDC01B4045F1D9D0E6FDF7DDFDD6F81F
:103D4800903023F08003C6F8903007464FF0B04615
:103D580041F28838D6F890301905E3D5FDF7CCFD47
:103D6800C01B4045F6D9B9E6FDF7C6FDD6F8903038
:103D780023F080030746C6F8903041F28838D6F819
:103D880090301A0516D4FDF7B7FDD6F8903023F019
:103D98000103C6F8903007464FF0B04841F2883624
:103DA800D8F890309B07BDD5FDF7A6FDC31BB342DD
:103DB800F6D993E6FDF7A0FDC01B4045DFD98DE697
:103DC8000C2D4ED04FF0B04302281A6822F08072B2
:103DD8001A6033D1FDF790FD0546FFF7DEFC38BBCE
:103DE800D4E90C314FF0B0420B43D0682D49014063
:103DF8000B43E16B0B43216C0B43616C0B43A16BD1
:103E080043EA0123D360136843F080731360D368D7
:103E180043F08053D360FDF76FFD0446FFF7BDFC08
:103E2800002882D1FDF768FD001B0A28F6D955E65F
:103E3800FDF762FD401B0A28CFD94FE6FDF75CFD70
:103E48000446FFF7AAFC30B94FF0B042164BD168D0
:103E58000B40D360D4E5FDF74FFD001B0A28F0D9CD
:103E68003CE601283FF4CCAD4FF0B043226BDB6851
:103E780003F0030191427FF4D8AD616B03F0700247
:103E88008A427FF4D2ADA16B03F4FE42B2EB012F5C
:103E98007FF4CBAD626C03F0604393423FF445AFCF
:103EA800C3E500BF8C80C111FCFFFEEE2DE9F04197
:103EB8000D46044610B90120BDE8F081684E33680C
:103EC80003F007038B4216D323689A0727D54FF0D0
:103ED800B047A268BB6823F0F0031343BB60FDF74B
:103EE8000BFD0646BB68DB0319D4FDF705FD831BF4
:103EF800022BF7D911E0336823F007030B43336033
:103F0800FDF7FAFC0746336803F00703AB42DBD042
:103F1800FDF7F2FCC01B0228F5D90320CCE7236883
:103F2800580617D54FF0B0476269D7F8083123F023
:103F38000F0343EA1213C7F80831FDF7DDFC064604
:103F4800D7F80831D90305D4FDF7D6FC831B022B1B
:103F5800F6D9E2E723685A0713D54FF0B047E2686D
:103F6800BB6823F4E0631343BB60FDF7C5FC06465A
:103F7800BB689B0305D4FDF7BFFC831B022BF7D955
:103F8800CBE72368180714D54FF0B0472269BB6800
:103F980023F4605343EAC203BB60FDF7ADFC064659
:103FA800BB68590305D4FDF7A7FC831B022BF7D97F
:103FB800B3E72368DA070FD4294C236803F0070313
:103FC800AB4239D8FFF7C8FC264B1860264BBDE832
:103FD800F0411868FDF78EBC6268022A1DD1FFF710
:103FE800C7FB00283FF467AF4FF0B04641F288386E
:103FF800B36823F003031343B360FDF77DFC074662
:10400800B368626803F00C03B3EB820FD4D0FDF7FA
:1040180073FCC01B4045F3D97FE7032A02D1FFF7A1
:10402800BCFBDEE712B9FFF7A9FBDAE74FF0B043B4
:104038001B685B05D8D43EE7236823F007032B43AE
:104048002360FDF759FC0646236803F00703AB42DB
:10405800B8D0FDF751FC801B0228F5D95DE700BFF9
:1040680000400058740000207800002008B5FFF7D1
:1040780073FC4FF0B043044A9B68C3F3022352F821
:104088002330D84008BD00BF10F2000808B5FFF77C
:1040980063FC4FF0B043044A9B68C3F3C22352F851
:1040A8002330D84008BD00BF10F200084FF0B043DD
:1040B800D3F89000C0F3400070474FF0B0410209B8
:1040C800D1F8883002F47F22000123EA020300F4C9
:1040D8007F200343C1F8883070474FF0B041020C8D
:1040E800D1F88830120423EA020343EA0040C1F8F9
:1040F8008800704770B5066816F48036044638D0D4
:10410800FFF7B0FAFDF7F8FB614E05463368DB05AB
:1041180029D54FF0B043616BD3F8902002F4407278
:10412800914214D0D3F89010D3F8902042F4803202
:10413800C3F89020D3F8902021F4407022F4803204
:104148008D07C3F89020C3F8900000F190804FF0DD
:10415800B042616BD2F8903023F440730B43C2F83D
:104168009030002605E0FDF7C7FB401B0228CDD99B
:1041780003262568E8070AD54FF0B0416268D1F8F0
:10418800883023EA124392B21343C1F88830A90752
:104198000AD54FF0B041A268D1F8883023EA12431B
:1041A80092B21343C1F88830AA0609D54FF0B0423D
:1041B8002169D2F8883023F440630B43C2F8883071
:1041C800AB0502D5206AFFF788FF680502D5606A4B
:1041D800FFF783FF290502D5A06AFFF77EFF6A066D
:1041E80002D56069FFF769FF2B0602D5A069FFF7C2
:1041F80064FFE80502D5E069FFF75FFFE90610D51F
:104208004FF0B042E168D2F8883023F440730B4392
:10421800C2F88830B1F5807F02BFD36843F080735D
:10422800D3602A040ED54FF0B042216BD2F8883003
:1042380023F040430B43C2F8883019B9D36843F0E0
:104248008073D3606B0410D54FF0B042E16AD2F8A6
:10425800883023F040530B43B1F1005FC2F8883037
:1042680003D1D36843F48033D360304670BDFDF783
:1042780043FB41F288360546FFF718FF01283FF453
:1042880066AFFDF739FB401BB042F5D970E700BFB8
:104298000004005830B590F82C30012B02464FF03E
:1042A800020022D0174B82F82D00CA24012582F87B
:1042B8002C505C6253245C62B1F5807F146B996961
:1042C80014D121F488519961596C24F0010421F02A
:1042D800004159641463DD650A4BFF2159620020CF
:1042E800012382F82D3082F82C0030BD21F40851CA
:1042F8009961D96C24F0020421F00041D964146357
:10430800D865E9E70028004070B50B4E036B756D62
:104318001D40EA07044603D50123F365FDF7FFFBBB
:10432800AB0704D50223F365204600F0CBF901233F
:1043380084F82D3070BD00BF0028004038B50A4C05
:10434800E36823F02003E360FDF7D6FA0546E36847
:104358009B0601D5002038BDFDF7CEFA401BB0F50D
:104368007A7FF4D90320F6E7002800402DE9F041D0
:10437800114DEC6814F0400407461AD1EB6843F07D
:104388008003EB60FDF7B8FA4FF003080646EB68C8
:104398005B0601D4032C02D12046BDE8F081FDF76D
:1043A800ABFA801BB0F57A7F84BF87F82D80032491
:1043B800EDE70024F0E700BF0028004038B50F4CB7
:1043C800E36823F08003E360A3699B06054606D4EF
:1043D800FFF7B4FF10B1032085F82D0038BDA3699D
:1043E80023F02003A361FFF7A9FF10B1032085F88C
:1043F8002D00A36943F02003A361EFE700280040E4
:1044080038B5044600284BD090F82D3003F0FF0251
:104418001BB980F82C20FDF7C7F80223214D84F83A
:104428002D30EB68DB0632D4CA236B6253236B62F0
:104438002046FFF79BFF78BBAB6923F08E6323F020
:104448004003AB6121696368AA690B431343A269FE
:104458001343AB61D4E9022343EA02432B61D4E955
:104468000931EA680B4322F4F8521343EB60204603
:10447800FFF7A4FF80B9D4E90713AA690B4322F018
:104488006042134362691343AB61FF236B620123EC
:1044980084F82D30002002E0024BFF225A6238BD1A
:1044A8000120FCE7002800400023092803D840EA3F
:1044B8000310C0B270470A380133C0B2F5E70000F4
:1044C8002DE9F04790F82C30012B05464FF00200FB
:1044D80069D0012385F82C304E4B85F82D00DE6815
:1044E80006F44076B6F5807F78D04C69087891F864
:1044F800019091F802A091F82470002A55D19B6987
:1045080013F0400308BFCB70FFF7CEFF8046484644
:10451800FFF7CAFF02465046FFF7C6FF81463846F6
:10452800FFF7C2FF0B6ACF78234343EA875343EA76
:10453800090343EA084343EA022343EA0063354A8E
:10454800CA205062532050628C6A8869B4F5807F13
:10455800946945D124F4885494610124D465B6F54E
:10456800807F09BFCB6913640343536418BF506449
:10457800284B4A681A672A6B42F001022A639A6933
:1045880042F488529A61244AD2F8803043F40033C6
:10459800C2F880301F4BFF225A620020012385F8A1
:1045A8002D3085F82C00BDE8F087B4F1803F07D0A6
:1045B800B4F5000F04D09B6913F0400308BFCB701B
:1045C8000B6ACA781C4344EA0A0444EA004343EAF3
:1045D800092343EA825343EA0763B0E70023AEE7BF
:1045E80024F4085494610224D465B6F5807F09BF89
:1045F800CB6993640343D36418BFD064054B4A68FE
:104608005A672A6B42F002022A639A6942F40852F6
:10461800B8E700BF002800400008005890F82C2098
:10462800012A03464FF0020012D00A4A83F82D00EF
:10463800CA21516253215162916941F0200191616F
:10464800FF2151620020012283F82D2083F82C00DD
:10465800704700BF0028004090F82C20012A03462C
:104668004FF0020019D00D4A83F82D00CA2151627B
:104678005321516291690A4841F080019161D0F853
:10468800801041F48021C0F88010FF215162002081
:10469800012283F82D2083F82C0070470028004061
:1046A80000080058064B5A6D520610B5044603D54B
:1046B8004022DA65FDF736FA012384F82D3010BD63
:1046C800002800407047890001F1804101F531411F
:1046D8000A607047890001F1804101F5314108689D
:1046E80070470000034AD2F8903043F40043C2F800
:1046F8009030704700040058034AD2F8903023F4F1
:104708000043C2F89030704700040058074B1A68FD
:1047180022F040021A6040F441704FF4B852186019
:104728005A601A6842F040021A6070470000015847
:1047380037B5054600284ED0837903F0FF046BB1E6
:10474800032C0BD0254B4FF400629A612868FFF7C1
:10475800DDFF002401232B71AC602FE000236B7177
:104768002846FCF7E3FF1E4AD2F8903043F4805302
:10477800C2F89030002CE5D102234FF0B042AB7163
:10478800D2F8943023F40043C2F89430154B1B68D8
:104798001C214B43DB0C64214B430193019B93B9D0
:1047A8000124AC60FFF79EFF0C4B9A6842F400624C
:1047B8009A604FF400629A61002CC7D00123AB7154
:1047C800204603B030BD019B013B0193D2F89430E1
:1047D8005B04E3D4E6E70124F2E700BF00040058D5
:1047E800000800587400002037B5174D2B680246A2
:1047F8001C204343DB0C6420434314480193019B72
:1048080093B901209060114C21732B681C214B43F4
:10481800DB0C64214B430193019B6BB90120906031
:104828000A4BDB6803B030BD019B013B01938368F1
:104838009C07E4D50020E6E7019B013B0193A368B0
:10484800DB07E9D5ECE700BF740000200000015841
:1048580037B5184D2B6802461C204343DB0C6420F7
:10486800434315480193019BA3B901209060124C62
:10487800FF2323732B681C256B43DB0C64256B43D8
:104888000193019B73B9012090600B4BDB680B709F
:1048980003B030BD019B013B019383689C07E2D5BF
:1048A8000020E4E7019B013B0193A368DB07E8D5FF
:1048B800EBE700BF74000020000001580F4B13B550
:1048C8001B680F4C182253431B0D642253430146A7
:1048D80001936269019B02F0040223B902238B60F1
:1048E800012002B010BD019B013B0193606910F0EB
:1048F8000200F6D0002AECD11046F2E7740000203E
:104908000004005807B50379012B0FD10A4B1B6827
:10491800182253431B0C0193FFF7EEFE019B013B4A
:104928000193019B002BF9D1FFF7DCFE03B05DF882
:1049380004EBFFF7C3BF00BF74000020F8B51E46A4
:104948008379012B154604460F46DAB22DD14379F7
:10495800012B2AD0022342718371FFF7D3FF0D2167
:104968002046FFF7C9FEFFF73FFF390A2046FFF749
:104978003BFFF9B22046FFF737FF2E44B5420ED170
:104988002046FFF7AFFEFFF799FFA0680123003824
:10499800A3714FF0000318BF01206371F8BD15F82B
:1049A800011B2046FFF720FFE8E70220F6E7F8B5ED
:1049B8001E468379012B154604460F46DAB22FD1DD
:1049C8004379012B2CD04271FFF79CFF1D21204613
:1049D800FFF792FEFFF708FF390A2046FFF704FFAA
:1049E800F9B22046FFF700FF00212046FFF7FCFE42
:1049F8002E44B5420ED12046FFF774FEFFF75EFF46
:104A0800A06801230038A3714FF0000318BF0120EC
:104A18006371F8BD29462046FFF71AFF0135E8E71C
:104A28000220F6E7F8B51F468379012B15460446A0
:104A38000E46DAB22CD14379012B29D04271FFF707
:104A480061FF06F0EF03A3F184025342534123713F
:104A580031462046FFF750FEFFF7C6FE2F44AF420F
:104A680010D1FFF73FFE842E02D02046FFF726FF25
:104A7800A06801230038A3714FF0000318BF01207C
:104A88006371F8BD15F8011B2046FFF7ADFEE6E798
:104A98000220F6E7F8B51E468379012B1546044631
:104AA8000F46DAB227D14379012B24D04271FFF7A0
:104AB80029FF39462046FFF71FFEFFF795FE002124
:104AC8002046FFF791FE2E44B5420ED12046FFF74F
:104AD80009FEFFF7F3FEA06801230038A3714FF029
:104AE800000318BF01206371F8BD29462046FFF76F
:104AF800AFFE0135E8E70220F6E737B50023ADF849
:104B0800043001AA022312210546FFF7C3FFBDF8AE
:104B18000440022364BA01AAA4B219462846FFF742
:104B280081FFE20702D5284609F088FBA30702D5D2
:104B3800284609F089FB600702D5284609F0AEFB34
:104B4800210702D5284609F0AFFBE20602D5284620
:104B580009F0B0FBA30602D5284609F099FB6006C8
:104B680002D5284609F076FB210606D514F4807193
:104B780018BF0121284609F073FBA20502D5284673
:104B880009F07EFB630402D5284609F099FB03B0BF
:104B980030BDF8B51E468379012B154604460F46ED
:104BA800DAB227D14379012B24D04271FFF7AAFE4C
:104BB8000E212046FFF7A0FDFFF716FE39462046D6
:104BC800FFF712FE2E44B5420ED12046FFF78AFDAC
:104BD800FFF774FEA06801230038A3714FF00003AB
:104BE80018BF01206371F8BD15F8011B2046FFF7B7
:104BF800FBFDE8E70220F6E7F8B51E468379012BAE
:104C0800154604460F46DAB22BD14379012B28D03A
:104C18004271FFF777FE1E212046FFF76DFDFFF773
:104C2800E3FD39462046FFF7DFFD00212046FFF768
:104C3800DBFD2E44B5420ED12046FFF753FDFFF7AA
:104C48003DFEA06801230038A3714FF0000318BF90
:104C580001206371F8BD29462046FFF7F9FD0135AB
:104C6800E8E70220F6E7026852E8003F23F0C003B5
:104C780042E8003102680029F5D102F1080353E83F
:104C8800003F23F4000302F1080C4CE8003100292E
:104C9800F3D12023C0F888307047000010B50268AF
:104CA80052E8003F23F4907342E80031026800297B
:104CB800F5D10F4C02F1080353E8003F234002F1FD
:104CC800080C4CE800310029F4D1C36E012B07D140
:104CD80052E8003F23F0100342E800310029F7D1E1
:104CE8002023C0F88C300023C366436710BD00BF83
:104CF800FEFFFFEF38B50546C8B12423C0F8883059
:104D080003681A68002422F001021A601C605C60C3
:104D18009C60FCF7B3FFC5F8904085F88440C5F85F
:104D280088402046C5F88C40EC662C6738BD0120C9
:104D3800FCE70000F8B504461346D4F88850202D47
:104D480032D1F1B1EAB1E06FA4F85620A4F85420AA
:104D580000262122C4F890602165C4F888202268C2
:104D680088B1124FC762124F0763124F2832C0E949
:104D78000D76FEF73FF930B11023C4F89030C4F82F
:104D8800885001200FE0236840221A62226802F14D
:104D9800080353E8003F43F0800302F1080141E8AB
:104DA80000300028F3D1F8BD0220FCE7C14D00080F
:104DB800094E0008154E000808B50346806A1B68AE
:104DC8001B6813F0200317D1A0F85630026802F1CF
:104DD800080353E8003F23F08003083242E800311B
:104DE80002680029F2D152E8003F43F0400342E84C
:104DF80000310029F7D108BDFCF7BAFFFBE770477F
:104E080008B5806AFFF7FBFF08BD7047806A38B5B0
:104E18000468D0F88830D0F88C50A268120606D5FD
:104E2800212B04D10023A0F85630FFF71CFFA368FC
:104E38005B0606D5222D04D10023A0F85E30FFF7CB
:104E48002DFFD0F8903043F01003C0F89030FFF7F2
:104E5800DCFF38BD08B5806A0023A0F85E30A0F8F2
:104E68005630FFF7D2FF08BD704700000368D969C4
:104E78001A682DE9F04140F60F0631429D68044654
:104E880010D18E0640F1978002F0200605F0805779
:104E98003E4300F09080436F002B00F08580BDE812
:104EA800F0411847AB4EAC482E401040304300F05C
:104EB8008280CF0709D5D00507D501201862D4F81C
:104EC800900040F00100C4F890008F0709D5E8076A
:104ED80007D502201862D4F8900040F00400C4F806
:104EE80090004F0709D5E80707D504201862D4F8C1
:104EF800900040F00200C4F890000F070BD502F0B4
:104F08002000304307D008201862D4F8900040F001
:104F18000800C4F890000E050AD5500108D54FF4D2
:104F280000601862D4F8903043F02003C4F8903041
:104F3800D4F89030002B37D08B0609D502F0200228
:104F480005F080552A4303D0636F0BB1204698477C
:104F58002668D4F89020B36802F0280203F04003D2
:104F680053EA0205204621D0FFF798FEB3685F0692
:104F780017D5226802F1080353E8003F23F04003E5
:104F8800083242E800310029F3D1D4F8800040B15A
:104F9800724B8363FEF7A7F830B1D4F88000836BB7
:104FA8007DE72046FFF731FFBDE8F081FFF72DFFD1
:104FB800C4F89050F8E7E06E012840F08980CE06EA
:104FC80040F18680D00640F1838010221A629A68E8
:104FD80051064BD5D4F8802011684A6892B2002A4D
:104FE800E2D0B4F85C009042DED9A4F85E200A68EA
:104FF80092062FD453E8002F22F4807243E8002150
:105008000029F7D103F1080252E8002F22F001022B
:1050180003F1080040E800210029F3D103F1080258
:1050280052E8002F22F0400203F1080040E8002176
:105038000029F3D12022C4F88C20E16653E8002F20
:1050480022F0100243E800210029F7D1D4F88000AB
:10505800FEF714F802232367B4F85E30B4F85C1046
:10506800C91A89B22046FFF7FFFE9DE7B4F85E2013
:10507800B4F85E00B4F85C1080B292B2002893D005
:10508800891A89B200298FD053E8002F22F4907230
:1050980043E800200028F7D1314D03F1080252E817
:1050A800002F2A4003F1080646E800200028F4D122
:1050B8002022C4F88C206067E06653E8002F22F0B5
:1050C800100243E800200028F7D102232367C9E72C
:1050D800CF0209D56E0207D54FF4801220461A6216
:1050E800BDE8F04100F0A0BD08060BD502F0800035
:1050F80005F40005284305D0A36F002B3FF454AFF7
:105108002046CCE64F0611D556060FD553E8002F9A
:1051180022F0400243E800210029F7D12023C4F8F7
:105128008830A1672046FCF723FE3DE70D0206D52F
:10513800500004D52046BDE8F04100F077BDCB0112
:105148007FF532AF002ABFF62FAF2046BDE8F04109
:1051580000F06BBD01000010200100045D4E000846
:10516800FEFFFFEFD0F88C20B0F86010222A08B5B7
:10517800036855D15B6A826D0B401370836D0133F0
:105188008365B0F85E30013B9BB2A0F85E30B0F8A2
:105198005E309BB2002B42D1026852E8003F23F4F4
:1051A800907342E8003103680029F5D103F1080241
:1051B80052E8002F22F0010203F1080C4CE800210C
:1051C8000029F3D12022C0F88C20184A4167934265
:1051D800016705D1C26E012A0ED0FCF7D7FD1EE08B
:1051E8005A681102F6D553E8002F22F0806243E88E
:1051F80000210029F7D1EDE70022C26653E8002F0D
:1052080022F0100243E800210029F7D1DA69B0F84A
:105218005C10D20644BF10221A62FFF725FE08BDB3
:105228009A6942F008029A61F9E700BF00800040DD
:10523800D0F88C20B0F86010222A08B5036852D143
:105248005A6A1140826D22F8021B8265B0F85E200E
:10525800013A92B2A0F85E20B0F85E2092B2002A1D
:1052680040D153E8002F22F4907243E8002100292E
:10527800F7D103F1080252E8002F22F0010203F1EE
:10528800080C4CE800210029F3D12022C0F88C201A
:10529800174A41679342016705D1C26E012A0ED0B1
:1052A800FCF774FD1EE05A681102F6D553E8002F8A
:1052B80022F0806243E800210029F7D1EDE70022BF
:1052C800C26653E8002F22F0100243E800210029AB
:1052D800F7D1DA69B0F85C10D20644BF10221A621E
:1052E800FFF7C2FD08BD9A6942F008029A61F9E722
:1052F800008000402DE9F74F0368B0F86080DF694F
:105308001A689D68D0F88C1001922229044640F052
:10531800B480B0F86890DFF86CA1DFF86CB10026B3
:10532800B9F1000F01D0BB0621D4B4F85E309BB2AE
:10533800D3B1B4F868209A4216D9226802F108035A
:1053480053E8003F23F08053083242E800312268D6
:105358000029F2D14D4B636752E8003F43F0200328
:1053680042E800310029F7D103B0BDE8F08F236887
:10537800A26D5B6A03EA08031370A36D0133A3658A
:10538800B4F85E30013B9BB2A4F85E302368DF6955
:1053980078072CD0F9070AD5019AD20507D501213B
:1053A8001962D4F8901041F00101C4F89010B807C0
:1053B80009D5E90707D502211962D4F8901041F000
:1053C8000401C4F890107A0709D5E80707D5042125
:1053D8001962D4F8903043F00203C4F89030D4F83E
:1053E800903023B12046FFF710FDC4F89060B4F860
:1053F8005E309BB2002B93D1216851E8003F23F423
:10540800807341E8003023680028F5D103F10802D1
:1054180052E8001F01EA0A0142E800100028F5D10D
:1054280020215B45C4F88C10606720670AD0596852
:10543800090207D553E8001F21F0806143E80010F6
:105448000028F7D1E16E012913D1E66653E8001F61
:1054580021F0100143E800100028F7D1D969CA06E5
:1054680044BF102119622046B4F85C10FFF7FCFC19
:1054780056E72046FCF78AFC52E79A6942F0080290
:105488009A6171E7FEFFFFEF008000406D51000850
:105498002DE9F74F0368B0F86080DF691A689D68E6
:1054A800D0F88C1001922229044640F0B280B0F85E
:1054B8006890DFF868A1DFF868B10026B9F1000F3D
:1054C80001D0BB0621D4B4F85E309BB2D3B1B4F896
:1054D80068209A4216D9226802F1080353E8003F6F
:1054E80023F08053083242E8003122680029F2D1C3
:1054F8004C4B636752E8003F43F0200342E8003119
:105508000029F7D103B0BDE8F08F2368A26D596A6E
:1055180008EA010122F8021BA265B4F85E20013AEC
:1055280092B2A4F85E20DF6978072CD0F9070AD573
:10553800019AD20507D501211962D4F8901041F0DB
:105548000101C4F89010B80709D5E90707D5022169
:105558001962D4F8901041F00401C4F890107A0749
:1055680009D5E80707D504211962D4F8903043F02B
:105578000203C4F89030D4F8903023B12046FFF7E6
:1055880044FCC4F89060B4F85E309BB2002B95D10F
:10559800216851E8003F23F4807341E80030236814
:1055A8000028F5D103F1080252E8001F01EA0A01B8
:1055B80042E800100028F5D120215B45C4F88C1082
:1055C800606720670AD05968090207D553E8001FA9
:1055D80021F0806143E800100028F7D1E16E01292D
:1055E80013D1E66653E8001F21F0100143E80010CC
:1055F8000028F7D1D969CA0644BF1021196220468C
:10560800B4F85C10FFF730FC58E72046FCF7BEFB07
:1056180054E79A6942F008029A6173E7FEFFFFEFC8
:10562800008000403952000838B5044603682169F3
:10563800A2681D68C0690A4361690A437D4902433B
:1056480029400A431A605A68E16822F440520A4322
:105658005A60794AA16993421CBF226A11439A6829
:1056680022F06E4222F430620A439A60DA6A616A72
:1056780022F00F020A43DA62704A93421CD14FF0BB
:10568800B043D3F8883003F0030343F44033A3F561
:105698004033013B022B00F2C780694A9B5CB0F59E
:1056A800004F40F08980082B24D8DFE803F061C060
:1056B8008323802323236500624A934209D14FF054
:1056C800B043614AD3F8883003F00C0343F4402315
:1056D800E4E7594A93420DD14FF0B043D3F88830EC
:1056E80003F44063B3F5006F1AD005D853B1B3F58E
:1056F800806F12D0012009E0B3F5406FFAD14FF462
:1057080000400EE0FEF7B2FC58B900204FF001133C
:10571800A3660023C4E91D3338BDFEF7AFF8F3E7ED
:105728004A4865684A4B626A05EB450133F812201E
:10573800B0FBF2F39942DDD8B3EB053FDAD800238A
:105748001946FBF72DFA090241EA10616B080002BD
:10575800C0182A464FF0000341F10001FBF720FA78
:105768003C4BA0F540729A42C4D82368D860CCE775
:10577800FEF77CFC0028C8D06168354B626A33F8B4
:105788001220B0FBF2F24B0803EB42034FF6EF7224
:10579800B3FBF1F3A3F110019142ABD823F00F0250
:1057A800216892B2C3F342031343CB60ADE7FEF71F
:1057B80065F8DFE72548DFE7082B9BD801A252F8F8
:1057C80023F000BF15580008215800082D5800087C
:1057D800FD56000827580008FD560008FD56000829
:1057E800FD560008F15700084FF400406368616AED
:1057F800174A32F81120B0FBF2F000EB5300B0FB6F
:10580800F3F04FF6EF73A0F11002ACE7FEF72EFCB1
:1058180000283FF47AAFE9E7FEF738FCF8E7FEF72F
:105828002DF8F5E70948E1E7B0F5004FF4D1FEF7A8
:105838002DFC9FE7F369FFCF00800040003801404E
:1058480070F200080044004073F2F4070024F400EA
:1058580080F20008FFFC0F00836ADA0710B506D54E
:105868000168C46A4A6822F4003222434A609C07ED
:1058780006D50168046B4A6822F4803222434A60E4
:10588800590706D50168446B4A6822F480222243EE
:105898004A601A0706D50168846B4A6822F40042F8
:1058A80022434A60DC0606D50168C46B8A6822F484
:1058B800805222438A60990606D50168046C8A687A
:1058C80022F4005222438A605A060FD50168446CBC
:1058D8004A6822F480122243B4F5801F4A6005D139
:1058E8004A68846C22F4C00222434A601B0606D52B
:1058F8000268C16C536823F400230B43536010BD46
:105908002DE9F041DDF8188004460E4615461F467D
:105918002268D36936EA03030CBF01230023AB4294
:1059280001D0002027E0B8F1FF3FF2D0FBF7E4FFF9
:10593800C01B4045206802D8B8F1000F1DD150E8BF
:10594800003F23F4D07340E80032002AF7D100F179
:10595800080353E8003F23F0010300F1080141E880
:105968000032002AF3D12023C4F88830C4F88C30E0
:1059780084F884200320BDE8F08103685A07C7D55E
:10598800C3691B05C4D54FF40063036250E8003FA8
:1059980023F4D07340E80032002AF7D100F108035D
:1059A80053E8003F23F0010300F1080141E8003209
:1059B800002AF3D12023C4F88830C4F88C30C4F806
:1059C8009030D5E773B504460026C0F89060FBF721
:1059D80093FF23681B681A07054619D423681B68B8
:1059E8005B070AD56FF07E43009300222B464FF4E5
:1059F80080012046FFF784FFB0B900202023C4F8B7
:105A0800883084F88400C4F88C30E06620670CE0A5
:105A18006FF07E430093324603464FF40011204650
:105A2800FFF76EFF0028D9D0032002B070BD10B573
:105A3800044650B3D0F888301BB980F88430FCF79E
:105A4800ADF822682423C4F88830136823F00103D2
:105A580013602046FFF7E8FD012816D0A36A13B1AA
:105A68002046FFF7F9FE23685A6822F490425A60EC
:105A78009A6822F02A029A601A6842F001022046C7
:105A88001A60BDE81040FFF79DBF012010BD00005F
:105A980030B581658168A0F85C200023B1F5805F8E
:105AA800A0F85E20436735D10369002B40F2FF134D
:105AB80018BFFF23A0F860300023C0F890302223DD
:105AC800C0F88C30016801F1080353E8003F43F047
:105AD8000103083141E800340368002CF2D1456E17
:105AE80084680169B5F1005F34D1B0F86850954217
:105AF80030D8B4F5805F1DD1254A264C002918BF3F
:105B080022464267C1B153E8002F42F4807243E84D
:105B18000021F7E729B90369002B14BF7F23FF236E
:105B2800C8E7B1F1805FC5D10369002B0CBF7F23A3
:105B38003F23BFE7174AE4E703F1080252E8002FC2
:105B480042F0805203F1080040E800210029F3D117
:105B5800002030BDB4F5805F0FD10F4A0F4C0029EB
:105B680018BF2246426751B153E8002F42F49072A1
:105B780043E800210029F7D1EAE7084AF2E753E8A9
:105B8800002F42F0200243E800210029F7D1DFE787
:105B980099540008FD520008395200086D51000858
:105BA800D0F88C30202B30B415D1B9B1B2B1002364
:105BB8000468C3660A4B9C420AD063681B0207D577
:105BC80054E8003F43F0806344E80035002DF7D1E6
:105BD80030BCFFF75DBF022030BC70470120FBE7F7
:105BE80000800040436E30B52BB90123A0F86A301D
:105BF800A0F8683030BD0368094D9A689968094C67
:105C0800490FC2F342626B5C615CDB00B3FBF1F3EA
:105C1800A0F86A30AB5CA25CDB00B3FBF2F3E7E709
:105C2800A0F2000898F200087047704770471FB547
:105C380004AB03E9060090F88430012B04463AD0FF
:105C4800012380F884302423C0F8883003681A6858
:105C580022F001021A609A6822F440120A439A60FC
:105C680071B95A68BDF80C009DF80E1022F01002A8
:105C780002435A605A6822F07F4242EA01625A603F
:105C88001A6842F001021A60FBF736FE6FF07E4296
:105C9800034600924FF4800100222046FFF730FEB1
:105CA80038B92023C4F88830002384F8843004B03D
:105CB80010BD0320F8E70220F9E790F88430012BA3
:105CC8000FD0012380F88430016851E8002F42F09A
:105CD800020241E80023002BF6D180F884301846F0
:105CE80070470220704710B590F88430012B0446A5
:105CF80017D02423C0F8883003681A68196821F07F
:105D08000101196042F000524FF0005141661A60DB
:105D1800FFF768FF2023C0F88830002084F884004B
:105D280010BD0220FCE770B590F88430012B0446C2
:105D380017D005682423C0F888302E682B6823F014
:105D480001032B60AB6823F060431943A960FFF798
:105D580049FF20232E60C0F88830002084F8840092
:105D680070BD0220FCE7000038B5084D052455F841
:105D7800043B2BB9013C14F0FF04F8D1204638BD90
:105D8800DB6898470028F5D0F9E700BF84050020B4
:105D9800034BD870034B1B681B6C03B11847704743
:105DA8009805002080050020034B1874034B1B68DE
:105DB8005B6C03B1184770479805002080050020E8
:105DC800F0B5314D314B95F90420314E91B00C4668
:105DD800012795F905108DF8047002288DF809201F
:105DE8008DF80A1010D18DF80800D8711C7202F0D5
:105DF8009FFD337803B114B101A803F003FA254BD2
:105E0800059A1A6011B0F0BD59714FF480711A717A
:105E1800D9801C7233788DF8087053BB1F2306A8ED
:105E28008DF81C208DF8183002F064FF20238DF8BF
:105E3800183006A82B798DF81C3002F05BFF22235E
:105E48008DF8183006A86B798DF81C3002F052FFD7
:105E580021238DF8183006A86B798DF81C3002F0D4
:105E680049FF29238DF8183006A80B4B079302F039
:105E780041FF02F05DFD012306A88DF818308DF86A
:105E88001C3002F037FFB4E7980500207C000020A2
:105E98007405002078050020000400017FB509235F
:105EA80001A88DF8043003F0ADF90038044B059AC9
:105EB8001A6018BF0120404207B05DF804FB00BF1C
:105EC8007805002070B504460B46134962784A707D
:105ED8000020A2780A7208701A884A729A788A7220
:105EE800DB780B746368CB600C4B1B68DA6A2AB1E9
:105EF800237803F0FB030A2B00D09047084E0525B2
:105F080056F8043B1BB15B6A0BB120469847013D2C
:105F180015F0FF05F4D170BD880000208005002031
:105F28008405002070B50446104801230370637887
:105F38004370A3788372E368C360E37803762369C8
:105F48004376237943720A4B1B689B6A03B19847CF
:105F5800084E052556F8043B1BB19B690BB120463A
:105F68009847013D15F0FF05F4D170BD9C00002055
:105F78008005002084050020014B1868704700BF89
:105F88007805002000B58BB0012368468DF80030F5
:105F980002F088FD38B99DF80400003818BF0120C8
:105FA8000BB05DF804FB0020FAE7000008B501F02B
:105FB80073FE48B9FFF7E6FF012806D0054BD879EC
:105FC800197AFFF7FDFE012008BDBDE80840FFF77C
:105FD800CBBE00BF7C0000202DE9F04186B005460D
:105FE8000E46174601F058FE00287FD101F06CFEDE
:105FF800044640B9FFF7C6FF012807D03D4B197A80
:10600800D879FFF7DDFE6FF0020462E0DFF8E88080
:1060180088F80860003E18BF01268DF80460374EE6
:10602800687833798DF81230694602F0D9FC002877
:106038003ED08DF804400394ADF810406FF006048C
:1060480095E803002E4B83E80300337988F80A307B
:10605800394601A803F0DAF92A4B059A1A60112883
:1060680041D801A353F820F0CF600008F56000087C
:10607800EF600008EF600008EF600008EF600008BC
:10608800EF6000080F600008EF600008EF6000088C
:10609800EF600008E9600008EF600008EF600008A2
:1060A800F5600008F5600008F5600008E360000886
:1060B8002B788DF808306B78ADF810306B68039347
:1060C8004FF0FF34BCE7104B00221A70E31D18BFD5
:1060D8001446204606B0BDE8F0816FF00404F8E7E6
:1060E8006FF00504F5E74FF0FF34F2E76FF00104B5
:1060F800EFE700BF7C0000209C00002098050020EE
:10610800AC000020780500207C05002037B501F0A0
:10611800E5FD144D052455F8043B5BB11B694BB1F3
:1061280055F8043C9B682BB1984718B155F8043CC6
:106138001B699847013C14F0FF04ECD1FFF714FEEB
:1061480068B9094D2B7853B1084BADF80040D978A0
:10615800019422466846FFF73FFF00B92C7003B050
:1061680030BD00BF840500207C0500209805002074
:1061780030B58BB0054601F08FFD0446002839D1B3
:10618800FFF700FF012838D168468DF8004002F07B
:1061980089FC10B14FF0FF3004E09DF80430AB42A9
:1061A80002D100200BB030BD012DF3D0022D11D04B
:1061B800002DF7D1002BF4D068468DF8045002F07A
:1061C80099FD0028E6D10E4B1B681B6B002BE8D00D
:1061D8009847E6E7002BDDD168468DF8045002F0B9
:1061E80089FD0028D6D1064B1B681B6B002BD8D025
:1061F8002846EDE76FF00100D4E76FF00200D1E721
:106208008005002010B504468AB018B94FF0FF3059
:106218000AB010BD002368468DF8003002F042FC39
:106228000028F3D19DF804302370F1E77FB50022F0
:106238000B4620498DF8072001220A7042784A70DF
:106248000446002A33D102790A721A884A729A7867
:106258008A72DB780B740369CB60C378164D8DF8AE
:106268000830037B8DF80930836803932B68DB6A59
:106278000BB102A898472B689B6B13B1227E02B121
:1062880098470E4E052556F8043B1BB1DB690BB148
:1062980020469847013D15F0FF05F4D10DF10700A0
:1062A800FFF7B0FF637913B1054B01221A7004B0F0
:1062B80070BD00BF880000208005002084050020F4
:1062C8007C05002010B504468AB018B94FF0FF309D
:1062D8000AB010BD202368468DF8003002F0E2FBBA
:1062E8000028F3D1024A9DF9043023701371EFE7B7
:1062F8009805002000B58BB02323019068468DF8DF
:10630800003002F0F7FC003818BF012040420BB003
:106318005DF804FB70B5654C01468EB01822204626
:1063280006F0FEF8624B00221A70FBF7FBFF237899
:106338004068012202FA03F1014004D15D4B08468E
:1063480008F0E4F8FEE75C495C481A4602F032F9C6
:1063580018B14FF0FF300EB070BD272304A88DF898
:10636800103002F0C7FC564E564D002870D101235C
:1063780033702B68DB690BB100209847272304A8EA
:106388008DF8103002F08EFB059B93F848202270A0
:1063980093F8182193F81A316270A370464BD3E929
:1063A800020105F0AFFF05460028D2D1464E06236C
:1063B80004A88DF8103002F075FB059B736104A8E2
:1063C80002F098FC022304A88DF81030059602F01C
:1063D80069FB0836032304A88DF81030059602F0EF
:1063E80061FB0F2606F052F8012304A88DF814303B
:1063F8008DF8106002F07EFC10230DEB03008DF881
:1064080010308DF8145002F075FC04238DF810300C
:1064180004A8A3788DF8143002F06CFC3A238DF8A8
:10642800103004A86369059302F064FC02A920787F
:106438008DF8086004F0E8F8003818BF0120E07112
:106448001420FFF757FFE07903F0A4F9284682E704
:1064580028238DF810302B681B6943B104A802F07B
:1064680021FB2B6805981B6940F2C45198472723E4
:1064780004A88DF8103002F03DFC50B9012304A89F
:106488008DF8103002F00EFB9DF81430002B7FF4CD
:106498006EAF3378002B7FF46CAF052204A88DF81B
:1064A8001020059302F026FC78E700BF980500202D
:1064B8007C050020A8F20008C0050020D8050020AF
:1064C80074050020800500205C05002037B50023F6
:1064D8000D4601930446D0B900F0A8FB0190019B3A
:1064E800D3B10F4A42F824300E4A9A620E4A126813
:1064F800916B1963916C596392690C49D9625A611D
:1065080028465B680A49F2229847002006E001A95C
:1065180000F092FB0028E2D04FF0FF3003B030BD0E
:1065280084050020C95D000880050020A55E0008DC
:1065380068040020194B07B51860194B194A1A60EE
:10654800194A5A60194A9A60194ADA60194B02685E
:106558001A6042685A6082689A60C268DA60164AAD
:106568001A6182695A61154BC26B5A60144A0191CB
:1065780019609A601946134ADA600020FFF7A6FFEF
:1065880048B901A800F056FB003818BF0120404266
:1065980003B05DF804FB4FF0FF30F9E780050020F9
:1065A800D80500202D5F0008356200084D660008F8
:1065B800CD5E0008C0050020C1A50008B005002078
:1065C800995D0008B15D000851B118B1012804D0E7
:1065D80000207047044B0B607047044B0B60F7E7D3
:1065E8004FF0FF30704700BF0004000101000102B6
:1065F80008B503F0EBF8002814BF6FF00100002085
:1066080008BD08B502F0BCF9002814BF6FF00100FE
:10661800002008BD10B504468AB018B94FF0FF3005
:106628000AB010BD212368468DF8003002F03AFA0E
:106638000028F3D1024A9DF9043023705371EFE723
:10664800980500202DE9F0412E4D2F4F00232B7087
:1066580043786B703B689B6A8AB004460BB1284646
:106668009847DFF8A880052658F8043B1BB11B6A39
:106678000BB120469847013E16F0FF06F4D1237867
:10668800052B2FD00B2B35D0012B25D1204C0623E1
:1066980068468DF8003002F005FA0199E07905F0B6
:1066A80077FE10B91B4B019A5A611B48FFF70AFE87
:1066B8001A48FFF7AFFF6B788BB9A371184B58785E
:1066C800FFF756FD3B685B6A0BB1114898476B783A
:1066D80013B9E07905F0ECFE0AB0BDE8F081FF23BC
:1066E800A371EFE70F4B01225A74227A9A74627AE7
:1066F800DA74F1E76378002BEED00AB0BDE8F04118
:10670800FFF7CCBB9C0000208005002084050020FA
:106718007C0000205C050020800000208100002013
:10672800980500208800002030B58BB0FFF769FF7E
:106738000446F0B903F048FF831C1DD0F8B9134D87
:106748002B685B69DBB1272368468DF8003002F0BF
:10675800A9F92B6801985B694FF4B961984703F070
:1067680045FF78B92CB9094B1B68DB690BB10120CF
:10677800984720460BB030BD6FF00704EFE74FF0A5
:10678800FF34ECE74FF0FF34F3E700BF800500204B
:10679800014B1878704700BFEC050020014B587872
:1067A800704700BFEC05002070470000044B9A7A40
:1067B8000AB101225A70034B5B6903B1184770474D
:1067C800EC050020B800002073B5224C6378002B3C
:1067D80033D008F085F966680546FFF7CDFB064417
:1067E800AE4214D2A37A93B1E0228DF800208DF83E
:1067F8000130217AE368019301226846FFF7ECFB38
:1068080008B1073010D100236370A372656094F853
:106818003430EBB1002384F834300F4B5B6BBBB1E1
:1068280002B0BDE87040184740F2DC510B4808F050
:1068380023FA0A4808F0E6F9E8E794F83520002A30
:10684800E5D094F8360084F83530FFF791FCDEE7A0
:1068580002B070BDEC050020B8000020240600201E
:1068680037B5104D104CC8B1C1B101236272002276
:106878002860E16023700D480D4B00924FF0FF3106
:1068880008F014F900250B4825822022294605F036
:106898005BFE6570A574A58603B030BD00232B6030
:1068A8002370EFE7E8050020EC050020240600200F
:1068B800B5670008000600202DE9F0478E4C2378C4
:1068C8008CB0002B56D0C2780AB9837B13B1238AC7
:1068D80001332382437B002B4CD0E02A4AD100238A
:1068E800A372876897F80080B8F1220F27D8B8F10B
:1068F800220F30D8DFE818F04100FB0052005A00A0
:1069080061006E0075008E009D00B400C7002F0066
:106918002F002F002F002F002F002F002F002F00F7
:106928002F002F002F002F002F002F002F002F00E7
:106938002F002F002F002F00C900D000D400B8F17D
:106948007E0F00F0CC80B8F17F0F00F0DF80B8F147
:106958007D0F00F0AB80A57A002D00F05B81674CBD
:10696800637A3BB94FF47A71204608F085F92046DE
:1069780008F048F90CB0BDE8F087E368012200216F
:10698800A2721970A37AE1689818A0720620C854F8
:10699800A37AE1689818A072CA54DCE7584B9B6A3E
:1069A800002BD8D0012102209847D4E77B7884F8BF
:1069B8003630012384F83530CDE704238DF80430D0
:1069C8007B78003B18BF012301A88DF8083002F03E
:1069D80091F9C0E77878003818BF012002F0DAFE94
:1069E800B9E7484E0FCE01AD0FC50FCE0FC596E8DB
:1069F800070085E807007B780A2BACD8424A126862
:106A08005268002AA7D00CA901EB830353F82C0C79
:106A18009047A0E77878431E012B9CD83A4B013861
:106A28001B6818BF012020729B68002B93D09847E1
:106A380091E7E26801230821A3721170627A057B4D
:106A4800A17AAA4228BF2A46934284D285685A1C52
:106A5800EB5CE56801334E1CA6726B54D3B2EDE7CC
:106A6800E3680122A27209221A70A37AE268218AD5
:106A7800581CA072D154A27A238AE1681B0A501CC0
:106A8800A0728B5467E7238265E705238DF80430ED
:106A980001A802F0B7FB5EE7194BDB6A98475AE793
:106AA800194B78781B686075DB68BEE7037B072B9A
:106AB8007FF451AF06238DF80430B7F80130ADF8F4
:106AC80008307B793A791B0443EA0223FA781343A6
:106AD800642253430393BB798DF81030D8E73B22E7
:106AE80001A88DF804208DF8083002F003F901237D
:106AF80084F834302FE700BFEC050020240600207E
:106B0800B8000020F4F00008E80500202A2301A8B6
:106B18008DF8043001F0C6FF94F80A90E6689DF8F5
:106B280008009DF809509DF80A709DF80BC09DF863
:106B38000D309DF80E209DF80F109DF80CE009F11E
:106B4800010A84F80AA006F80980354E94F80A90DC
:106B58003668D4F80C8009F1010A84F80AA096F87E
:106B680003A008F809A094F80A90D4F80C8009F159
:106B7800010A84F80AA096F802A008F809A094F877
:106B88000A90D4F80C8009F1010A84F80AA096F852
:106B980001A008F809A094F80A9009F1010A84F8FC
:106BA8000AA096F80080E66806F8098094F80A803A
:106BB800E66808F1010984F80A9006F808C094F814
:106BC8000AC0E6680CF1010884F80A8006F80C701F
:106BD800A77AE66807F1010C84F80AC0F555A57A8A
:106BE800E6686F1CA7727055A07AE568461CA67205
:106BF8002954A17AE0684D1CA5724254A27AE16832
:106C0800501CA0728B54A37AE268591CA17202F836
:106C180003E0A0E6034807F0A7FF6570AAE600BFF7
:106C2800E80500202406002070470000004870474F
:106C3800B8000020002070474FF0FF307047000078
:106C4800044B054A93F81831022B18BF062382F823
:106C580090347047000C0020C8110020034BD3F873
:106C6800483313B15B6903B118477047C811002056
:106C7800034A137843F004031370FFF7EFBF00BF14
:106C8800C41100201FB50A4B8DF8090093F87C2029
:106C98008DF80A2093F88C2093F848000D3202A949
:106CA8008DF8082003F0B0FCC0B205B05DF804FB15
:106CB800000C002010B5074C04F5806007F054FF65
:106CC80094F81A3413B1012384F81934BDE810403C
:106CD800FFF7C4BFC811002010B50C4CD4F84033DE
:106CE80043F08003C4F8403394F81A3413B10020F9
:106CF800FFF7E0FF94F8913423F0120343F01203F6
:106D080084F89134BDE81040FFF79ABFC8110020FD
:106D18002DE9F041DFF8AC8098F81831022B0646CF
:106D28000D4602D0284BDB6A984702F0E9FD04467D
:106D380028B1022002F0DAFD002002F0DCFD98F80C
:106D48001831012B17D102F0DDFD074630B10020C4
:106D580002F0CDFD002002F0CFFD3C4602F0D4FD4C
:106D680048B1002002F0C4FD002002F0C6FDBDE8D5
:106D7800F041FFF765BF002CF9D1144C94F890242A
:106D880094F81A34BAB90BB184F84164304602F069
:106D980065FFD8F82C0007F0ADFED4F8B43398425C
:106DA800E5D30B4807F0E0FE94F8913443F0100364
:106DB80084F89134DBE70BB184F84154284602F09B
:106DC8004DFFF1E7000C00202CFA0008C811002044
:106DD8006015002073B5164C164D04F57A76EB6CE9
:106DE80095F8502095F9781095F84800009603F02A
:106DF80031FC95F8303184F8FC3395F8480040F2BE
:106E0800012304F224423146A4F8FA3303F02EFC9D
:106E180058B194F8243484F86A34074B00205B6B2B
:106E2800984794F8FB3384F8903402B070BD00BFE3
:106E3800C8110020000C00202CFA0008074A10B5E1
:106E4800137843F002031370FFF708FFBDE8104002
:106E5800034B01220021022007F058BBC411002077
:106E6800F1F20008074A10B5137843F008031370CD
:106E7800FFF7F4FEBDE81040034B01220021022079
:106E880007F044BBC411002001F300082DE9F041CC
:106E98000F4616461D46804607F022FE0B4A0C4C4C
:106EA8001378278123F0110343F011031370C4E909
:106EB800000866812573FFF7D1FEBDE8F041054B58
:106EC80001220021022007F021BB00BFC4110020CD
:106ED8007417002011F3000813B507F001FE0D4BDD
:106EE8006C461860204607F04FFD94E803000A4AF4
:106EF8000A4B83E80300137843F020031370FFF76D
:106F0800ADFE074B01220021022002B0BDE810406F
:106F180007F0FCBA84170020C411002000150020D7
:106F28001EF30008F8B5334D95F81841012C0646B4
:106F38004BD0022C51D064B938B9D5E91B0105F101
:106F4800740383E803002046F8BD01283DD00228D9
:106F580001D00324F7E7284F85F8180107F5747E58
:106F6800BEE80F0007F57A7CACE80F009EE8030046
:106F780095F8E9308CE8030087F8FB63E3B195F8EE
:106F88000031022B18D1D5F804316B67C7F8EC3300
:106F980095F87D3095F8082187F8F83395F88C3006
:106FA80085F8782087F8F93397F81B2487F8E823C1
:106FB80040F20133A7F8FA33002387F81A340F4B4D
:106FC800DB6A9847FFF706FFBDE702F0A4FC04461A
:106FD8000028B8D185F81861B5E70028B9D1064B63
:106FE80085F81801062283F89024044BDB6A984739
:106FF8003446A8E7000C0020C81100202CFA00082D
:107008002DE9F04192B0064602F07AFC002840F0E3
:107018005981AD4D95F81831012B09D02B6BAB4C2C
:1070280093B194F80431BBB1042B6FD0032003E073
:1070380002F068FC18B10F2012B0BDE8F08102F030
:1070480063FC0028EAD0F6E7B5F82031D4F81C2410
:10705800013B53432B63E4E79D4803F00CFA0028F7
:1070680040F02C8194F80C3123802B6B0C930DF19C
:10707800180895F839308DF83830404695F81C31A5
:107088008DF83A3007F0A6FCD5F82831009302AF06
:1070980098E80600D5F82431384607F032FC97E81E
:1070A80003000FAB83E80300EB6A0D9300238DF810
:1070B80044302388ADF8463095F8303101228DF8F8
:1070C80039201BB98DF844208DF83930814B009355
:1070D800814B95F84800A3F179020CA903F009FB4C
:1070E800C0B10B28A8D1D4F8941499B1002EA3D01C
:1070F800D4F84033794843F02003C4F8403307F00C
:10710800BBFD764807F07EFD002095E7704803F048
:10711800E6F9A4E795F8487095F9693095F93920AA
:1071280095F87D106E4E384603F0F0FA009641B29D
:10713800EB6C95F850203846183603F08BFA009619
:10714800EB6C95F8502095F9701095F8480003F00D
:1071580081FAD4F8C413AB6DD4F8DC230B44C4F81B
:10716800B033EB6D1344C4F8B43394F80431042BF2
:1071780007D02B6E0B44C4F8B0336B6E1344C4F8BD
:10718800B4330023089395F8303183B108A802F08E
:1071980095FC00284ED195F9390094F837629DF88E
:1071A8002070FFF76FFD3E4480B2B04240D3002309
:1071B8008DF8133095F839308DF8213095F838303E
:1071C8008DF82230D5F880300993D5F884300A93A9
:1071D8002388ADF82C3095F8303194F81B648DF87D
:1071E8002E3095F848003F4B8DF820600DF11302C2
:1071F80008A903F043FA012384F8413495F839309B
:1072080084F842349DF8133084F84334D4F81C349D
:10721800C4F85064C4F84834C4F8583402F076FB13
:1072280050B1D4F81C0402F083FB28B1102003E706
:10723800082001E71320FFE695F81831012B01D14A
:1072480002F078FB02F065FB0023059394F8043103
:1072580095F9395094F81B649BB1042B7FF4E6AE82
:1072680005A802F067FE58BB94F8183413B1059BC3
:10727800013B0593164B05983246E9B202F0C0FE71
:1072880002E0134802F090FEC0B9D4F8403394F8F5
:107298000C11218043F00203C4F8403394F81834E9
:1072A80011480133DBB284F8183484F845340F4BA5
:1072B80000259B6AC4F89854984725E71120BBE637
:1072C8001220B9E60E20B7E6000C0020C8110020F5
:1072D800D0120020300C00205C1600203015002051
:1072E80080150020E4150020CA1100202CFA00089F
:1072F800F0B5504C504EB4F8DC202287D4E92D016B
:1073080094F8B12084F8692004F16C0282E8030043
:10731800D4E92F0104F1740282E80300B4F8C42010
:10732800A4F87C2091B0D4F8CC20D4F8C810C4F8C4
:1073380084200025D4F8D020C4F888200123A4F89C
:107348002031C4F8801084F83051A56284F81B51AC
:1073580084F83A5084F81D5184F81E51C4F8345109
:10736800C6F89854A6F8185486F81A54A4F8385150
:107378008DF8183004F50973039304F50A7394F82B
:107388004800A4F84651049303A92C4B84F84551AE
:10739800C4E94F55059303F045F9E36EC6F8D433B5
:1073A80094F87D3086F8E03394F88C3086F8E13331
:1073B8004FF48073A6F8E23386F8D05394F830314E
:1073C80086F8E43306F574770FCF06F57A740FC4A0
:1073D80097E8030040F2012384E80300A6F8FA3393
:1073E800D6F8483386F81B54CDE901551BB15A68C5
:1073F8005B6901920293124B0793A3F1480208922A
:10740800A3F1140209920F4A0B9229330A93A2F1AD
:107418009C030C93A2F198030D93131D0E9301A9DD
:1074280002F14C0307A802F599620F9302F05DFA86
:1074380011B0F0BD000C0020C8110020E416002097
:1074480030160020E40C0020F8B50D4F0D4C0E4E00
:107458000D4607F089FB3B6B984796F8480004F205
:107468002442294603F002F948B194F8243484F8F8
:107478006A34706D7B6B9847EB7C84F89034F8BD68
:107488002CFA0008C8110020000C00200F4890F8C2
:107498001B3480F8B8330E4B93F8692080F8BB236F
:1074A80093F87D2080F8C82393F88C2080F8C923AE
:1074B80093F8303180F8CC330022A0F8CA2300F5C5
:1074C8006E7100F56070FFF7BFBF00BFC8110020E4
:1074D800000C0020114890F89034EBB190F81B3460
:1074E80080F8D0330E4BDA6EC0F8D42393F87D20A1
:1074F80080F8E02393F88C2080F8E12393F830316A
:1075080080F8E4334FF48072A0F8E22300F5747138
:1075180000F56670FFF798BF704700BFC8110020DC
:10752800000C002070B5344C2421204605F00EF8DC
:10753800636A984218BF60624FF01C012F4814BF5D
:107548000125002505F002F8636C984218BF6064B5
:107558004FF480712A4818BF45F0020504F0F6FF81
:10756800D4F84831984218BFC4F848014FF0D40104
:10757800244818BF45F0040504F0E8FFD4F8203289
:10758800984218BFC4F820024FF000011E4818BFE7
:1075980045F0080504F0DAFFD4F82432984218BF01
:1075A800C4F824024FF46071184818BF45F010055C
:1075B80004F0CCFFD4F8A835984218BFC4F8A80541
:1075C8004FF01401124818BF45F0200504F0BEFF23
:1075D800D4F8C03598420F4B18BFC4F8C005D3F88B
:1075E800483318BF45F040052BB11B691BB128462D
:1075F800BDE87040184770BD000C0020280C002022
:10760800480C00204C0D0020240E0020280E0020DD
:10761800AC110020C81100202DE9F04F91B04FF0B7
:107628000008012B05460F4602928DF81580ADF82B
:10763800188003D8C84EC146B94502D311B0BDE879
:10764800F08F15F8090002F077FA4844B842F5DCE3
:1076580015F8093009F10104023BE4B2112BEDD809
:1076680001A252F823F000BFB9760008EB760008B3
:10767800EB770008157800089D780008C5780008A1
:107688003779000869790008E57900084576000827
:1076980045760008437A00084576000845760008D4
:1076A800017B0008297B00086D7B0008AB7B000884
:1076B800052002F0EDFA90B10521002002F0ACFAA5
:1076C8002A5DA64B09F1030409F102095FFA89F959
:1076D80083F85C2415F8092083F85D24E4B2A146F8
:1076E800AAE700238DF816308DF817308DF81C3076
:1076F8008DF82030B8F1000F6CD14FF0050896F8DE
:107708007C208DF83920631E96F839208DF83B20AF
:107718002B4496F838200D938DF83C2096F81A31B2
:1077280096F868208DF83D20D6F82C218DF83A304F
:107738000C9273B37B1C1B1BDBB28DF8383008AB83
:10774800019307AB009396F848000DF117030DF16C
:1077580016020CA902F09EFF8DF8150000F0070034
:10776800072813D196F939209DF9163086F8393053
:107778009A429DF8173086F83830B8BF01229DF834
:107788001C30B8BF86F81D2186F868304FF0000914
:1077980009E00523D1E701220DF11501032002F0CC
:1077A800DBF809F101095FFA89F29DF82030B3FB93
:1077B800F8F19142EFD82344DCB2631EDBB29F425A
:1077C8000DD9EA5C032A9AD0A74288BF1C464FF01D
:1077D800010884E709F105095FFA89F4F7E71C460F
:1077E800F5E72B5D012203F00F0309F1020986F882
:1077F8001B3102FA03F35FFA89F9A6F82031002257
:1078080006A9042002F0A8F84C4668E707238DF87B
:1078180015302B5D96F84800C3F3021203F00F03EE
:107828008DF8303009F10303DBB28DF83120EA5CC2
:1078380009F10403DBB209F10504EB5C09F1020963
:107848005FFA89F91B0443EA022315F80920134358
:10785800642253430CA90D9302F02BFF00F0070399
:10786800072BE4B28DF815000CD19DF8303086F85E
:10787800703086F878300D9BF36673679DF8313069
:1078880086F869308DF81800012206A9052002F053
:1078980063F824E7314BD3F848336BB11B685BB10D
:1078A8009847029B8DF8180003F03F038DF81930B4
:1078B800022206A90620EAE7FF20F2E703238DF853
:1078C80015302B5D8DF824300CAB089309F10303B8
:1078D800DBB209F10604EA5C96F8480009F10403F2
:1078E800DBB208A9EB5C1B0443EA022309F102029C
:1078F800D2B209F10509AA5C1343642253435FFA23
:1079080089F90C9300230D9315F809308DF8383058
:1079180002F0D5FEC3B20028E4B28DF81530FFF6A8
:10792800DEAE8DF81830012206A90720AFE72B5DDF
:1079380003F00F03012B4FF47A7238BF012353432E
:1079480009F10209B36513445FFA89F9F365002266
:1079580006A9082056E700BF000C0020C811002027
:107968002B5D96F84800C3F340128DF81D2007A937
:10797800C3F3001203F00F038DF81C208DF81E309E
:1079880002F0A3FE09F1020901305FFA89F93FF418
:107998003BAFBDF81C30914AA6F87C309DF81E30EC
:1079A8009DF81C40D05CF8F70DFF0223C6F8800054
:1079B8000CA996F848008DF830308DF8324002F066
:1079C80023FE96F93930089040B29842B8BF18465D
:1079D80086F83900002206A9092013E703238DF849
:1079E80015302B5D8DF8303009F10303DBB209F156
:1079F8000504EA5C96F8480009F10403DBB209F1D2
:107A08000209EB5C5FFA89F91B0443EA022315F8C3
:107A180009201343642253430CA90D9302F05BFE23
:107A2800C3B20028E4B28DF81530FFF658AE8DF8D1
:107A38001830012206A90A2029E7092002F028F9AE
:107A4800DFF89CA1002854D00921002002F0E4F8B6
:107A58000023ADF8263009F10203DBB24FF47A7146
:107A6800EA5C09F10303DBB20DF1300BEB5C1B049C
:107A780043EA02232A5D134309F10402D2B209F151
:107A8800060409F10509AA5C5FFA89F943EA026369
:107A980015F8092003934A4312125846ADF82420DA
:107AA80006F072FF039B03F1965303F5A91303F540
:107AB800EC530893DAF83C3300930DF1200999E868
:107AC8000600DAF838330AA806F01BFF0B9B009370
:107AD8009BE806000A9B484606F0F8FE99E8030072
:107AE80006F02AFF01F021FF0123E4B28AF83834B6
:107AF800F5E58AF83804F2E50C2002F0C9F8002808
:107B08003FF4EDAD0C21002002F086F8344B93F8D9
:107B18009034043B012B7FF6E2AD01F002FFDEE575
:107B280009F10203DBB22A5DE95C09F10303DBB268
:107B380009F10504EB5C09F104095FFA89F91B04F2
:107B480015F8090043EA012313436421594300F05F
:107B58000F0001F0E7FEE4B28DF81800012206A933
:107B6800112094E60D2002F093F800283FF4B7ADF9
:107B78000D21002002F050F809F10203DBB2194A86
:107B8800E85C2B5D126809F1040409F103095FFA46
:107B980089F943EA002015F80910E4B201F0C4FE9F
:107BA8009DE52A5D09F1020309F1040409F10309BD
:107BB800DBB25FFA89F9E95C15F809301B0443EA7E
:107BC800012313436420584301F0B0FEE4B28DF85A
:107BD8001800012206A9132059E600BF2BF300085C
:107BE800C8110020741700200E4B93F891249207B7
:107BF80003D593F88F24012A08D90B4991F81A2143
:107C080022B18A6A501C18BF01328A620022A3F886
:107C1800182483F81A24D3F8402322F00202C3F868
:107C280040237047C8110020000C002070B5184C84
:107C3800184D04F55A7006F097FFD4F84033D4F87D
:107C48009804D5F8906023F02003C4F8403338B185
:107C580006F050FF864203D2002385F83A3070BD03
:107C68000120FFF7CDF90028F9D00B28F7D095F8B7
:107C7800393084F84234092094F8183484F84534AB
:107C880084F8410401F0EAFFBDE87040FFF7ACBF9B
:107C9800C8110020000C0020094BD3F84023012A0A
:107CA8000AD008490978C90708D43AB993F8920460
:107CB800013818BF01207047002070470120704725
:107CC800C8110020C4110020034BD3F84003431E01
:107CD80058425841704700BFC81100202DE9F04FA5
:107CE800A9B0EFF3108272B6DFF8F4820021D8F859
:107CF8000030C8F8001082F31088BA4C002B00F04E
:107D0800E480DAB29B06039264D5B74D95F8183132
:107D1800022B02D0B54BDB6A9847EFF3108972B695
:107D2800B34F06F0DDFE3E68D4F8B013361A31447E
:107D3800B04806F0A1FFAF4806F064FFD4F8B413CA
:107D4800AD48314406F098FFAB4806F05BFF89F375
:107D5800108894F81A34002B00F06D81152312A9AD
:107D680095F848008DF8483002F04EFCD4F8B4136A
:107D78000F900144A14806F07FFFA04806F042FF9B
:107D88003B6894F81B24EB620DAF38468DF87020E1
:107D98001D9306F01FFED5F82831009306AE97E82C
:107DA8000600D5F82431304606F0ABFD96E803000E
:107DB8001FAB83E80300D4F81C341E9395F83031C8
:107DC80095F84800003B18BF01231CA98DF87130B5
:107DD80002F023FC039BDF064BD5834DDFF820A27E
:107DE800D5F8E420BAF90A30059298F800200493EF
:107DF800002363F300020A9388F8002084F84434CF
:107E0800049AA4F8223484F82534C4F82834A4F851
:107E18002C3484F82E34C4F8303484F82034C4F870
:107E2800343484F83834C4F83C34704B9AF90C90E4
:107E3800A4F88C2494F89024DB6A84F88E9484F84F
:107E48008F24DAF80470BAF80860984794F88F34E9
:107E580013B9694806F088FE3146384601F04EFDF0
:107E68008346002800F0EA80049BA4F87E3484F856
:107E78008094039B19071AD55B4B93F81831022B92
:107E880002D05A4BDB6A98470220FEF7D9FE84F8E5
:107E9800410401F0E3FE94F81A3413B1012384F885
:107EA800193494F8913443F0100384F89134039B07
:107EB8005A0703D506210520FEF72AFF039B9B07D7
:107EC80003D504210320FEF723FF01F035FD94F8C4
:107ED8009124D7065FD5002384F89234D4F8403330
:107EE8001E0644BF23F08203C4F8403312F0050F86
:107EF80000F0FC820B2001F0CBFE002800F0F68297
:107F080094F89134DD0700F1F182580740F10883B5
:107F1800D4F8403323F00203C4F84033D4F84023A4
:107F280082BB94F8915415F001011EBF2B4662F3F1
:107F3800000384F8913494F891345E0744BF6FF3DA
:107F4800820384F89134012384F8923421B1D4F85F
:107F580044332C481B6898476D070BD52A4801F015
:107F6800A3FE01F0D1FE28B194F8913443F0040344
:107F780084F8913401F0CEFC94F891346FF3041333
:107F880084F89134012384F8923494F8913443F0BE
:107F9800200384F8913494F8913418070AD56FF3C4
:107FA800C3031A4984F89134D4F84433A1F1240066
:107FB800DB68984794F8913499070AD56FF3410321
:107FC800124984F89134D4F84433A1F16C005B6809
:107FD800984794F89034022B1AD1FEF7FBFE17E06D
:107FE800C4110020C8110020000C00202CFA000841
:107FF800841700204815002060150020C8150020AF
:1080080074170020081600201C16002054160020A3
:1080180094F891349A0640F1C6826FF3451384F8B8
:108028009134D4F84033002B40F0BD8229B0BDE82C
:10803800F04FFFF777BA84F84134A1E695F8182194
:10804800012A0CD101F05EFC804668B1584601F067
:108058004EFC584601F050FC042384F88F347EB956
:10806800012384F8213450E101F04EFC0028F6D0B9
:10807800404601F03DFC404601F03FFC0523ECE79B
:108088003B7804935B09013B062B00F21882DFE87A
:1080980013F0070016029500160292001602070256
:1080A800102EDDD995F830311297F6B28DF84C6064
:1080B800002BD5D11CA804F05DF912AA1CA9FF2039
:1080C80002F0B2F89DF85830C3F3030307468DF861
:1080D8002C3095F8480095F87D308DF82D30072222
:1080E8000BA902F0A4FA002F5DD100285BD09DF8FF
:1080F80053309DF852201599C5F8E4101B0443EA43
:1081080002239DF8512002201343C5F8E03004F003
:108118003FF99DF8583095F8480085F82E71C3F35B
:108128000212C3F3030385F8703085F878309DF8A0
:10813800593085F86920012B38BF01234FF47A7232
:108148005343AB651344EB650DF15A034FF0010837
:108158001093113E94F81B348DF83C300FA985F824
:1081680068808DF8446002F06AFA0223404685F878
:10817800303101F08DFD18B14146384601F04CFD13
:1081880094F88F34012B00F2A88194F81A34002B4C
:1081980040F09B8194F8913443F0100384F89134B3
:1081A800FEF74EFD65E6012001F072FD0028E7D0DC
:1081B80001210720E2E7012384F8203495F87D3077
:1081C8008DF82E3094F824348DF82D3095F88C30B5
:1081D80095F848000D330BA98DF82C3002F014FAED
:1081E800A6F10D031BB2099023EAE37300B28342A0
:1081F8003FF736AF0B2E7FF633AFBB4B25931CA84A
:10820800FF231C978DF874608DF8983002F0D8F829
:10821800074600287FF424AF95F81831012B13D1B5
:1082280001F070FB002873D0384601F060FB384637
:1082380001F062FB04239DF87C101E9884F88F34AB
:10824800C1F3001101F077FB9DF87C301E99C4F84A
:10825800341413F00F0203D09DF89000002863D166
:108268009DF89800002862D0002A7FF4F9AE9DF8A6
:108278009020002A0CBF4FF002084FF0030800229C
:108288000A92D5F8EC20914254D195F8E9100029CA
:1082980050D0D5F80C1195F8EAB009680A9195F80C
:1082A8001811022902D1032184F88F14B8F1030FA1
:1082B8007FF4D6AE13F0600F7FF4D2AE059201279B
:1082C80095F82E31BBF1000F37D0BBF1010F38D133
:1082D800012B34D16FF0090646FA08F606F00106BC
:1082E800C6F10206F6B2BDF87E100AAA304601F0C1
:1082F8002DFE40B307280CBF0823012384F821343E
:108308000A9BC4F83034C4F86C34FEF7E5FCB0E5D9
:1083180001F0FAFA002897D0384601F0E9FA384611
:1083280001F0EBFA052386E74FF00008A7E74FF0C6
:108338000108A4E74FF0010BC2E70426D3E70326A0
:10834800D1E70123DAE71CAB009305990A9B324673
:10835800584601F0BBFE20B102280CBF0A230B23AC
:108368007FE60A9BC4F83034C4F86C349DF87C303E
:1083780084F82104C3F3401384F82E3484F8443479
:1083880094F88F3484F82274012B9EBF0122A862CE
:1083980085F81E21012FC4F8280484F82C0484F8D9
:1083A800410438D1022284F8202495F83A20002A82
:1083B8004AD19DF87C20D60646D4012B94F8401467
:1083C8009DF87C2005D8012901D1900601D501F03E
:1083D8005FFBB8F1020F94F88F3443D0B8F1030F64
:1083E8000AD09DF87C10B8F1010F4A4601F00F0140
:1083F80020A83BD0FFF710F99DF8903084F823347B
:10840800259BC4F828349DF8983084F82C3401232F
:1084180084F82D3430E0049A02F0E002A02A1BD13F
:1084280095F82E11012285F83A2009B92799696330
:10843800012B84F8202407D9D5F89020C4F83C24CF
:10844800DAF80020C4F8982495F81821002AB4D145
:10845800012284F82524B0E7002285F83A2084F820
:108468002024A6E79DF8981025984A46FFF7D4F8E7
:108478009DF8903084F823349DF89020E02A08D1A4
:1084880095F81F312BB984F82324C4F82834A4F8AC
:108498002C3494F8913443F0020384F891346FE655
:1084A800114D013EB2B2791C284604F039F8032375
:1084B800A4F82034C4F8285484F82C64E9E701238C
:1084C80084F82134FEF708FC5AE694F84434002B6B
:1084D8003FF460AE0020FEF7EDFB94F88F34022BDA
:1084E8003FF45EAE56E600BF0014002094F89134C5
:1084F800590715D5012001F0CBFB60B1012001F02F
:108508009DFB08B984F81804D4F8403323F002031B
:10851800C4F8403304E0062001F0BAFB0028F3D188
:1085280094F89134DA077FF5F9AC94F840240AB14D
:10853800032A18D11D4A94F8181492F86820914219
:1085480005D29B0723D594F88F34012B1FD81848E0
:1085580006F00AFBD4F8403323F02003C4F8403374
:10856800FFF742FBDAE4012A11D194F81924002A12
:108578003FF4D4AC0D4A94F8181492F8682091424C
:10858800E5D29F0703D594F84434002BDFD194F843
:10859800913400206FF3041384F8913484F819049B
:1085A800FFF744FBBAE429B0BDE8F08F000C0020C7
:1085B800301500202DE9F04F89468DB090460746CA
:1085C800002800F08F81002900F08C810368002BBF
:1085D80000F088814368002B00F084818368002BB9
:1085E80000F08081C368002B00F07C81104602F007
:1085F80007F8002800F07881BD4CBE4D384601F0E0
:10860800C1FA40F2C4520021204603F09DFF40F217
:108618001C520021284603F097FFB74BC4F82C31B1
:1086280004F50973089304F50A7300264046099374
:1086380008A9B24B84F848800A9384F8186184F832
:108648008C608DF82C6001F0EDFF0F2306A994F8DB
:1086580048008DF8183001F0D7FF801B18BF0120A3
:108668004FF00A0B84F81C0106A994F848008DF80D
:1086780018B001F0C9FF4FF0060A84F8DC0006A91B
:1086880094F848008DF818A001F0BEFF102384F874
:10869800DD0006A994F848008DF8183001F0B4FF01
:1086A8001123C4F89C0006A994F848008DF81830E6
:1086B80001F0AAFF1223C4F8A00006A994F8480004
:1086C8008DF8183001F0A0FF1323C4F8A40006A900
:1086D80094F848008DF8183001F096FF1423C4F878
:1086E800A80006A994F848008DF8183001F08CFF0E
:1086F8001623C4F8AC0006A994F848008DF8183081
:1087080001F082FF172384F8B10006A994F8480005
:108718008DF8183001F078FF18230DEB0301C4F829
:10872800B400C4F8BC0094F848008DF8183001F083
:108738006BFFC0B21D2384F8B80084F8C00006A9F6
:1087480094F848008DF8183001F05EFF1E2384F875
:10875800C40006A994F848008DF8183001F054FFB9
:108768001F2384F8C50006A994F848008DF818302E
:1087780001F04AFF2023C4F8C80006A994F848006D
:108788008DF8183001F040FF0B23C4F8CC0006A97F
:1087980094F848008DF8183001F036FF0C2306A92C
:1087A800A4F8D00094F848008DF8183001F02CFF98
:1087B800D4F89C306365D4F8A030A365D4F8A4300D
:1087C800E365D4F8A83023664FF00108D4F8AC303C
:1087D8000590A4F8D200636684F8B080C4F894B019
:1087E80084F898A0C4F84CB084F850A084F8688045
:1087F80084F81F81C5F84893FEF77AFD404B009630
:1088080032464FF0FF3105F55A70C5F84473C4E994
:108818000B6684F8198185F89164C5F8408306F0E1
:1088280045F9384B009632464FF0FF3105F5607038
:1088380006F03CF9344B009632464FF0FF3105F50F
:10884800667006F033F902AF304B009632464FF0AF
:10885800FF3105F5806006F029F9384606F0BAF8C8
:1088680097E8030004F5927383E80300284B294F27
:108878001E60294BC5F84C33284BC5F85433284B98
:10888800C5F85C33274BC5F85033274BC5F8583328
:1088980005F553703B68984704F5A67003F088FB0C
:1088A80020B1112630460DB0BDE8F08F204601F00A
:1088B8001DFB0028F5D101F041F8B8B91B4801F0BB
:1088C80067FB06460028ECD17B69984703F006FE53
:1088D800BB6D94F819019847FB6A9847012385F8FE
:1088E8009234DFE70326DDE70926DBE71326D9E71D
:1088F800000C0020C811002000040001E41600202C
:10890800357C000895740008DD740008BD6C00080B
:10891800C41100202CFA0008E16E0008956E0008CA
:10892800796C00086D6E0008456E0008E80C0020A0
:1089380008B5034B0020C3F84003FEF781F908BDD2
:10894800C811002010B5FFF7A7F90A4C60B90A4B07
:1089580093F81831022B02D1084BDB6A98470123A0
:10896800C4F84033002010BDD4F84003013818BFC4
:108978000120F8E7C8110020000C00202CFA00089C
:1089880038B5134C04F55A7006F0EEF804F560702B
:1089980006F0EAF804F5667006F0E6F804F580607B
:1089A80006F0E2F800F0B5FF0A4B0025DB6A9847AD
:1089B800C4F84053FEF7B6FD0749084840F2C452D0
:1089C80003F0AEFD0123C4F84033284638BD00BF8C
:1089D800C81100202CFA0008000C00203C060020DA
:1089E80070B52E4B8AB0054693F8DD008DF8090066
:1089F80093F8DC008DF80A0029489A6A90F8180460
:108A0800039200268DF80B0004960C46002940D0EE
:108A18000692D3F8882007921A8F93F81A118DF8C6
:108A2800151052BAADF8202093F87C2093F84830FE
:108A38008DF8243003AB8DF822008DF823200093A5
:108A48000DF10A020DF10B030DF1090105A88DF8CE
:108A5800146000F0DDFE9DF90900FEF713F960705F
:108A680004A801F02BF8B0B9049A0F2A0DD863783E
:108A78009A420AD81544AB42A3EB02012CBF00204E
:108A880001202170C0000AB070BD002323700820A7
:108A9800F9E70320F7E71320F5E700BF000C0020F3
:108AA800C81100201FB50446002800F01281007884
:108AB800412800F20881DFE810F0420048004D002C
:108AC800520056005A005F00060106010601060121
:108AD800060106010601060166006A006E007900BB
:108AE8008000830086008B0089008D00910094002F
:108AF80097009A009D00A000AF00B300BB00B7002C
:108B0800BF00C200C600CF00CB00CD000601D300D5
:108B18000601060106010601060106010601060115
:108B28000601060106010601060106010601DB0031
:108B3800DF00E300E800EC00F000F400FD00674B04
:108B480093F81831237104B010BD644B93F8303199
:108B5800237102E0606803F0C7FB0020F3E7606858
:108B680003F008FCF9E75D4B93F81A31F0E75B4B2B
:108B7800D3F8E0306360F0E7584B211D93F83001DB
:108B880003F010FCE9E7554B93F81931E0E7534B34
:108B980093F88C30DCE71C238DF808304F4B02A982
:108BA80093F8480001F030FD6060D6E74C4B043480
:108BB80093E8030084E80300CFE74A4B0434F7E75F
:108BC800494B0434F4E7494B0434F1E71A23E3E74B
:108BD8001923E1E7414B93F86830B9E73F4B5B6DE8
:108BE800C8E73E4B9B6DC5E73C4BDB6DC2E73B4B93
:108BF8001B6EBFE7394B5B6EBCE702238DF808306C
:108C0800364B02A993F87C2093F848008DF80A2087
:108C180001F0FAFC2071A0E7304B93F8DD3097E7BC
:108C28002E4B93F8393093E72C4B93F8DC308FE7D1
:108C38002A4B93F838308BE7284BDB6C9AE7274BA5
:108C480093F8503084E7254BD3F88430636084E789
:108C5800224B8FE7264B8DE7204BD3F8CC30F5E736
:108C68001E4BD3F82C31636001F05CFDA06074E703
:108C78001A4BD3F890307DE7184B93F81F3167E70C
:108C8800164BB3F88830A38067E7144BB3F88A30E3
:108C9800F9E7124BB3F8D030F5E7104BB3F8D23000
:108CA800F1E70E4B93F848200AB1062A13D1B3F81E
:108CB800A035E8E7094B93F848200AB1062A0AD1FB
:108CC800D3F8A43556E7204604B0BDE8104000F0BC
:108CD80024BE032037E7182035E700BF000C00202A
:108CE8006C0C0020B40C0020740C0020BC0C00207C
:108CF8003C0600207FB5044610B9032004B070BDBF
:108D0800A44DD5F840339A0700F171820278412AC0
:108D180000F26A82DFE812F04200480056005C0068
:108D2800600065006A007700820088008E00940069
:108D38009A00A000A600AC00B6006802BB00DD00E7
:108D4800F000170139012A0144014D015101550173
:108D580059015D016802610173019B018901AD013F
:108D6800B301BA01BF01C40168022A02680268029D
:108D7800680268026802680268026802680268029B
:108D880068026802680268026802680236023B02EA
:108D9800400245024A024F0254025E020079FEF781
:108DA800C1F80028AAD105E00379022BA5D07A4A98
:108DB80082F8303195F8913443F0200385F89134E6
:108DC80000209BE7406803F081FA0028F2D094E77E
:108DD800406803F0BFFAF8E76F4B027983F81A216D
:108DE800E8E76D4B4268C3F8E020E3E76A4E416864
:108DF80096F8300103F0CCFA00287FF47EAF636860
:108E0800C6F8E430D6E7416800293FF476AF002081
:108E180001F0EEF90028CDD011206FE74168002954
:108E28003FF46BAF0120F3E7416800293FF465AFD9
:108E38000820EDE7416800293FF45FAF0920E7E724
:108E4800416800293FF459AF0C20E1E74168002947
:108E58003FF453AF0D20DBE7416800293FF44DAFE5
:108E68000E20D5E7416800293FF447AF0F20CFE730
:108E78004A4C494B007983F81901A36D9847E36A76
:108E8800984797E7444B027983F88C2092E7424E43
:108E9800037A8DF8043096F8480096F87D308DF8FE
:108EA8000530072201A901F0C2FB00283FF425AFD5
:108EB800636896F848000193002201A901F0B7FB06
:108EC80000283FF41AAF6C36D4E9010186E80300A4
:108ED80070E7314E037A8DF8043096F8480096F81A
:108EE8007D308DF80530072201A901F0A0FB00288C
:108EF8003FF403AFB436E7E7274E037A8DF8043022
:108F080096F8480096F87D308DF80530072201A9BB
:108F180001F08DFB00283FF4F0AED4E9010106F121
:108F2800740383E8030096F81831022B7FF442AFEC
:108F380096F83031002B3FF43DAF184BDB6A984769
:108F4800FDF748FF36E7144E037A8DF8043096F89B
:108F5800480096F87D308DF80530072201A901F008
:108F680066FB00283FF4C9AEBC36ADE74368029300
:108F780001238DF80C30084B02A993F8480001F042
:108F880063FB00287FF416AFB7E64368029300231B
:108F9800EFE700BFC8110020000C00202CFA0008E1
:108FA80003795A1E0E2A3FF6A8AE934A82F8683013
:108FB80000E7914B42685A65FCE68F4B42689A6518
:108FC800F8E68D4B4268DA65F4E68B4B42681A6620
:108FD800F0E6894B42685A66ECE6874C037994F8C8
:108FE80048008DF80430062201A901F020FB002872
:108FF8003FF483AE9DF8043084F8DD30DAE67E4C29
:1090080003798DF8043094F8480094F87C308DF892
:109018000630052201A901F00AFB00283FF46DAED5
:109028009DF8043084F83930C4E6734C037994F819
:1090380048008DF804300A2201A901F0F8FA002846
:109048003FF45BAE9DF8043084F8DC30B2E66A4C3D
:10905800037994F848008DF80430092201A901F039
:10906800E6FA00283FF449AE9DF8043084F8383019
:10907800A0E6614B4268C3F89420DA649AE65E4B36
:10908800027983F8982083F8502093E65A4B426877
:10909800C3F884208EE6584B4268C3F8CC2089E692
:1090A800012B40F0A480554C2421204603F04EFAB1
:1090B800636A984201D0172020E61C2104F1280099
:1090C80003F044FA636C9842F5D14FF4807104F1CF
:1090D800480003F03BFAD4F848319842EBD1D42148
:1090E80004F5A67003F032FAD4F820329842E2D19F
:1090F800002104F5097003F029FAD4F824329842C3
:10910800D9D14FF4607104F50A7003F01FFAD4F84E
:10911800A8359842CFD1142104F2AC5003F016FAC6
:10912800D4F8C0359842C6D1334E2146304640F275
:10913800C45203F0F5F9204640F2C452002103F06E
:1091480003FA95F81B3485F8E833736FC5F8EC33E8
:1091580096F87D3085F8F83340F20123A5F8FA3304
:10916800274B96F819019B6D984723E68379012BC5
:109178003FF6C3AD204B42684068C3F82C2100F08D
:10918800D1FE47E61C4B4268C3F8902012E61A4B02
:10919800027983F81F210DE6174B8288A3F88820EF
:1091A80008E6154B8288A3F88A2003E6124B8288CA
:1091B800A3F8D020FEE5104B8288A3F8D220F9E569
:1091C8000D4B93F848200AB1062A12D1A288A3F8B9
:1091D800A025EFE5084B93F848200AB1062A08D1E4
:1091E8006268C3F8A425E5E500F099FBD9E50120FC
:1091F80084E5182082E500BF000C00203C06002012
:109208002CFA00082DE9F04387B00023ADF80030B0
:109218000646002800F0ED800361FEF73DFD20B111
:109228000124204607B0BDE8F08300F073FD002854
:10923800F6D100F069FD014618B96F48142203F011
:1092480083F96E4D95F89134012243F0040385F8B3
:10925800552485F8913433788DF804300021013B8A
:109268008DF80520ADF806100C2B00F2BA80DFE867
:1092780003F007B8B8B87881B8B88FB8AC99A80027
:10928800D5F8407317F02007CAD196F80480B8F1D2
:10929800020F45D1DFF868815A4CFEF729F896F994
:1092A800051098F848003A4601F01BFA88F839008A
:1092B800B37988F83830384607238DF80530FDF73C
:1092C80031FEFF2304F58670A5F80C31C5F8084176
:1092D80085F8047103F04EF804F58A7003F004F879
:1092E8003846FDF78DFE044640B196F9051098F80A
:1092F8004800012201F0F5F988F83900D5F89434CE
:109308003361002C71D000F0FFFC002889D195F85A
:10931800913485F81A0460F3820385F8913480E764
:10932800B8F1010F4FF00204E8D1DFF8D4908DF8BE
:10933800144099F8480089F81D7102A901F072F9E2
:10934800337989F830318DF805708DF80680FDF78E
:1093580085FC95F8913443F0100385F89134002486
:10936800CCE700226946022000F0F6FA0028F6D081
:109378001324C3E7244BB288DB6B96F90C10B06852
:109388009847D5F8403343F00203C5F84033E6E781
:1093980002A90D2000F060FB0028E0D000226946F9
:1093A8000D20E1E7164B93F81831D3B9347904F05E
:1093B800070000F0ADFA8DF8004001226946102040
:1093C800D2E7002269461220CEE78DF8072000F088
:1093D80090FA044638B900F089FA204600F08BFA72
:1093E8008CE702248AE7012488E701A800F0DEFB65
:1093F80017E7032415E700BF1C160020C81100203A
:10940800000C0020CA1100202CFA00082DE9F04FAA
:1094180099B08046059118B9032019B0BDE8F08FBE
:1094280000230361FEF738FC0646002840F0AB80B5
:1094380045460FCD0EAC0FC45A4C98F800A0B8F8AA
:109448000C7098F90EB0142204F58860314603F0C8
:109458007BF8012284F84124534C94F83021022AE5
:1094680035460BD194F81821022A07D194F81E2109
:1094780022B9BAF1010F38BF4FF0010ABAF1010F52
:109488002DD0BAF1030F2CD0BAF1000F35D102223A
:109498009DF83C30DDF84090029362F347150126B1
:1094A80094F87C108DF8321002220CA994F8480028
:1094B8008DF8302001F0A8F894F81A3194F830C1EA
:1094C80094F81D1140B20222002B6FD0BCF1010F9D
:1094D80065D1002963D1002E6DD1104627E0042202
:1094E800D6E70023DDF83C90BDF840709DF942B006
:1094F800029365F01F050126D2E74FF0000BD9460D
:10950800CDF808B0CCE74FF0010084F81A04DDE08C
:1095180005F29A420BA900F0DDFA002800F020813C
:109528001320049B33871F4B002283F81A241D4BFA
:10953800D3F89434C8F810306FE705F29A452A46F4
:109548000BA900F0C7FA0028EAD10B9B84F8280180
:10955800C4F82C5184F8303102E1B9F1000F00F061
:10956800FF80002A00F0FC804946E01C02F0D8FF8A
:1095780094F8373201332380F2E01220D1E7022039
:10958800CFE70720CFE7012047E7064B93F8912460
:1095980083F840A442F0010283F89124C7E7EEB9AA
:1095A8000220C4E7C8110020000C0020002E94D02F
:1095B8005845B8BF584694F87C308DF820000522ED
:1095C80094F848008DF8223008A901F030F80028F6
:1095D8003FF422AF9DF8203084F83930694A6A4B4D
:1095E800D2F89804D3F8904038B105F083FA664B66
:1095F80084423CBF002283F83A20198F1A8F93F8CF
:1096080030010491996A099152BA0028B9D093F8A7
:109618001B0100B9186393F81801ADF858200138F8
:1096280093F87C2093F81A411491D0F1000BD3F8E9
:1096380088108DF85B204BEB000B93F8482093F8CB
:109648003A0093F868308DF85A3009AB00934F4BC5
:1096580003904FF001008DF84C0015918DF85C20B7
:10966800A3F12F01A3F1300213A88DF84D4000F0AB
:10967800CFF8039B4FEA0B1B4BEA431B00264BEA30
:10968800801B4BEAC413B1453E4C039308BF3746D1
:109698003A46494604F59C70CDE90A669B46268001
:1096A80084F81A6402F03CFFE9B2A570C5F34215CC
:1096B800FAB2042D344E039B84F837223FF423AFCB
:1096C800072D3FF44AAF022D7FF459AF304D84F88F
:1096D8000D110420029984F80401FF2084F80C017C
:1096E80084F8281184F81431D6F8E410C4F8085125
:1096F80005F59B730AA8C4F8101184F83021C4F842
:109708002C3100F017FC00287FF437AF0A9BA4F82F
:1097180044040BA8A4F81631C4F84C3400F0CEF970
:1097280000287FF4FDAE0B9BD3B196F93900FDF705
:10973800A9FA94F83732002B3FF4FFAE0B9B0F2B9E
:109748003FF6E6AE05F58B720BA90F2000F0C2F9C3
:1097580000287FF4E5AE0B9B63F3030B84F814B188
:109768000598FDF74DFC00287FF4DBAE099B86F8D1
:109778003A00B36200F07EF900283FF406AF1320E8
:10978800D1E600BFC8110020000C0020680C0020A2
:10979800CA11002037B50B4D8DF8040004460F227E
:1097A80095F8480001A900F042FF40B1064A85F843
:1097B8001C4192F8913443F0200382F8913403B0AD
:1097C80030BD00BF000C0020C811002010B5FFF705
:1097D800B9F8044688B90A4805F0C6F9094805F0F9
:1097E800C3F9094805F0C0F900F093F8FDF780FDCA
:1097F800064BDB6A9847204610BD0124FBE700BFF3
:109808003015002048150020601500202CFA0008AB
:109818002DE9F04F8BB047780093149B90F90C809A
:1098280090F90D6090F80E908B46416819600446D7
:109838009246002F57D002238DF8103004A9C37B1D
:10984800007C8DF8123000F0DFFEB4F808C06189A2
:1098580043B26068984545466144B8BF1D466045B7
:1098680034BF00270127884209D30A218DF8101038
:10987800207C019304A900F0C7FE019B46B2B4F80E
:1098880008C0608961680CEB400E714520D3A1EBDC
:109898000C01B1FBF0FC00FB1C11C9B998450ADCAE
:1098A800237833B10223207C8DF8243006A900F0F8
:1098B800B9FE4FF0010921238DF81030207CE37B9D
:1098C8008DF8115004A98DF8123000F09DFE45B2B4
:1098D800009B8BF8005038468AF8006083F80090A7
:1098E8000BB0BDE8F08F4546F2E770477047704708
:1098F80070470020704770477047704700207047D6
:1099080000207047002070470020704700207047F3
:109918007047704770470220704702207047022046
:1099280070477047002070477047704700207047A5
:1099380000207047704770477047000010B5054C0D
:109948004FF403722046002102F0FEFD0020C4E916
:10995800000010BD881700202DE9F84381461746FE
:1099680000293FD0244B002503F1010C1A46280199
:10997800103312F8018FB8F1000F36D19A42F8D19E
:109988001E4E33680BB9C6F800C073680BB1C3F834
:1099980000C03318002401359C6083F80C900D300A
:1099A8002B01BAB206EB05153044F750C6F804C0CF
:1099B80002F0B6FDB9F1110F4FF0000398BF104C3B
:1099C8006B71D6F8083298BF24FA09F403F1010341
:1099D80098BF04F001043B442C71C6F80832404695
:1099E800BDE8F8834FF00108F9E70135202DBBD118
:1099F8004FF00208F3E700BF8F17002088170020F8
:109A08002007020010B510B3124A1368984204D117
:109A180003681360002304E00B4613B119688842F9
:109A2800FAD15168884208BF53600BB101681960C8
:109A3800D2F808328168013B00245B1A0460214691
:109A4800C2F80832102202F07FFD204610BD012026
:109A5800FCE700BF88170020054B1B6813B11A7973
:109A68008242FAD1002B0B600CBF03200020704704
:109A78008817002010B5054B186800B910BD037B86
:109A880004680BB9FFF7BEFF2046F6E788170020E9
:109A980038B5084B084C186800B938BD0379056813
:109AA800112B05D824FA03F3DB0701D5FFF7AAFF2A
:109AB8002846F1E7881700202007020028B1044B48
:109AC800D3F808320360002070470120704700BFB8
:109AD800881700202DE9F04107460E4615463AB38F
:109AE80031B3144B1C6800232CB93046FFF7E6FF4E
:109AF8000020BDE8F081A268F91A0132914210D322
:109B08002279EA54581C22895FFA80F8611D55FAB7
:109B180080F002F005FDA368246898445FFA88F392
:109B2800E2E720462468FFF76DFF002CF9D1DCE757
:109B38000120DEE7881700200238C0B211289ABF3A
:109B4800014B185C002070473BF3000830B50B4B05
:109B580093F820200446084672B100211C3305788A
:109B6800A54208D001319842CDB20CBF0448043058
:109B7800AA42F4D8002030BD1046FCE79419002012
:109B8800A019002010B5084C00232060142204F10D
:109B98000C00FF2184F82030C4E9010002F0D4FC55
:109BA800012384F8213010BD9419002010B50E4A05
:109BB80092F82010042915D8936804781C7044780A
:109BC8005C70C478807898700131DC7082F820105D
:109BD80002F11C018B4214BF043302F10C039360A1
:109BE800012010BD0020FCE794190020094B93F8D0
:109BF800200068B15A6803F11C018A4200F1FF3065
:109C080014BF043203F10C0283F820005A600120CB
:109C1800704700BF9419002010B5074B93F8202017
:109C28000446084632B15968FFF790FF10B1012386
:109C38004470837010BD00BF9419002008B5064B0E
:109C480093F820202AB15968FFF780FF08B14078BF
:109C580008BD0120FCE700BF9419002030B50A4A6E
:109C680092F82010536882F8210061B191680124AC
:109C78001C32DD78587005B99C7093420CBF034BB9
:109C880004339942F5D130BD94190020A019002061
:109C980008B5044B5968FFF759FF003818BF012071
:109CA80008BD00BF941900202DE9F3410422154E88
:109CB800044600210DEB020096F8208002F044FCD7
:109CC8000025EBB2984502D802B0BDE8F081736870
:109CD800197821705A7862709F785FB1336820468E
:109CE8009B689847FFF782FF17B901A8FFF75EFF47
:109CF8000135E6E7DB788DF804108DF805208DF83E
:109D08000730EFE794190020014B93F820007047C3
:109D180094190020034B93F82000042894BF0020D6
:109D280001207047941900201FB50024CDE9024492
:109D3800C41F8DF800408DF801100C0AADF80420FE
:109D4800090C120C8DF803108DF806208DF80730D9
:109D580002461B0A012168468DF802408DF808303A
:109D680002F04FFA002818BF0E2004B010BD2DE9EC
:109D7800F04188B017460D460F9A064600284DD088
:109D880000240121CDE904448DF810109DF8381005
:109D98008DF81510ADF81630190CCDE900441B0EDE
:109DA800CDE902448DF81930ADF81A20130C120EC3
:109DB80007948DF818108DF81C308DF81D20E3B22B
:109DC8004FEA0318002D5FFA88F803DC002008B07A
:109DD800BDE8F081013310218DF81F303A466B46FB
:109DE8000DEB010002F0A3F90346C8B9102DAC46EB
:109DF800A8BF4FF0100CDAB2624503F1010303DB90
:109E0800103D2DB20134DAE708EB020020326A4433
:109E1800315C12F8202C4A403254ECE70920D6E78E
:109E28000E20D4E70138032815D8DFE800F002082F
:109E38000C100A4B1B681B690B6000207047074B0E
:109E48001B685B69F8E7054B1B689B69F4E7034BE4
:109E58001B68DB69F0E70520704700BFB8190020D0
:109E68002DE9F041C4B00C464A9E17461D4680466F
:109E7800B8B3B1F5807F36D84FF4887200216846B0
:109E880002F062FB492300934FF48073ADF804306D
:109E98002B0C8DF80830330CADF80650ADF80A607D
:109EA8008DF80C3022460023414604A82D0E360EAC
:109EB8008DF80E308DF809508DF80D608DF80F4033
:109EC80002F02EFB04F110014B9A3B4689B268461A
:109ED80002F017F910B1012818BF0E2044B0BDE8F0
:109EE800F0810920FAE70D20F8E7000010B590B1DD
:109EF8000A4C28220021206002F026FB2368084A29
:109F08001A6000204FF0FF32C3E90302C3E90522BB
:109F1800C3E9072210BD0820FCE700BFB8190020DC
:109F280000010101024B1B6818600020704700BF48
:109F3800B819002030B1044B1B68DB68013303609B
:109F48000020704709207047B819002013B5002376
:109F58000C460193D2B101A9FFF764FF18B9019B20
:109F6800591C02D1146002B010BD99B2611A0029BF
:109F780002DD0B441360F6E702D113600720F2E715
:109F88001B0C1B0403F580332344F3E70920EAE79D
:109F980028B1044B1B681C3343620020704709201A
:109FA800704700BFB81900201FB5044600B300234E
:109FB80003A8039302F07CF9104ABDF80C3012682C
:109FC80020469380E38200F056FA98B904F118030A
:109FD800009321680123132202F08AF860B9204611
:109FE80000F049FA003818BF0120000104B010BD84
:109FF8000920FBE71020F9E70E20F7E7B819002041
:10A00800F0B5054687B01C463BB32F4E3368DB6876
:10A01800834257D894F82020002A14BF0922082226
:10A02800834205D3204600F05AFA70B110200AE0A6
:10A03800002301900093A36894F82810606AFFF742
:10A0480096FE0028EED007B0F0BD23792168B4F859
:10A0580008C0A768043B9AB209B90920F3E7B2F52A
:10A06800807F2DD8ADF80EC08DF817304FEA174C09
:10A0780004F12C033F0E8DF8117000932F0C082368
:10A088004FF0490EADF80C008DF814708DF81600DD
:10A098002F0E0DEB0300CDF808E08DF810C0ADF8D9
:10A0A80012508DF8157002F023F808B10E20CAE797
:10A0B800204600F014FA0028B8D13368DD60C2E702
:10A0C8000D20C0E70620BEE7B81900202DE9FF41A2
:10A0D8000A9D80460F4616461C46002D5AD000237E
:10A0E80003A910460393FFF79DFE18B1062004B09C
:10A0F800BDE8F081039B9C4201D80133F6D1284684
:10A1080000F05EF9002847D1264B1A78424503D063
:10A118001A79424542D10120AA68BA4240D103EBDC
:10A128008002EB6A92F801802979CDE9004304396D
:10A13800927828683B4689B2FFF792FE0028D6D16C
:10A1480095F820300194002B4FF00103009314BFC1
:10A158004246082295F82810686A3B46FFF707FE32
:10A168000028C4D1013E032EC1D8DFE806F002075B
:10A178000B0F0D4B1B681C611C62B8E70A4B1B6870
:10A188005C61F9E7084B1B689C61F5E7064B1B68A7
:10A19800DC61ACE70920AAE70F20A8E70B20A6E7B7
:10A1A8000220A4E7F0000020B81900201FB50A46D5
:10A1B8000B2A4FF00001CDE90011CDE9021107D0BB
:10A1C8000C2A13D00A2A0FD00A2005B05DF804FB28
:10A1D800012802D120238DF80030684602F011F8DA
:10A1E800002818BF0E20F0E73023F4E70B21F4E72E
:10A1F80038B5054602F000F8044678B97DB9094B30
:10A208001B680B219878FFF7D1FF38B90C21FFF7AD
:10A21800CDFF18B90A21FFF7C9FF00B10E24204667
:10A2280038BD00BFB81900202DE9F04380468FB033
:10A238000C461746002A6BD0002969D0002529460C
:10A248001D2206A8059504F091FE8DF81350344D93
:10A258002B680DF114099E88CDF804900DF11303B5
:10A2680002933B7900933B6832462146404601F011
:10A27800E4FF00284ED138683A79494602F050F98F
:10A28800384600F04FF8002846D13C7AFA79BB7975
:10A29800240444EA02241C432B689A6894423DD95A
:10A2A8009C609DF813000B21FFF780FF034658BB05
:10A2B8000C21FFF77BFF034630BB0A21FFF776FF2F
:10A2C800034608BB7B7ABA7AFF7A3F0447EA02273B
:10A2D8001F433A46334621460920FFF725FD03462A
:10A2E80090B933463A4621460820FFF71DFD03463C
:10A2F80050B92A689DF8131091700021D1604FF071
:10A30800FF31C2E90411916118460FB0BDE8F0832E
:10A318000923F9E70E23F7E70F23F5E70323F3E70C
:10A32800B819002010B50446002845D00168002956
:10A3380042D011F8013B43710322063002F0F0F8D5
:10A348002046032250F8091B043102F0E9F821687D
:10A35800CB79E3600A7A43EA0223E3604A7A43EA64
:10A368000243E3608A7A43EA0263E360CB7A2374A8
:10A378000B7B63742379212B1AD110220D3104F140
:10A38800120002F0CDF81D222168501C8B5C63621C
:10A39800085C43EA0023901C6362085C033243EACA
:10A3A800004363628A5C43EA02636362002010BD73
:10A3B800112B03DC0D22E7E70220F8E70120F6E77E
:10A3C80010B50446002854D00168002951D00B78F4
:10A3D80043714B7883608A7843EA02238360CA78A2
:10A3E80043EA024383600A7943EA026383604B7954
:10A3F80003738B79C381CA7943EA0223027BC38141
:10A4080002F00F020831103002F08AF8237B002294
:10A4180003F00F0384F8202084F82820227903F120
:10A428000800111A04290DDD21680933043AD21AEB
:10A43800085C84F82000D2B2606A84F828201944A5
:10A4480002F06EF8237922681A44002012F8043CBE
:10A45800E36212F8031C43EA0123E36212F8021CC8
:10A4680043EA0143E36212F8012C43EA0263E36220
:10A4780010BD0220FCE710B5044660B3036853B36F
:10A488000279162A29D942791A700146082251F808
:10A49800060B013002F04EF82146082251F80E0B47
:10A4A800093002F047F82368E28A5A74E38A22687E
:10A4B8001B0A93742368A269DA74A36922681B0AC9
:10A4C80013752368628B5A752368E27E9A75172381
:10A4D8002371002010BD0120FCE70220FAE738B5FF
:10A4E8000446002863D00168002960D0037B90F8F7
:10A4F800282003F00F03002A57D1083320790432AB
:10A508001344984255D363790B702368A2685A7034
:10A51800A36822681B0A937023686289DA7023682B
:10A52800E27A1A712368227B5A712368E2899A7148
:10A53800E38922681B0A2146D371227B51F8100B4C
:10A5480002F00F02083001F0EBFF237B94F828207B
:10A5580003F00F0303F108052AB1226894F82010CC
:10A56800515503F10905206894F82820616A2844A8
:10A5780001F0D6FF94F828302268E16A2B44D154C0
:10A588005A1CE16A206892B2090A81549A1C21680F
:10A59800E08D92B28854DA1C216894F82F0092B2A8
:10A5A800043388542371002038BD0933A6E70120FD
:10A5B800FAE70220F8E70000024B1A8810431880D7
:10A5C800704700BFBC19002008B5074B1B883BB17A
:10A5D800FEF7B8F900280CBF00206FF0020008BD94
:10A5E8006FF00100FBE700BFBC19002010B5034B5A
:10A5F80000241C80FEF79CF9204610BDBC190020E1
:10A60800B0FA80F04009704782B018B9084602B025
:10A6180000F0CAB8002002B0704710B9084600F030
:10A6280077B9704710B9084600F08EB970470346ED
:10A63800084611460BB900F0E5B90020704710B97B
:10A64800084600F071BD704710B9084600F006BA18
:10A658000020704710B40446084611461A46019B6C
:10A6680014B910BC00F018BA10BC7047034608466D
:10A6780011460BB900F042BA0020704710B40446E6
:10A68800084611461A4614B910BC00F0AFBA0020AB
:10A6980010BC704730B40546084611461A46DDE935
:10A6A80002341DB9029430BC00F02EBB002030BC2F
:10A6B800704710B9084600F0DFBB0020704710B99A
:10A6C800084600F06FBD0020704710B9084600F03A
:10A6D800EEBB0020704710B9084600F0EBBB002025
:10A6E80070470346084611460BB900F005BC002028
:10A6F800704710B40446084611461A46019B14B91F
:10A7080010BC00F0FBBB092010BC704710B4044615
:10A71800084611461A4614B910BC00F063BDC8B209
:10A7280010BC70470048704701000102064B10B585
:10A738001B6A0446984730B10448054B20449842A8
:10A748008CBF0020012010BD2CFA000840C220C98F
:10A7580080B92A00F0B5114B85B00C4610491F5638
:10A76800054601F049F80F4BE4B25E6A072D4FF039
:10A778000103CDE9024301460AD105220023CDE9B0
:10A7880000234FF47A727A431846B04705B0F0BDFB
:10A7980008220020CDE900203A46F5E777F30008C3
:10A7A80050F300082CFA00081FB500230093037823
:10A7B800013B372B21D8DFE803F01C242020201E82
:10A7C800202020204143454E2055585B5E6164207F
:10A7D8006C1E6E73787A20207D8126202020202010
:10A7E800202020202020202083858A2020838A2062
:10A7F8008C90C3780BB102230093009805B05DF8E4
:10A8080004FB8378F6E743788DF8043005238DF848
:10A8180005308378003B18BF01235B008DF80630B4
:10A8280010238DF80730304B1B6801A803F55872C8
:10A83800CDE9022300F0C0FF0090DEE74023DBE70C
:10A848002023D9E7827890F9013012B9274AD35CDE
:10A85800D2E7274AFBE7827890F90130002AF8D13D
:10A86800244AF4E740F6B833C6E74FF47A73C3E7EF
:10A878004FF4FA63C0E741F28833BDE741F27073E1
:10A88800BAE71D484FF47A7101F02EFE00F5FA6020
:10A89800D2E71A4BB0E7144B1B6803F55873ABE7C4
:10A8A800114B1B6803F55B73A6E71023A4E70E4B57
:10A8B8001B68A1E74FF0834300939EE7104BFBE72B
:10A8C800104B99E740F21113ADF8003095E70323D8
:10A8D80092E790F901300C4AB9E70C4990F9010068
:10A8E80000F08AFFA8E700BFC4190020FFF30008A2
:10A8F80007F400080FF4000818FCFFFF00EA063709
:10A908009A99094040F7093777F3000850F300088F
:10A9180037B50B4B02781B680C2101FB02335B7ABD
:10A9280003EB4304074B1D6803690093C36842782F
:10A93800816805EBC40000F0DFFC03B030BD00BF48
:10A94800C4190020C019002070B586B0027B6423AA
:10A95800ADF80030012A4FF00003CDE90133CDE90D
:10A9680003338DF802308DF8143030D0022A39D0F4
:10A978005ABB03684BB343683BB31F4D80682B60D9
:10A988001E4B18226946186001F0CAFD1C4B2C6842
:10A9980093E807000C3384E8070093E8070004F104
:10A9A8000C06032386E80700A4F86C33012204F59B
:10A9B8005B7104F5587000F090FC2B684FF6B0728C
:10A9C800A3F878230522C3F87C2306B070BD0A4992
:10A9D80008684360036100F55B7100F5587000F08A
:10A9E8007CFCF2E7044B1B68B3F86023B3F86C13E4
:10A9F8000A43A3F86023E8E7C4190020C01900201F
:10AA080020F1000808B503460A2924D8DFE801F038
:10AA180006232323230B161B23212100BDE808400E
:10AA28000068FFF783BE90F900009978052271B994
:10AA380000F013FC003818BF012008BD052293F967
:10AA480000000021F4E790F900005978EEE70221B0
:10AA5800EEE70722F3E70020EFE7000010B50479DE
:10AA68001CB1012C0BD0002010BD0A4B01681B68DB
:10AA7800012203F5587000F030FC0120F4E7054B83
:10AA880001681B68224603F55B7000F026FC20462F
:10AA9800EAE700BFC4190020F7B50528144D1C4685
:10AAA800A8BF052058700E462946174600F0A4FE98
:10AAB80094F90130A070072B13D1322000F09CFDCF
:10AAC8000C4BDB6D0546984704F10C02083403462D
:10AAD800019200943A463146284600F092FD03B0B0
:10AAE800F0BD054A55F82310D05C00F07DFDE7E77E
:10AAF80050F300082CFA000877F300082DE9F04F0E
:10AB0800344F90F901607B68D0F804908BB004460C
:10AB1800884698470546002859D1E37C73B92E4AE0
:10AB28002378126803EB4303990002EB8303D3F8FD
:10AB38000490B9F1000F01D152F80190274B484613
:10AB480013F906B0FB689847A37CD7F818A02289A8
:10AB58000993072E28D100230121CDE90223204A99
:10AB68000693CDE90431CDE907330521CDE900216C
:10AB78004FF47A7202FB0BF24CF250311846D04770
:10AB8800637C13B3174B995D7B6D0D31C9B22846B1
:10AB98009847E07C3246494600F040FE88F800605D
:10ABA80001200BB0BDE8F08F002101250823CDE975
:10ABB8000013CDE90715CDE90511CDE9031102927E
:10ABC800A1782B465A462846D9E7074BDBE70020F1
:10ABD800E7E700BF2CFA0008C419002077F3000843
:10ABE800854501000FF40008FFF300082DE9F04F38
:10ABF8008DB090F90130DFF8FCA0DFF8FC90CDE9CA
:10AC08000A123E4A12F903B00278DAF800300C252D
:10AC180005FB02333A4A5B7A126803EB430302EB03
:10AC2800C303044693F9021090F9020000F0DFFD17
:10AC38003449064694F9010000F0DEFDA268616817
:10AC48008046304600F005FD2178DAF80020D9F872
:10AC58000C306943074650589847D9F81C309C4631
:10AC680094F901300025072B4FF47A63CDE9075397
:10AC7800CDE905552DD10123CDE903530523CDE9B0
:10AC880001534FF47A7303FB0BF3009339464346A1
:10AC980046F2A81228466746B8472378DAF8002013
:10ACA8000C214B4394F90110D05800F0D9FDA1892B
:10ACB80094F90100FFF74EFD0B9B217B1860D9F832
:10ACC8005430284698470A9B01201E700DB0BDE8F5
:10ACD800F08F01200823CDE90350CDE901032A466E
:10ACE800CDF800B0654643463946A84701200546D9
:10ACF800D3E700BFC41900202CFA000877F3000836
:10AD0800C019002050F300082DE9F04F8FB000243F
:10AD180005468A46914698460494ADF81440ADF825
:10AD2800024007264FF0010B2B7AA34206D9686828
:10AD380004A9204400F0F2FB00285ED102238DF81C
:10AD4800083002A86B7A8DF80A30FFF72DFDAB7A30
:10AD58008DF81D309DF811308DF81E309DF8123099
:10AD68008DF81F309DF810308DF82030EB7A8DF873
:10AD780021302B7B8DF822306B7B8DF8233010230C
:10AD88008DF81C608DF824303A4E8DF82C000DF1AA
:10AD980002030A9305238DF82D3033680C9307239B
:10ADA800ADF834302B6806930DF1120204AB0DF1A7
:10ADB800110106A800F0CCFB072805460BD1306826
:10ADC8000C22002100F5587001F0BEFB3368BDF875
:10ADD8000220A3F860239DF811308AF800309DF80E
:10ADE800123089F800309DF8103088F80030189B30
:10ADF80028461C700FB0BDE8F08F9DF81330BDF8E1
:10AE08001470ADF802702044C4B2F3B917B3194AEC
:10AE180000201168072602464FF00C0C062B1BD1A8
:10AE28000CFB00FE51F80EE0BEF1000F04D00BFA47
:10AE380000F23A4397B2012201301028EED1002ADD
:10AE48003FF472AFADF802706EE75A1E042A01D9BA
:10AE5800062BDCD0062667E747FA00FE1EF0010F36
:10AE6800EAD00CFB00FE51F80EE0BEF1000F08BF5F
:10AE78000626E1E7C419002038B505464068FFF703
:10AE880055FC0522841D002195F90000E4B200F06C
:10AE9800E4F908B904F0FD0495F90100072200213E
:10AEA80000F0DBF908B904F0FB04204638BD0020A7
:10AEB8007047000010B503780F2B044618D8406877
:10AEC800FFF734FC22780B4902EB42020968831C25
:10AED80001EB820051F82220DBB21AB903F0FD031E
:10AEE80058B210BD032B06BF626842600223F7E721
:10AEF8000020F6E7C4190020022070472DE9F04F22
:10AF0800DFF838810446D8F8000099B0894617461A
:10AF180000211E460122032300F55870CDE90611D1
:10AF2800CDE908118DF814108DF81510ADF816300C
:10AF380000F0B5F938B9D8F80020B2F8603343F01A
:10AF48000303A2F86033D8F80020637A8DF828301C
:10AF580002F55871CDE90B12394A94F90830126894
:10AF68000D920DF116020F922268109262681192EA
:10AF7800D4E90301A27A8DF8482001228DF84920EE
:10AF880013AA82E803001025227DE18A8DF8293072
:10AF980018468DF85420ADF83850FFF7DBFB0AABA4
:10AFA80017930DF11503169000933146019705ABE1
:10AFB80006AA10A800F0BCFB064698BB9DF8141022
:10AFC800204F013901F090FA1F4B1B690393C4B25B
:10AFD8004FF00C0B04F160036B44D8F8000013F831
:10AFE80048AC9DF814300BFB0AFC01343946B4FB1D
:10AFF800F3F203FB1244D0F87C33B0F9782350F80D
:10B008000C00DDF80CC0E4B2E04728B189F800A0D4
:10B01800304619B0BDE8F08F013D15F0FF05D9D1D4
:10B028000D26F5E70C2801BFD8F80020B2F86033E8
:10B0380043F00303A2F86033EAE700BFC419002015
:10B04800C0190020400D03002CFA0008F8B5067955
:10B05800012E054601D80620F8BD0F2E2BD803680F
:10B06800187A40F303000522002140B200F0F5F8F9
:10B078002B680446187A40F303100522002140B2D9
:10B0880000F0EBF8A8B1B4FA84F4640929680B7AE3
:10B09800086843F3030243F3031352B25BB29A42C4
:10B0A800C8BF0124FFF742FB48B9002CD3D10420C4
:10B0B800D2E70124EAE70320CEE70520CCE7002CFD
:10B0C800FBD10C4F29683B6806EB460003EB800078
:10B0D8000C2201F025FA3A680C2303FB06232046CC
:10B0E8005C72B2F860130123B3400B43A2F86033DB
:10B0F800B2E700BFC419002010B4017801290ED9A5
:10B10800084B18680C234B43C4180022C250C4E9EA
:10B11800012200F5587010BC102200F0A7B80020DA
:10B1280010BC7047C41900202DE9F04186B05023A7
:10B138008DF81430037A102B074630D14368DD7B35
:10B148006DBB0224A8466426062C14D87A68535D81
:10B1580003932A44517843EA01230393927843EAFC
:10B1680002437343CDE9033863B968468DF800405C
:10B17800FFF7C2FF0DE0CDF80C808DF81480CDF8F4
:10B188001080F2E703AB01A801938DF80840FFF7A0
:10B198005DFF0134E4B2102C05F10305D4D106B0EB
:10B1A800BDE8F0811FB502680379116851B901A89B
:10B1B8008DF80430FFF7A0FF78B9002040B205B041
:10B1C8005DF804FB02A802928DF80C30FFF73EFFF1
:10B1D8000628F2D8024B185CF0E70320EEE700BF20
:10B1E80070F30008C90020B9034B0B449856C0B24D
:10B1F8007047024BF9E700BF7FF30008BFF3000870
:10B20800F0B59A42069D03DB9DF914309A4220DD81
:10B218000020F0BD03EB430331F814C005EB8303B2
:10B2280000264CFA06F7FF0707D51F7A07F00F0E1E
:10B23800724502DBB2EB171F0DDD0136102E03F14C
:10B248000C03EED10134E4B22301DBB29842E1D819
:10B25800DEE70024F8E70120DBE7884204DB9042C0
:10B26800CCBF0020012070470020704710B514099A
:10B27800B4EB111F03464FEA11100ED391420CD2C2
:10B2880002B201F00F0133F81240012000FA01F177
:10B2980024EA010123F8121010BD0020FCE7F0B5E4
:10B2A80028B100EB410501270020914200D3F0BDF1
:10B2B800002435F802CB234607FA04F636EA0C06D2
:10B2C80008BF013304F1010408BFDBB2102CF3D12D
:10B2D80018440131C0B2C9B2E7E710B500B149B9A5
:10B2E80010BD31F8134020F813400133DCB2A242FC
:10B2F800F7D8F5E70023F9E782B030B5048804935E
:10B308006AB9B3F5616F18D349F6AF2542F21072E6
:10B31800AB4298BF4FF47A72944238BF1446012C5E
:10B3280038BF01246143BDE83040C3688B428CBFFD
:10B338005B1A0023C36002B070476422ECE7000088
:10B348002DE9F04F91B01546DDF86C8004939DF817
:10B35800683009930C46064603F0C2FB684ADFF8DA
:10B36800A4B10590A8F5F633303BB3FBF2F3534391
:10B3780003F5F63203F5A83303F5C07303931823D6
:10B3880013FB054330320692089300254FF0FF3A2D
:10B39800089BA34207D1002D14BF50464FF0FF3041
:10B3A80011B0BDE8F08FBDF97030ADF82C300B99B5
:10B3B800CDF86C804046CDF8288003F021FBB4F826
:10B3C80000906EB9B8F5616F5BD349F6AF2242F2CF
:10B3D8001073904598BF4FF47A73994538BF9946D2
:10B3E8004B46012B38BF01230793002E52D1B9F1E8
:10B3F800640F48D1A0605F46A1680EA803F022FB45
:10B408000F9B0093DDE90A120E9B0CA803F079FA52
:10B41800049B0C9A0BB9099B2BB12369BB4202D13F
:10B42800394B9A420DD9394BE760984509D9002321
:10B43800ADF83430069B0D990C93184603F0E0FAEA
:10B44800A060606800B9E760276126B103F052FB8D
:10B45800E3680344E360D4E903329342059B1D99F2
:10B468006360079B88BFE2604B43E168994202D260
:10B478000498A8B9A6B101231D442375EDB2183468
:10B4880086E76423A9E7B9F57A7F0ABF204F214FE1
:10B49800A060B1E7049B0BB9C4F80CB05F46D0E7D5
:10B4A80000209342207506D85B1A9A4505F10105DC
:10B4B80028BF9A46EDB2002EE1D1B9F1640F164AC1
:10B4C800ADF8346019D049F6B023B9F57A7F18BFC2
:10B4D8001346904584BF039A9B180C931C9B0093BA
:10B4E8000CAF97E806001B9B384603F00AFA97E86A
:10B4F800030003F085FA8246C1E74FF46163E8E789
:10B508008051010040771B007F5101002FEC0100A2
:10B5180080A81201002E930230EC01000378032B5F
:10B5280014D1437803F00F021B098A704B7083789B
:10B538008B80C27843EA02238B800379C3F302121B
:10B5480003F00F03CA700B70052070470020704786
:10B558002DE9F34798464379057990F907609146B4
:10B56800044690F906208A4683B190F9087075B3AD
:10B578000F2A12D194F909200F2E1ED194F90A60CE
:10B58800072D24D1002F08BF012720E090F90B7068
:10B5980090F9092090F90A60E9E7A369019394F901
:10B5A80015300093216994F91430207BFFF728FEA9
:10B5B8000028E1D105F0FD05DEE794F91D30B3421E
:10B5C8000FDC94F91C30B342DADA05F0FB052846A3
:10B5D8008AF8002089F8006088F8007002B0BDE899
:10B5E800F0871E46CCE70000024B03FA00F0B0FBE0
:10B5F800F1F0704740420F004FF4FA53B3FBF0F0FC
:10B60800704730B54FF47A750C1F6A4300FB04226B
:10B6180052001EBF00F1FF341219B2FBF0F2914242
:10B6280038BF1146039A1160820048431CBF01309D
:10B6380040084FF47A71121A01FB1323002BCABF7A
:10B6480003F2E73393FBF1F1B3FBF1F1049B1960CB
:10B6580030BD38B5400014460D46F5F7B3F801463D
:10B668002846F4F7FDFF2146F4F7FAFFF4F7ECFE5D
:10B6780003F0AAFCF4F7C8FF40B238BD2DE9F74F34
:10B68800019300231F469C461C01058A5FFA84FE2D
:10B6980004F0F004A54206D8019B82F800C01F7090
:10B6A80003B0BDE8F08F0EEB4E054FEA4309AD003D
:10B6B8000024466836F809602641F60727D58668CB
:10B6C80006EB050A765916B3067836B9466926B1E7
:10B6D80036F809602641F60719D59AF8086090F9F6
:10B6E80001B046F303084FFA88F8D8450FDC46F353
:10B6F800031676B25E450ADB9AF8096006EB46083F
:10B70800C66806EBC806367D4EB90137FFB201346C
:10B71800102C05F10C05CCD10133DBB2B4E70CF1E8
:10B7280001060EEB040801F80C805FFA86FCEEE7D0
:10B738002DE9FF4704464068DDE90C671D468A4647
:10B74800914603F0D7F923681B1A3B604FF00008B5
:10B758000123337085F80080636813B1236883423E
:10B7680024D8CAF80080D4F81CC0A3699CF800E06B
:10B778000393D4E9030101AB83E80300237D00931D
:10B78800DCF80C10237A627A7046FFF7D9FD33464D
:10B7980038602A46E0694946FFF770FF2B782BB1DD
:10B7A800C7F80080002004B0BDE8F0873378002B8C
:10B7B80014BF0B200C20F6E737B590F9002090F95C
:10B7C8000250954204460FD0013A52B295420BD02E
:10B7D800A368019394F9013000936168E0782B46DF
:10B7E800FFF70EFD0028EFD0104603B030BD8842A9
:10B7F800B8BF08467047000051F82000054B984232
:10B8080005D0054BC31A58425841400070470120E3
:10B81800704700BF90D0030020A1070005281FB57E
:10B828000ED80C4B53F820300093CDE901120A4B87
:10B8380001220021022002F069FE05B05DF804FB38
:10B84800CDE90012054B01220021022002F05EFE24
:10B85800F3E700BF84F4000817F4000836F4000882
:10B8680007B5054BCDE9000101220021022002F0B5
:10B878004DFE03B05DF804FB52F4000810B5102229
:10B8880004460021F13000F05FFE0021C4F81411D5
:10B898002046F022BDE8104000F056BE0246084699
:10B8A800102100F0A5B92DE9F0430446D0F81401A1
:10B8B80085B00E46154604F2011988B3C0F1100888
:10B8C8009045474628BF1746BAB2484400F028FEBC
:10B8D800D4F814313B440F2BC4F814312DD9A845A2
:10B8E8002BD204F1F00304F5807113F8012F187CB2
:10B8F8008B4282EA00021A70F7D104F1F108102293
:10B908004146684600F00CFE22466946684600F04B
:10B91800E9F910226946404600F002FE3E44ED1B5C
:10B9280004F5807804F1F107102D09D8AAB2314640
:10B93800484600F0F5FDC4F8145105B0BDE8F083A1
:10B9480004F1F003711E13F8012F11F8010F43459C
:10B9580082EA00021A70F6D110223946684600F0D1
:10B96800DFFD22466946684600F0BCF910226946A8
:10B97800384600F0D5FD1036103DD5E7F0B589B052
:10B988000C46102200210546684600F0DDFD2246DF
:10B998006946684600F0A6F99DF90030002B6A4612
:10B9A8004FF0000143DA137812F8010F01315B0000
:10B9B80043EAD0130F2902F8013CF4D19DF80F3067
:10B9C8005B0083F08703D4F81401DBB210288DF8EC
:10B9D8000F303BD104F58073694604F5887013F87D
:10B9E800016F11F8012B984282EA06021A70F6D10B
:10B9F80004F1F00304F5807113F8012F187C8B42D1
:10BA080082EA00021A70F7D110220DEB020004F14D
:10BA1800F10100F085FD2246294604A800F062F9EC
:10BA280010220021684600F08FFD09B0F0BD1378A0
:10BA380012F8010F01315B0043EAD0130F2902F815
:10BA4800013CF4D19DF80F305B00BCE79DF9003054
:10BA5800002B6A464FF0000137DA137812F8016FAD
:10BA680001315B0043EAD6130F2902F8013CF4D1F7
:10BA78009DF80F305B0083F08703471CDBB28DF81D
:10BA88000F30102F04EB0003C0F10F064FF08002B7
:10BA980088BF002600F5817083F801210021324615
:10BAA80020443E4403F062FAC4F8146104F580733C
:10BAB800694604F5887013F8016F11F8012B984254
:10BAC80082EA06021A70F6D192E7137812F8016F2B
:10BAD80001315B0043EAD6130F2902F8013CF4D187
:10BAE8009DF80F305B00C8E70A780378534003706D
:10BAF8004A784378534043708A78837853408370F8
:10BB0800CA78C3785340C3700A79037953400371E4
:10BB18004A794379534043718A79837953408371D1
:10BB2800CA79C3795340C3710A7A037A53400372BE
:10BB38004A7A437A534043728A7A837A53408372AB
:10BB4800CA7AC37A5340C3720A7B037B5340037398
:10BB58004A7B437B534043738A7B837B5340837385
:10BB6800CA7BC37B5340C373704710B50B781478F6
:10BB78006340037054784B786340437094788B78B3
:10BB880063408370D478CB786340C37014790B79A1
:10BB98006340037154794B796340437194798B798D
:10BBA80063408371D479CB796340C371147A0B7A7B
:10BBB80063400372547A4B7A634043728B7A947A67
:10BBC80063408372D47ACB7A6340C372147B0B7B55
:10BBD80063400373547B4B7B63404373947B8B7B41
:10BBE80063408373CB7BD27B5340C37310BD00008B
:10BBF800A1F11003DBB2102B2DE9F04704D8374C24
:10BC080024FA03F3DB0705D4002382F8F030FF2081
:10BC1800BDE8F087531E4418A0424ED101F11C0321
:10BC28009B005FFA83F9C3F30313013B2C4D82F8A1
:10BC3800F03001240B46D618B3FBF1F001FB1030AD
:10BC480010F0FF0016F804AC16F803EC16F802CC56
:10BC580016F8017C36D115F80E8015F80CE015F8A9
:10BC680007C015F80A70E00900EB400084EA0808EC
:10BC780000EBC0006400C0B2E4B24440C246581AA7
:10BC8800C0B212F800808AEA080A02F803A0104439
:10BC9800043390F801808EEA080E86F801E090F8E7
:10BCA80002E08CEA0E0C86F802C0C078DBB247408E
:10BCB8009945F770BFD80020AAE710F8015B03F890
:10BCC800015FA9E71829DAD9102801BF15F80AA0D9
:10BCD80015F80EE015F80CC0EF5DD0E70101010082
:10BCE8009CF600082DE9F04FA3B092F8F0301D91B2
:10BCF8001B920193002B00F0538101461EA8FFF709
:10BD080034FF1B9BA74CA84DA84E10330293002369
:10BD180003939DF87C0004909DF886000590205CB4
:10BD280006909DF87B000790205C089004989DF889
:10BD380081C0205C099014F80C000A909DF88000DE
:10BD48000B909DF885009DF878809DF87DE09DF822
:10BD580082A09DF887900C909DF87A00029B1C9316
:10BD680014F80A2014F8093014F8081014F80E70A2
:10BD78000D90205C0E909DF87F000F90205C109035
:10BD88000B98205C11900C98205C12909DF8840010
:10BD980013909DF8790014909DF87E001590205C12
:10BDA80016909DF883001790205C18901398205CDB
:10BDB80019901498205C1A90039801300390029807
:10BDC800DDF804B0103002909DF80C00834536D899
:10BDD8008DF878108DF87A2009990E9A8DF87C10D4
:10BDE8008DF882201199069A8DF880108DF87E20A2
:10BDF8001999169A8DF884108DF886200A99189A40
:10BE08008DF87D108DF887201299109A8DF87B3067
:10BE18001B9B8DF881108DF883201A99089A1D981C
:10BE28008DF885108DF87F201EA903EB0B128DF875
:10BE38007970FFF79AFE002023B0BDE8F08F15F85F
:10BE480008B082EA03008BEA000016F80EB080EA18
:10BE58000B008DF8780015F80E004B40434016F89B
:10BE68000A0043408DF8793081EA070315F80A1073
:10BE7800594016F80930594016F808308DF87A10EC
:10BE88007A40534015F8092053408DF87B30089AC2
:10BE9800069B5340049AAA5C534016F80C20534062
:10BEA8008DF87C30DDE908325A4015F80C305340E3
:10BEB800059AB25C53408DF87D30DDE909325A406D
:10BEC800059BEB5C5340079AB25C53408DF87E307B
:10BED800069B0A9A5340049AB25C5A40079BEB5C53
:10BEE8005A408DF87F200E9B109A53400B9AAA5CFB
:10BEF80053400C9AB25C53408DF88030DDE9103223
:10BF08005A400C9BEB5C53400D9AB25C53408DF841
:10BF18008130DDE911325A400D9BEB5C53400F9A9A
:10BF2800B25C53408DF88230129A0E9B53400B9AA4
:10BF3800B25C5A400F9BEB5C1C995A408DF88320E9
:10BF4800169B189A5340139AAA5C5340149AB25CF1
:10BF580053408DF88430DDE918325A40149BEB5C6D
:10BF68005340159AB25C53408DF88530DDE919329B
:10BF78005A40159BEB5C5340179AB25C53408DF8BE
:10BF880086301A9A169B5340139AB25C5340179AFC
:10BF9800AA5C1EA853408DF88730FFF7A5FDB8E6C8
:10BFA800FF2049E79CF600089CF400089CF500086F
:10BFB80008B538B1044A05491060D82200F0B0FA33
:10BFC800002008BD0220FCE7C8190020CCFB0008AF
:10BFD8000A4B1A6870B5002302F1180503EB031425
:10BFE8002E5D864204D1183422440A60002070BDB8
:10BFF80001330B2BF2D10320F9E700BFC819002049
:10C008002DE9F041CCB00646DDF8488117461C46BC
:10C018000D4631B3B8F1000F23D006A8FFF72EFC68
:10C02800204601A9FFF7D4FF0446B0B9019906A834
:10C038000131FFF733FC26B11022314606A8FFF77D
:10C0480032FC3A46294606A8FFF72DFC06A902A8A5
:10C05800FFF794FC029BC8F8003020464CB0BDE8BE
:10C06800F0810224F9E7000030B595B013A9044621
:10C07800FFF7AEFF002830D11B490C2303FB00F269
:10C08800555CA5422BD1139B187C1090D87B0F9040
:10C09800987B0E90587B0D90187B0C90D87A0B905B
:10C0A800987A0A90587A0990187A0890D87907905F
:10C0B800987906905879059018790490D878039063
:10C0C800987802900A445B78019393680093002261
:10C0D800064B1146022002F019FA15B030BD0130A6
:10C0E8000B28CBD1F9E700BF14F900089CF700082A
:10C0F8000B2B10B402D810BCFFF782BF032010BC72
:10C10800704730B50D4685B01446014668B103AA9C
:10C11800002000922A460390FFF772FF18B903988F
:10C12800001B18BF012005B030BD0220FBE72DE938
:10C13800F0430D46BFB014469946804620B31BB362
:10C1480011F00F0122D1F02201A800F0FDF92046DC
:10C158006946FFF73DFF044648B9009801AA102137
:10C168000130FFF745FD2E46AF1BFFB21EB9204632
:10C178003FB0BDE8F08301AA09EB070108EB07000F
:10C18800FFF7B0FD103EEFE70224F0E70524EEE7E5
:10C19800F0B5184E3468024685B00846002304F10D
:10C1A800180103EB03154F5D97421ED10D2A05F1C7
:10C1B800190513D10023CDE90033CDE902330C2250
:10C1C80010216B46FFF7B3FF04463068102269461A
:10C1D800284400F0A5F9204605B0F0BD014610221C
:10C1E800601900F09DF90024F5E701330B2BD8D135
:10C1F8000324F0E7C819002009B1FFF7C9BF0220DE
:10C2080070471FB51446A0B10C2A01D10B2912D1D1
:10C218000023CDE90033CDE902330A466B461021ED
:10C22800FFF785FF18B969462046FFF7B1FF04B04C
:10C2380010BD0220FBE70320F9E7F8B51E46DDE94B
:10C2480007479DF818505BB354B34FB3212D29D835
:10C2580019462A46204600F063F90122631C691E2C
:10C26800B018FFF764FFF8B9E37ADB093B70EBB964
:10C278006319204613F8012C13F8021C120642EA2F
:10C28800014213F8041C0A4313F8031C012342EA71
:10C298000122291FFFF735FF003818BF0120F8BD1C
:10C2A8000220FCE70520FAE70720F8E70420F6E774
:10C2B80010B5044628B1044B5B69984720600020FC
:10C2C80010BD0220FCE700BF2CFA000808B50146A3
:10C2D80030B1044B0822186800F022F9002008BD8C
:10C2E8000220FCE7C819002008B530B1044B082229
:10C2F800196800F015F9002008BD0220FCE700BF0E
:10C30800C81900207FB5124E0023044602A80193E5
:10C318000D46FFF7E9FF33685B6901936CB102AA28
:10C32800082312F8011B41B9013B13F0FF03F8D1B0
:10C3380002A8A04702A8FFF7C9FF35B1019B23B99E
:10C3480001A8A8473368019A5A61002004B070BD5B
:10C35800C819002008B5014638B1054B18680822ED
:10C36800104400F0DDF8002008BD0220FCE700BF03
:10C37800C819002008B538B1044B196808221144BF
:10C3880000F0CEF8002008BD0220FCE7C819002004
:10C39800034B1B6802280CBF1961596100207047C4
:10C3A800C819002041B1054B1B6802280CBF1B6946
:10C3B8005B690B600020704702207047C819002095
:10C3C80030B58FB0002405460CA80994FFF78CFF00
:10C3D8009DF8373007939DF8363006939DF8353031
:10C3E80005939DF8343004939DF8333003939DF8FA
:10C3F800323002939DF8313001939DF8303000932C
:10C40800224621461E4B022002F080F80AA8FFF7B8
:10C41800B1FF9DF82F3007939DF82E3006939DF8B5
:10C428002D3005939DF82C3004939DF82B30039301
:10C438009DF82A3002939DF8293001939DF8283001
:10C44800009322460F4B2146022002F05FF809A90B
:10C458002846FFF7A7FF9DF8243003939DF8253061
:10C4680002939DF8263001939DF8273000932246C9
:10C47800054B2146022002F049F80FB030BD00BF3D
:10C48800F8F7000836F8000874F8000808B5002026
:10C49800FFF7EAFD0120FFF7E7FD0920FFF7E4FDBC
:10C4A8000820FFF7E1FD0020FFF78AFF002008BD04
:10C4B80010B504460B20FFF7D7FD0C20FFF7D4FD7D
:10C4C8000920FFF7D1FD0820FFF7CEFD0A20FFF76E
:10C4D800CBFD2046FFF774FF002010BD014B18600C
:10C4E800704700BFF80000200B4A30B514680B4DA8
:10C4F80043F2390305FB04331360091A6FF0004255
:10C50800B3FBF2F2C2EBC27201319B1A93FBF1F258
:10C5180001FB1233184430BDF80000206D4EC641AF
:10C5280001380A44914200D1704711F8013B00F8E4
:10C53800013FF7E710440A44914200D1704711F8CF
:10C54800013B00F8013DF7E702F010BD30B530B10E
:10C558000A4D01444FF0FF33814201D1D84330BD29
:10C5680010F8012B5340082243F30004013A2C40F1
:10C5780092B284EA5303002AF6D1EDE72083B8ED9E
:10C5880001207047054B4FF400529A62044B1B6818
:10C5980013B15B6803B11847704700BF0004004837
:10C5A800CC1A0020054B4FF480529A62044B1B684A
:10C5B80013B1DB6803B11847704700BF0004004897
:10C5C800CC1A0020012070470120704701F048B9BB
:10C5D80001F036B910B501F019FE0E21044640F6F7
:10C5E8001F1001F02DF92046012101F0F9FDBDE8E9
:10C5F800104001F0D7BA000070B50C4E01EB4003B3
:10C608000D46B3654FF6FF71002304461A460846E7
:10C6180001F05EFB96F85600002101F0E1FD294685
:10C628002046BDE8704001F095BA00BFE81A002026
:10C6380010B5044601F0AAFE01281CD101F0AEFE97
:10C6480034B11248214602F017FB104802F0DAFA1A
:10C658000F4C104B00214FF48052A1659A6194F859
:10C66800560001F0BDFD63786BB16FF07F40BDE807
:10C67800104001F053BA002340F262211A460846DE
:10C6880001F026FBDCE7A0688001F0E7D01A002063
:10C69800E81A002000040048002001F0BFB900009B
:10C6A80008B501F0C7F80438C0B2032896BF024B9A
:10C6B8000020185C08BD00BF28FA000808B501F082
:10C6C800BAFD033008BD01F049B901F009B908B550
:10C6D80001F000FD00B208BD38B50D46144601F062
:10C6E8005DFB284601F092FD0E21054640F61F101D
:10C6F80001F0A6F828460121074D01F071FD01F06F
:10C7080051FA4FF47A716143284602F0B5FA284687
:10C71800BDE8384002F076BA441B002001F03EBB69
:10C7280008B5084B002193F8560001F059FD002385
:10C738004FF4C0711A46084601F0CAFABDE808402D
:10C7480001F024BAE81A002010B5044601F01EFED4
:10C7580001281CD101F022FE34B11248214602F012
:10C768008BFA104802F04EFA0F4C104B00214FF490
:10C778008052A1659A6194F8560001F031FD637802
:10C788006BB16FF07F40BDE8104001F07DB9002328
:10C7980040F262211A46084601F09AFADCE7A068DE
:10C7A8008001F0E7D01A0020E81A002000040048B1
:10C7B80008B54FF0040001F017F9BDE80840022061
:10C7C800F5F7A2B808B500231A461946184601F02D
:10C7D8007FFABDE8084001F06DB900001D4B73B544
:10C7E8001D4D186000241D486C70C5E90144AC65F6
:10C7F80001F098FAAC8101F003FA2146204601F0D5
:10C808004BFC21460422012001F0FCFA144E154D80
:10C818004FF6FF7123462246084601F059FAFFF702
:10C82800C7FF2246104B00944FF0FF31304602F00C
:10C838003DF90E4B009422464FF0FF31284602F096
:10C8480035F9304602F090F9284602B0BDE870404C
:10C8580002F08AB9CC1A0020E81A00202DD8000866
:10C86800441B0020D01A00208DC50008ADC5000863
:10C878000128084805D1084BC17719700E3001F01E
:10C88800A7BB437D012B03D1034B81751970F5E7D5
:10C89800704700BFE81A0020FC0000200D4B10B5BF
:10C8A800044618735873012000F016F85CB134215F
:10C8B8004FF4E86000F0C4FF4421BDE8104040F2A6
:10C8C800417000F0BDBF14214FF4E86000F0B8FFDC
:10C8D8002421F2E7E81A002038B5114C05462070EB
:10C8E80001F061FD052D04D8DFE805F0090B0317F9
:10C8F8001709032001F070FA0023637338BD002084
:10C90800F8E7012001F068FA207B637B8342F5D0C9
:10C918006073BDE83840FFF7C1BF0220EAE700BFF7
:10C92800E81A00202DE9F0431E4687B0002305468B
:10C93800CDE901330C46174601F027FD032D61D8D8
:10C94800DFE815F07B00C3000E010400A27C082A72
:10C9580004D94FF0FF3007B0BDE8F083A16801A803
:10C9680001F0DCFE21680029F3D042F210729142F6
:10C97800E37C864D51D80322AA7385F83820E963F1
:10C9880085F844304FF002086368A17DDB002B82F4
:10C998000423AB74A37CDB00EB7402294FF0000383
:10C9A8002B75637D02D0227D022A42D103F10F024A
:10C9B800D2B2012A01D9012BCBD1754B754A19681E
:10C9C80003944FF0010903A88DF8149001F0DAFCE4
:10C9D8000028BED1287685F817906875FFF75CFEA9
:10C9E8004046FFF779FF6C4801F086FA6B4801F082
:10C9F800EFFA01A800F084FF208A00F055FFA08913
:10CA080000F09AFF384601F001FC604C84F85600AB
:10CA180001F0C0FC666000209DE74FF00008E96364
:10CA2800890885F80E8085F8388085F844302964AF
:10CA3800AAE7EB7529766A75D0E72368002B88D0BA
:10CA4800A27C082A85D8514DA16801A801F066FE8C
:10CA5800002385F838302268EA63E27C85F84420B0
:10CA6800A269AB732A646268A17DD2002A8204227B
:10CA7800AA74A27C2B75D2000229637DEA7402D0C5
:10CA8800227D022A1DD103F10F02D2B2012A02D956
:10CA9800012B7FF45EAF3E4B3E4A196803944FF07A
:10CAA800010803A88DF8148001F06CFC00287FF4BD
:10CAB80050AF287685F817806875FFF7EDFD0020E0
:10CAC8008FE7EB7529766A75F7E7304D012185F810
:10CAD8003810227885F85020637885F85130A3788B
:10CAE80085F85230E3788B4202D0022B03D03BB951
:10CAF80085F8533004E00B3A012A29D885F85310F9
:10CB08004FF0010885F80E80A388AB83A379AB7733
:10CB1800E37985F82030237A85F82130FFF7BCFDCA
:10CB28004046FFF7D9FE1C4801F0E6F91B4801F022
:10CB38004FFA95F85130062B40F689000AD100F0DB
:10CB48008FFE00F0FB0140F6890000F079FE59E7FE
:10CB58000023CDE700F084FE40F00401C9B2F2E7FB
:10CB68002368013BB3F57A7FBFF4F3AE0320FFF7E8
:10CB7800B3FE0648022380F83830236883641623FE
:10CB880080F84C30383001F0B7F93BE7E81A00205C
:10CB9800CC1A0020441B0020201B0020F61A00207D
:10CBA8002DE9F041002686B01F461446CDE90166FE
:10CBB80080460D4601F0E9FBB442764C16BF0123CE
:10CBC800334637466370B8F1000F06D0B8F1010F4D
:10CBD8007CD0002006B0BDE8F081AB68002B00F0E7
:10CBE800D680EB68002B00F0D280AA7F082A00F2DA
:10CBF800CE80296901A801F091FD2868003818BF86
:10CC0800012000F0D9FF84F83880AB68E36395F819
:10CC1800203084F84430686801F05AFB84F80E80AC
:10CC280084F84500EB68DB002382EB7FA374AB7FBD
:10CC3800DB00E37495F82130237595F82230002B3A
:10CC48003ED12A7D95F82410A275022995F8232053
:10CC580001D0022B36D102F10F03DBB2012B02D92E
:10CC6800012A40F0948000238DF814304A4B4B4A37
:10CC78001968049503A801F085FB002840F0878017
:10CC880001232076E3756075FFF706FD0020FFF7A6
:10CC980023FE434801F030F9424801F099F901A810
:10CCA80000F02EFEA88B00F0FFFD288B00F044FE5C
:10CCB8004FF4FA53AA687B43B3FBF2F3A36088E707
:10CCC800FF22BFE7E27521766375DDE72B8E002B27
:10CCD8005DD095F83230A86A012B0CBF95F8148006
:10CCE8004FF0FF08003818BF012000F065FFF8B2C8
:10CCF80000F06EFF012184F8381095F82C2084F894
:10CD0800502095F82D3084F8513095F82E3084F85D
:10CD1800523095F82F308B4202D0022B03D03BB90A
:10CD280084F8533004E00B3A012A28D884F85310C9
:10CD38002B8EA38395F83230A377AB8E23840126FC
:10CD4800A67384F81F80FFF7A7FC3046FFF7C4FDE1
:10CD5800134801F0D1F8134801F03AF994F821305A
:10CD6800B34240F236700CD100F07AFD00F0FB01BE
:10CD780040F2367000F064FD4FF6FF739EE7002323
:10CD8800CEE700F06DFD40F00401C9B2F0E74FF0C6
:10CD9800FF301FE7E81A0020CC1A0020D01A002024
:10CDA800201B0020F61A00202DE9F04F85B082469E
:10CDB8000E9DBDF840B09DF844709DF848900192D2
:10CDC80088461E4601F0E1FABAF1010F524C54D0E0
:10CDD800BAF1040F00F09180BAF1000F3AD10B229A
:10CDE800304684F8442084F838A0E56301F070FAEE
:10CDF800019B23644FEACB03B9F1000F238241F66C
:10CE08000403638214BFF2230123E37587F001074B
:10CE18000123237684F8450084F80EA084F814A032
:10CE28006775FFF739FC5046FFF756FD04F13800E7
:10CE380001F062F804F10E0001F0CAF8374A1068F0
:10CE4800516802AB03C302A800F05AFD40F2FF107C
:10CE580000F02AFD404601F0D9F90E2184F8560069
:10CE680040F61F1000F0ECFC94F8560001F092FA1E
:10CE7800169B636005B0BDE8F08F294984F838A097
:10CE8800EAB2895D84F8502076BB0B3D012D8CBF3A
:10CE980000250125053A012A04D8BBF10C0F38BF3B
:10CEA8004FF00C0B1F4B9DF83C201B7884F8535017
:10CEB800E37701259DF8543084F8511084F8522006
:10CEC80084F82130A573A4F81CB0A77784F82090C3
:10CED800FFF7E2FB2846FFF7FFFC134801F00CF8C8
:10CEE800124801F075F8B5E7012E04D1A5F10C033D
:10CEF8005D425D41CEE70025CCE75046FFF7ECFCEC
:10CF0800022384F8383004F138001623A56484F825
:10CF18004C3000F0F1FF9DE7E81A002038F10008D6
:10CF2800F6F90008FC000020201B0020F61A00205B
:10CF38002DE9F04F87B0DFF8B4B29DF864A09DF8F2
:10CF48004C90029314469DF854309DF85020BDF83B
:10CF58004880039205468BF801A0BDF84460019310
:10CF68000F4601F012FABAF1000F18BF4FF000088F
:10CF7800DFF87CA2039AB9F1000F08BFFF22012D48
:10CF88008AF8002000F0C880052D48D0002D40F018
:10CF9800C080284600F010FE0B2238468BF844204B
:10CFA8008BF83850CBF83C4001F092F9019B8BF894
:10CFB800450041F60402002BABF812209AF8002035
:10CFC8008BF8162014BFF22201228BF81720F600E6
:10CFD800012289F001098BF818208BF80E50ABF864
:10CFE80010608BF814508BF81590FFF755FB284606
:10CFF800FFF772FC0BF1380000F07EFF0BF10E001A
:10D0080000F0E6FF7B490868496804AA03C204A83F
:10D0180000F076FC40F2FF1000F046FC71E00120C1
:10D0280000F0CAFD09224FF000098BF84420384669
:10D038004FF44872CBF840208BF83890CBF83C403E
:10D0480001F046F94FF48052ABF812209AF800200C
:10D058008BF845008BF8162028460122F6008BF83D
:10D0680017208BF80E90ABF81060ABF814908BF883
:10D078001890FFF731FC0BF1380000F03DFF0BF181
:10D088000E0000F0A5FF5B498868C96804AA03C2BE
:10D0980004A800F035FC40F2FF1000F005FC40F653
:10D0A800B80000F0DDFB00F0EF0140F6B80000F03A
:10D0B800C7FB042140F6B90000F0C2FB40F69B0014
:10D0C80000F0CEFB00F0E30141F0080140F69B00C0
:10D0D80000F0B6FB40F2D16000F0C2FB40F018014E
:10D0E800C9B240F2D16000F0ABFB40F2AC6000F096
:10D0F800B7FB00F08F0141F0500140F2AC6000F046
:10D108009FFB4FF4FA5202FB08F2B2FBF4F2CBF8A1
:10D11800082007B0BDE8F08F002000F04DFD36492B
:10D128008BF83850E2B2C95D8BF85020002F4DD1F2
:10D138000B3C012C8CBF00240124053A012A02D89B
:10D148000C2E38BF0C26029B9AF800208BF8523020
:10D158008BF85340019B8BF81F2001249DF8602019
:10D168008BF821208BF851108BF820308BF80E406B
:10D17800ABF81C608BF81E90FFF78EFA2046FFF77D
:10D18800ABFB1E4800F0B8FE1D4800F021FF5FFA17
:10D1980088F000F01DFD40F6A30000F061FB00EAF6
:10D1A800040140F6A30000F04BFB9BF82120A242AB
:10D1B80040F2367013D100F053FB00F0FB0140F24F
:10D1C800367000F03DFB4FF6FF72A0E7012F04D147
:10D1D800A4F10C035C425C41AFE70024ADE700F02A
:10D1E8003FFB40F00401C9B2E9E700BFE81A00209C
:10D1F800FC00002038F10008F6F90008201B002088
:10D20800F61A0020F0B58BB00D46044617461E46A8
:10D21800FFF742FA0020FFF75FFB204600F0BEFD53
:10D2280000240123CDE9084303234FF4167229464D
:10D238002046CDE90644CDE90444CDE90244CDE9D0
:10D2480000532346FFF774FE2046FFF77DFAFFF7E9
:10D2580035FAF4F759FB01F043FC0446204601F087
:10D2680049FCB04205D30124FFF716FA20460BB05B
:10D27800F0BD00F02FFF00B28742EFDA0024F3E799
:10D28800F7B500230C4640F201211A460646084627
:10D2980000F01EFD644B654D4FF400529A6195F8FD
:10D2A8005600012100F09CFF2B78012B40F68900E5
:10D2B80013D195F85130062B0FD100F0D1FA00F0B8
:10D2C800FB0140F6890000F0BBFA2B78042B6CD8E0
:10D2D800DFE803F0524B527F090000F0C1FA40F03A
:10D2E8000401C9B2EDE7524A731E1046C6F10107A0
:10D2F8004FF0000CF9188C426FDC0022E70013464F
:10D30800BA4271D19A0142EAC3125B0183F0200349
:10D318001343661C0355F6B202234648AB73AE7638
:10D3280000F056FE0021F12000F08AFA0021F020DA
:10D3380000F086FAAB6C642B70D17021F32000F0FA
:10D348007FFA1D21F22000F07BFAE1008C1CF4200A
:10D35800090A00F075FA04F0FE01F52000F070FAF1
:10D3680033486FF07F4231461DE0EC77314800F0DA
:10D378002FFE0022214615E001F008F80128074693
:10D3880025D121460DF10702304601F004F8044684
:10D39800A0B99DF807302748AB7500F019FE9DF835
:10D3A80007102246304600F065FB6968224801F004
:10D3B80063FC214801F026FC002006E01F4B3A469A
:10D3C8000021022001F0A2F8032003B0F0BDAC75E3
:10D3D800CCE70223AB73AC76C8E713F8011FC94347
:10D3E800197002F801CB85E7D1106FEA020C715C65
:10D3F8000CF0070C013241FA0CF101F001014FEA7F
:10D40800E20C4B40D14310F80CE001F0070103FA9D
:10D4180001F141EA0E0100F80C1071E7E121F32057
:10D4280000F00EFA04218DE700040048E81A0020F5
:10D43800CC190020F61A0020441B002098F9000897
:10D44800F0B5BDF814409DF818709DF81CE09DF8E3
:10D45800205040B1012814D0012200239818013827
:10D46800B0FBF2F0F0BD87F00107E30003EBC70360
:10D4780018330EEB450503EBC5034FF47A714B43A4
:10D48800ECE7501F012803F1040302D80C2C38BF25
:10D498000C24D1B9A2F10B0CBCF1010F8CBF4FF0D9
:10D4A800000C4FF0010C2801002F00EBCE0014BF38
:10D4B80000251425A0EB8200062A4FEA820628449C
:10D4C800A2F102070DD8354610E0012906D1A2F1D4
:10D4D8000C00D0F1000C4CEB000CE4E74FF0000C12
:10D4E800E1E70830BCF1000FEDD0BD000028ACBF6B
:10D4F8002E182E1C701E90FBF5F003FB0044094B00
:10D50800062A5A5C8CBF0C340E340A2A09D8A300A8
:10D5180001334FF47A71BB404B43034951F8222041
:10D528009CE7FFDEF6F90008FCF9000808B5094B8E
:10D53800012193F8560000F053FE4FF4D7602D21D7
:10D5480000F07EF900F033FBBDE80840024800F027
:10D558007BBA00BFE81A0020FFFF0F0073B5A44C88
:10D56800B4F854300025202B8DF80350019500F0B5
:10D578001B8114D8082B0DD87BB1013B072B0CD885
:10D58800DFE813F042005B000B00CD000B000B003E
:10D598000B00FD00102B00F0008102B070BDB3F548
:10D5A800807F00F0988011D8402B00F01081802BEC
:10D5B800F3D1284600F032FA8E4B1B68002BECD0D2
:10D5C8009B69002BE9D028469847E6E7B3F5007F2A
:10D5D800E3D1894B01222946022000F097FF00F091
:10D5E80029F9042840F08580844B85484FF400527F
:10D5F8009A6201F0B9FA284600F010FA7D4B1B68D0
:10D60800002BCAD05B6814E07C4B7D484FF4005275
:10D618009A6201F0A9FA002000F000FA00F0B8FEC2
:10D62800012801D100F0BDFE724B1B68002BB4D05D
:10D638001B68002BB1D09847AFE7704B71484FF487
:10D6480080529A6201F090FA657895B9284600F000
:10D65800E5F9294640F6021000F0F2F840F64410C9
:10D6680000F0FEF840F00201C9B240F6441000F0A4
:10D67800E7F8FF220DF1030163485E4D00F05AFD03
:10D68800624800F071FD2B68002B86D09E68002E42
:10D6980083D094F82430012B08D194F9313094F9CF
:10D6A80030209DF803105848B04776E7E06B01A991
:10D6B80000F022FE019B9DF8031053484FF47A7244
:10D6C80003F5FA7393FBF2F32A685BB2956894F951
:10D6D8002920A84761E7284600F0A0F9454B1B68B8
:10D6E800002B3FF45AAF9B69002B3FF456AF012043
:10D6F8006AE700F09FF805287FF44FAF3F4B414899
:10D708004FF480529A6201F02FFA284600F086F909
:10D71800384B1B68002B3FF440AFDB6889E70021DA
:10D728003B4B0122022000F0F1FEA16D00293FF4DD
:10D7380034AFC1F3074140F6031000F081F894F8C4
:10D74800591040F6041000F07BF894F8581040F691
:10D75800051000F075F840F6021000F081F840F06E
:10D768000101C9B240F6021000F06AF8002340F245
:10D7780062211A460846A36500F0AAFA0DE7254B70
:10D7880001220021022000F0C1FE00F0FFFD012867
:10D798007FF403AF00F006FEFFE61F4B01220021D5
:10D7A800022000F0B3FEF8E6164801F0DDF96078D3
:10D7B80008B900F033F90F4B1B68002B3FF4EDAEAE
:10D7C800DB68002B3FF4E9AE9847144BE6E7144BAF
:10D7D80001222946022000F099FE607808B900F07D
:10D7E8001DF9044B1B68002B3FF4D7AE1B6920E7DB
:10D7F800E81A0020CC1A0020ADF9000800040048FF
:10D80800441B0020D01A0020CC1900200C1B00203B
:10D81800C1F90008CAF90008D4F90008DDF90008C0
:10D82800E6F90008024BA3F85400FFF797BE00BFC3
:10D83800E81A0020014B1878704700BF621B0020CF
:10D8480007B501238DF807100DF1070201460348BB
:10D85800F7F774F803B05DF804FB00BFC4010020BB
:10D8680007B5012301460DF107020448F7F79FF8B1
:10D878009DF8070003B05DF804FB00BFC401002059
:10D8880010B50446F4F7B8FD01280CD140F6231072
:10D89800FFF7E6FF00F0F901214340F62310BDE849
:10D8A8001040FFF7CDBF10BD10B50C4B1B780446D8
:10D8B8009BB94FF4D760FFF7D3FFC4F3002100F002
:10D8C800FE0001434FF4D760FFF7BAFFE1B240F220
:10D8D800B960BDE81040FFF7B3BF10BD631B00205F
:10D8E80010B51346EFF3108472B60A460146034892
:10D8F800F7F724F884F3108810BD00BFC401002096
:10D9080008B5014608224FF4D860FFF7E9FF002068
:10D9180008BD000007B5074B1B7840BAADF80400F6
:10D928002BB9022201A940F2BC60FFF7D9FF03B06E
:10D938005DF804FB631B002007B5074B1B7840BA52
:10D94800ADF804002BB9022201A940F2BE60FFF72E
:10D95800C7FF03B05DF804FB631B002010B5134636
:10D96800EFF3108472B60A4601460348F7F71FF82A
:10D9780084F3108810BD00BFC401002010B5134601
:10D98800EFF3108472B60A4601460348F7F701F927
:10D9980084F3108810BD00BFC40100200A46014668
:10D9A8000020FFF7EBBF000010B51346EFF310841B
:10D9B80072B60A4601460348F7F71EF984F3108841
:10D9C80010BD00BFC401002010B51346EFF310844A
:10D9D80072B60A4601460348F7F724F884F310881C
:10D9E80010BD00BFC401002013B504460020F4F7A1
:10D9F800DDFC0220FFF744FF04F0070401220DF1CB
:10DA0800070184208DF80740FFF7DEFF024B002254
:10DA18001A7002B010BD00BF621B002007B50122BA
:10DA28008DF807000DF107018020FFF7CDFF9DF865
:10DA38000730002B034B0CBF012202221A7003B0DF
:10DA48005DF804FB621B002007B5094B8DF8060042
:10DA580004221A70030C8DF804300322030A01A96A
:10DA680083208DF80530FFF7AFFF03B05DF804FBA6
:10DA7800621B002010B51446FFF790FF2046BDE852
:10DA88001040FFF7E1BF000007B5094B8DF806000D
:10DA980005221A70030C8DF804300322030A01A929
:10DAA80082208DF80530FFF78FFF03B05DF804FB87
:10DAB800621B002073B5002640F6E2000196FFF7CE
:10DAC800CFFE00F0FE01054640F6E200FFF7B8FE83
:10DAD80040F6E500FFF7C4FE00F07F01044640F67B
:10DAE800E500FFF7ADFE6FF07F40FFF7CDFF0422A2
:10DAF8000DEB020140F61900FFF730FF3046FFF743
:10DB08008DFF294640F6E200FFF79AFE214640F6CF
:10DB1800E500FFF795FE019802B070BD13B50C4BF8
:10DB280004460522972140F6AC001A70FFF788FEDC
:10DB3800230C8DF804300322230A01A982208DF8D2
:10DB480005308DF80640FFF73FFF02B010BD00BF5B
:10DB5800621B002007B5030C8DF80030030A8DF80E
:10DB680001300B0C49BA8DF80200ADF804100622FA
:10DB7800694694208DF80330FFF726FF024B0622F2
:10DB88001A7003B05DF804FB621B0020002208B580
:10DB98001146C520FFF718FF014B07221A7008BD70
:10DBA800621B002000221146D120FFF70DBF002282
:10DBB8001146D220FFF708BF07B501228DF80700EC
:10DBC8000DF107019F20FFF7FFFE03B05DF804FB8E
:10DBD80007B501228DF807000DF10701A020FFF716
:10DBE800F3FE9DF807103F2907D901F0F80101312C
:10DBF800C9B240F20670FFF723FE03B05DF804FBDC
:10DC080007B5F4F7F9FB431E584258418DF8070051
:10DC180001220DF107019620FFF7D6FE03B05DF84B
:10DC280004FB07B500F07F008DF8070001220DF115
:10DC380007018920FFF7C8FE03B05DF804FB000068
:10DC4800154B984207B51BD8144B98421BD8144B58
:10DC580098421BD8134B98421BD8134B984295BF38
:10DC680029226B222B236F238DF8042001A902227D
:10DC780098208DF80530FFF7A7FE03B05DF804FB88
:10DC8800E122E923F0E7D722DB23EDE7C122C52310
:10DC9800EAE775228123E7E700E9A43580F8A9328D
:10DCA8008044E52D000B6B1B40FC541907B58DF81B
:10DCB800062004228DF804008DF8051095200DEB40
:10DCC80002018DF80730FFF77FFE03B05DF804FB13
:10DCD80007B552BAADF8042040BA082249BAADF8DF
:10DCE8000000ADF802105BBA69461046ADF8063080
:10DCF800FFF76AFE03B05DF804FB07B50B0C0422BE
:10DD080000F0070049BA8DF80400ADF80610972016
:10DD18000DEB02018DF80530FFF756FE03B05DF8F4
:10DD280004FB000010B508B1194B1860F3F7F0FCBC
:10DD38000220FFF7A5FD0024164B20461C70FFF7B4
:10DD48006DFEF4F757FB012817D14FF42071FFF748
:10DD5800D4FF40F611102146FFF772FD4FF07F0007
:10DD6800FFF75FFF0E2140F61F10FFF769FDF4F77C
:10DD7800E9FA094B01221A7010BD102140F6111062
:10DD8800FFF75EFD102140F61210FFF759FDE9E795
:10DD9800641B0020601B0020621B002037B50C4D5F
:10DDA8002B7804461BB9FFF74BFF01232B70002388
:10DDB800084A6006E109F2F7F3FE042200BA01906E
:10DDC8000DEB02018620FFF7FFFD03B030BD00BF59
:10DDD800601B00200048E80107B5094B8DF80700D3
:10DDE8000146187018B940F2AC60FFF729FD01220E
:10DDF8000DF107018A20FFF7E7FD03B05DF804FB8A
:10DE0800631B0020012873B50C46164637D1002045
:10DE1800F4F7F4FAA042B8BF44B20E2805461AD166
:10DE280001231A4600210420FFF740FF6FF010037A
:10DE38009C42B8BF1C46182140F6E700FFF700FDDA
:10DE4800022201A98E208DF804408DF80560FFF7A5
:10DE5800BBFD02B070BD01230A28E4B21A464FF098
:10DE6800000105D11846FFF721FF033464B2DDE74E
:10DE78000720C5F10E05FFF719FF2C44F6E740F619
:10DE8800D800FFF7EDFC40F01E01C9B240F6D800FB
:10DE9800FFF7D6FC0120F4F7B1FAA042B8BF44B2AC
:10DEA800142805464FF001034FF000020CD105215C
:10DEB8000320FFF7FBFE023464B26FF008039C42B4
:10DEC800B8BF1C463821B7E7112805D10321022025
:10DED800FFF7ECFE0534EFE70E2804D102210846CF
:10DEE800FFF7E4FEE9E7C5F11605072104202544FC
:10DEF800FFF7DCFE6CB2E0E713B5314A044651681F
:10DF080010686B4603C32F4B20781B78834201D0DF
:10DF1800FFF762FF2378032B27D8DFE803F00239E5
:10DF2800283C6268284BB3FBF2F31A0CA1688DF801
:10DF380000208DF802301A0A237B8DF80330637BAA
:10DF48008DF801208DF80430204A00234806C909BD
:10DF5800F2F726FE030C40BA8DF80530ADF806003E
:10DF6800082269468B20FFF72FFD02B010BD2269F9
:10DF7800154BB3FBF2F31A0C8DF800208DF8023024
:10DF88001A0A237D8DF801208DF803300422E8E772
:10DF9800A3690093FAE762680B4BB3FBF2F31A0C20
:10DFA8008DF800208DF802301A0A237B8DF8033093
:10DFB800637B8DF801208DF804300522D1E700BF7E
:10DFC80048F10008631B00200000093D0048E801F3
:10DFD8001FB52E4A0446D1689068127C01AB03C372
:10DFE8001A702B4B20781B78834201D0FFF7F4FE80
:10DFF8002378032B26D8DFE803F002383302637A4C
:10E00800F12B21D14FF6FF70FFF784FC48F2050091
:10E01800FFF792FC02236288A188ADF8061052BA75
:10E02800E188ADF804208DF80B30227AA37A8DF8B8
:10E038000A20ADF808108DF80C30092201A98C20AF
:10E04800FFF7C2FC04B010BDF22BE4D141F60F502B
:10E05800FFF760FC41F22100FFF76EFC0623DAE7C8
:10E06800237B8DF804300122E8E7E389094A5BBA8B
:10E07800ADF80430237C13708DF80630637C8DF87E
:10E088000730638AADF808300622D7E748F1000860
:10E09800631B0020611B002007B502228DF80400D5
:10E0A8008DF805108F2001A9FFF78EFC03B05DF8ED
:10E0B80004FB000010B51346EFF3108472B60A464D
:10E0C80001460348F6F7E6FC84F3108810BD00BF4C
:10E0D800C401002007B5012201A91520FFF7EAFFB6
:10E0E8009DF804004042401003B05DF804FB0000B6
:10E0F80037B505460C46022201A91320FFF7DAFFBF
:10E108000A4B1B78012B0DD1094B1B78012B09D128
:10E1180040F20270FFF7A4FB9DF8053028702370C9
:10E1280003B030BD9DF80400F6E700BF631B002074
:10E13800611B0020F7B50D46064600240DF10701C6
:10E14800284617468DF80740FFF7D2FF2A78BA42CB
:10E1580007D89DF807003146FFF726FC204603B094
:10E16800F0BD0120FBE7000013B50322044601A916
:10E178001420FFF79FFF184B1A7822704AB1012A22
:10E1880017D014220021204600F0D2FA0F23237062
:10E198000DE09DF8043023719DF80530A2605B42C4
:10E1A8005B10A3719DF806305B425B10637102B08F
:10E1B80010BD9DF804305B425B1023739DF9053058
:10E1C80002339B1063739DF806305B425B10A373A8
:10E1D800024B1B682361EAE7631B00205C1B0020DD
:10E1E800012908B5034608460ED1012B07D10420A2
:10E1F800FFF746FB0220BDE80840F4F7D7B8022B2A
:10E2080014BF08460320F6E70120F4E738B50446B2
:10E21800F4F7EEF850B1022814BF0125022528466C
:10E2280002222146FFF7EEFD284638BD0F2CCCBF51
:10E2380002250125F3E70A2070470000014B012061
:10E248001B681847641B0020014B02201B681847F5
:10E25800641B0020014B40201B681847641B0020EA
:10E2680011B1012904D07047044B1B68802018475E
:10E27800024B4FF480701B68F9E700BF641B002055
:10E28800024B4FF400701B68184700BF641B002046
:10E29800014B20201B681847641B0020014B0420F9
:10E2A8001B681847641B0020014B08201B6818478F
:10E2B800641B0020014B10201B681847641B0020BA
:10E2C800024B4FF480401B68184700BF641B0020B6
:10E2D80068B1084A002352F83310814203D902EB8F
:10E2E800C302107970470133162BF4D1FEE71F20C3
:10E2F800704700BFB8FA000873B51D4B0193044678
:10E3080040F607000D46FFF7ABFAC0F3C103083328
:10E318006B4413F8042C00F00703013302FA03F3EB
:10E32800144AB2FBF3F2B2FBF4F007281ED84000FF
:10E3380003288CBF022304234FF4D66002FB03F4A6
:10E34800FFF78EFA060240F2B160FFF789FA06F489
:10E3580070663043030544BF6FEA00506FEA1050FF
:10E3680063094343DB112B6002B070BD0123E3E76F
:10E3780004080A0C0048E8014FF0FF3070474FF0DE
:10E38800FF3070474FF0FF307047704700207047EC
:10E398000020704770474FF0FF3070474FF0FF3054
:10E3A800704770477047704770B5EFF3108672B6C4
:10E3B800144B5C8A1A8A944213D1C4F5806292B2D3
:10E3C800904206D3844218D901229A7000221C80F8
:10E3D8005A825A8A0A800244C2F309025A820020E9
:10E3E8000DE006D9C4F58065ADB28542F1D8824208
:10E3F800E9E7121B92B28242EBD84FF0FF3086F366
:10E40800108870BD681F0020EFF3108172B6034AB0
:10E41800D38A0133D38281F310887047681F0020A4
:10E42800EFF3108172B6034AD38A013BD38281F39A
:10E4380010887047681F002010B50848182200216E
:10E4480000F076F906484FF48062002100F070F978
:10E45800044B05481B68BDE810401847681F00209A
:10E46800681B0020C0F10008E1E50008014B586076
:10E47800704700BF681F0020014B1872704700BF2B
:10E48800681F002073B5EFF3108572B61C4CE08A44
:10E4980000282FD1FFF7B8FF218A628A914227D03E
:10E4A800A378012B12D1238820805B1A9BB202210A
:10E4B800A382A17063B9A3702382238A9A428BBF77
:10E4C800D21AC3F58063A282A38201E0002BF4D0A4
:10E4D800238A0C4E1E4485F31088F3F703FA0A4B7F
:10E4E800A18ADB680193304602B0BDE87040184746
:10E4F800FFF796FF85F31088002002B070BD00BFBB
:10E50800681F0020681B0020C0F1000808B4F0B59F
:10E5180086B00023ADF800302C4B0B9C1D7A854249
:10E528004DD3D86881434DD15B681BB112B16946A0
:10E5380002A898470CAB22464FF400712448019377
:10E5480000F0F6FBFFF760FFBDF8003018440DF14E
:10E55800020180B2FFF728FF01302BD00022BDF85E
:10E568000030BDF802701B480DF1080C164691B238
:10E5780017FA82F58B42ADB216D83B449BB20EB166
:10E58800ADF80230BDF80250019B22464FF40071ED
:10E59800284400F0CDFBFFF743FFFFF773FF06B0F9
:10E5A800BDE8F04001B070471CF8011B415501322D
:10E5B8000126DCE7FFF734FF6FF00200EFE76FF0AA
:10E5C8000400ECE76FF00500E9E700BF681F0020D2
:10E5D800801F0020681B002013B5EFF3108472B66B
:10E5E800204B9A78588A022A1DBF1A8A998A52188B
:10E5F800002214BFC2F309029A7090421A8228D0EE
:10E60800D98A012925D19978012913D119888A1A1B
:10E61800022192B2997000219A82198062B99A7087
:10E628001A821A8A90428BBF801AC2F58062988239
:10E638009A8201E00029F4D01A8A0B48104484F326
:10E6480010880A4A998AD368019302B0BDE810403D
:10E65800184784F31088F3F749F902B0BDE8104071
:10E66800FFF7DEBE681F0020681B0020C0F100080D
:10E67800024A00231360024A136070478421002075
:10E688008021002010B5EFF3108472B641B1012942
:10E6980003D1064A13680343136084F3108810BD3E
:10E6A800024A136823EA0003F6E700BF842100202A
:10E6B80010B5EFF3108472B641B1012903D1064AAF
:10E6C80013680343136084F3108810BD024A13686B
:10E6D80023EA0003F6E700BF8021002038B5EFF3F6
:10E6E800108572B60A4B0B4C1B6833B123689847E8
:10E6F8006368984785F3108838BD074B1B681BB1C2
:10E70800A3689847E368F4E7236998476369F0E7E3
:10E71800842100205CF100088021002001380A448F
:10E72800914200D1704711F8013B00F8013FF7E72B
:10E7380000F01CBC10B5EFF3108472B6064A1368DB
:10E7480003431360054A52F83130034342F831302D
:10E7580084F3108810BD00BFAC210020A421002044
:10E7680070477047030C1B04C3B90004102310F052
:10E778007F4F02BF08330002DBB210F0704F08BFB2
:10E7880000014FEA1070064A08BF0433125C08BF44
:10E79800DBB2C3F11F03981AC0B270470023E6E743
:10E7A80068FB00082DE9F84F384D394ED5F8008040
:10E7B800DFF8E0B0DFF8E0A0DFF8E090D6F800C0BE
:10E7C800374FDBF80010374CDAF80020D9F8003062
:10E7D80008EA00002860286800EA020E1EEA0C0F0A
:10E7E80001D019421ED04FF0FF333B60FFF7B8FF4E
:10E7F800EFF3108472B63368DBF80020DAF8001003
:10E808000B4029680B4205D1D9F80030134201D1D9
:10E81800F2F7F6FF84F31088FFF7A3FFC5F800802E
:10E82800BDE8F88F236823680340134062681A42E2
:10E8380004BF4FF0FF32626060681840FFF792FF34
:10E8480062683860012303FA00F022EA000262607D
:10E85800EFF3108172B63A689340326822EA0302F5
:10E868003260226822EA0303236081F310880E4A8B
:10E878003B6852F823309847D6F800C0DBF8001000
:10E88800DAF80020D9F80030A5E700BF0001002021
:10E89800AC2100208C2100200401002090210020C0
:10E8A80088210020A42100209421002010B51146C1
:10E8B800EFF3108472B6FFF755FF034B43F82010AF
:10E8C80084F3108810BD00BF9421002082B082B06C
:10E8D8000DF1080C0CE90600BDF8042003930B4465
:10E8E800BDF810100A4491B212B2B2F57A7FA2BFF5
:10E8F800A1F57A72013312B20360828002B002B0CD
:10E90800704782B082B00DF1080C0CE90600BDF822
:10E9180004200393CB1ABDF81010521A91B212B208
:10E92800002ABEBF01F57A7203F1FF3312B2036009
:10E93800828002B002B0704730B585B0114D6B4689
:10E9480083E8030000230293ADF80C3003A82B6979
:10E958009847009BBDF804400290181ABDF80C3087
:10E96800E41AA3B224B2002CBEBF03F57A731CB21A
:10E9780000F1FF302B689847AB682046984705B0F0
:10E9880030BD00BF80F1000873B5114E0023054665
:10E998000093ADF8043001A833699847F3680090F4
:10E9A8009847736804469847009B1844BDF804309C
:10E9B80023449AB21BB2B3F57A7FA2BF0130A2F505
:10E9C8007A731BB228602846AB8002B070BD00BFC6
:10E9D80080F1000837B500230093ADF80430074BE9
:10E9E80004461B6901A898476D46009095E8030006
:10E9F80084E80300204603B030BD00BF80F1000862
:10EA080037B50F4D02AB03E90300EB6898476B6815
:10EA180004469847BDF80430009A1B1B99B21BB2F4
:10EA2800002BA2EB0002BEBF01F57A7102F1FF32A2
:10EA38000BB24FF47A7000FB023003B030BD00BF58
:10EA480080F100082DE9F0414FF47A75B1FBF5F536
:10EA5800C5EB4513DFF83C8005EB8303A1EBC3034B
:10EA68009CB2D8F80C3006469847D8F804300746C8
:10EA78009847E31999B21BB2B3F57A7F2844A2BF2D
:10EA8800A1F57A7301301BB23060B3803046BDE81F
:10EA9800F08100BF80F10008024B00221A60024B8F
:10EAA8001B681847B021002094F10008F8B5044607
:10EAB800174608461E467CB173B1084B00255B6AB1
:10EAC80025609847069B60602581A572E6602361F2
:10EAD800E77265612846F8BD0120FCE794F100085B
:10EAE80010B5034CE3699847A36ABDE8104018477E
:10EAF80094F1000870B5064DEB69064698476B6AB5
:10EB0800044630469847AB6A201ABDE8704018475B
:10EB180094F10008054B1B680BB9184670478342EF
:10EB280001D05B69F8E70120704700BFB0210020E1
:10EB38002DE9F3410B4E336A044698470123B76920
:10EB48002372D4F800800546B8472844804502D28D
:10EB5800B84728442060B3682068019302B0BDE834
:10EB6800F041184794F1000870B520B3EFF3108610
:10EB780072B6124D2B680122827253B10022427282
:10EB880098425C690ED102723CB120462C60FFF7B6
:10EB9800CFFF86F31088002070BD094BDB689847CB
:10EBA8002C60F6E71A465B69002BF2D09842F9D13F
:10EBB80043695361EDE70120EEE700BFB021002073
:10EBC80094F10008084B10B51A685369516911B9D6
:10EBD8005061416110BD046819688C4202D91A4617
:10EBE8005B69F3E71946F3E7B0210020044A13688C
:10EBF8000BB10021197243611060FFF799BF00BF84
:10EC0800B02100202DE9F041044600282DD0FFF75F
:10EC180081FF50BB657A45BBEFF3108872B6144E7E
:10EC28006768336A984787422CBF27602060114F76
:10EC3800A5724FF4807323813B684BB933699847B9
:10EC48002046FFF7D3FF88F310882846BDE8F081F7
:10EC5800B3699847236818443B6820601B6898424A
:10EC68002046EED3FFF7AEFFEDE70125EDE700BF45
:10EC780094F10008B021002010B5044608467CB184
:10EC8800084B5B6A984760602046FFF743FF40B136
:10EC98002046FFF769FF2046BDE81040FFF7B2BFE6
:10ECA800012010BD94F100082DE9F041EFF3108721
:10ECB80072B61D4E1D4D73699847336904469847CF
:10ECC8002B684BB94FF000082B688BB9286828BB14
:10ECD80087F31088BDE8F081011B241A1A688A425C
:10ECE8008CBF121900221A605B69002BF6D1E9E784
:10ECF8001C681CB1B36998478442E7D22C686369E1
:10ED08002B60A4F80880D4E9033098476389B3F5E9
:10ED1800807FD9D12046FFF775FFD5E7037A002B0E
:10ED2800D6D1FFF705FFD3E794F10008B021002002
:10ED38002DE9F04F97B000298046039140F30E81EA
:10ED48009A46044603991378A4EB0800013923B9BD
:10ED58000023237017B0BDE8F08F8842F8DA252B1E
:10ED680004D004F8013B1646721CEBE792F801C088
:10ED7800ACF13003D3F1000E4EEB030EACF13003CF
:10ED8800092B02F1010629D8324600254FF00A095D
:10ED9800164612F8013BA3F13000092819D9337837
:10EDA800692B00F09C801CD8632B28D0642B00F0C2
:10EDB8009680582B5BD0252B19D13378002B00F087
:10EDC800928004F8013BA4EB08038B4280F289800F
:10EDD800CAE709FB0533A3F13005D9E74FF0FF3542
:10EDE800DDE7752B7DD0782B43D0732B1ED02523E0
:10EDF80004F8013BA4EB08038B4272DADDE7002D2F
:10EE080005F1FF39D8BF4FF000094A4620462021B6
:10EE180000F0ACF85346A144002D53F8042B89F8B0
:10EE28000020D8BF01252C449A469DE74C4B5AF840
:10EE3800047B002F08BF1F463846F1F799F9A5EB68
:10EE4800000B8542B8BF4FF0000B5A46814620217F
:10EE5800204600F08BF8A34400234B4502DB0BEB64
:10EE6800090481E7FA5C0BF803200133F5E74EF05B
:10EE7800400E1020DFF8EC903B4F1EF0400F08BF0B
:10EE88004F465346BCF1300F0197A4EB08020CBF64
:10EE9800302720271EF0020FA1EB0202029753F839
:10EEA800041B22D0002920DA4942013D4FF02D0EE3
:10EEB80005AF009700278946DDF804A0B1FBF0F103
:10EEC80000FB119B48451AF80BB0DDF800A00AF8C2
:10EED80001BB07F10107CDF800A0ECD90EE04EF018
:10EEE800020E0A20C6E7013E6DE711B14FF0000E91
:10EEF800DEE730208DF814008E460127BCF1300F74
:10EF0800A5EB070504D02020002D05F1FF3509DC0D
:10EF1800BEF1000F04D02D21013A04F8011B83D063
:10EF280025440AE0013A04F8010BEDD17CE7029987
:10EF380004F8011B013A3FF477AF291B0029F6DCDE
:10EF480005A9394422442744A7423FF46DAF11F87C
:10EF5800010D04F8010B9442F6D165E70020F9E6AB
:10EF680078FB00087FFB0008A4FB00080244034666
:10EF7800934200D1704703F8011BF9E770B50D4DB6
:10EF88000D4C641BA4100026A64209D10B4D0C4C55
:10EF980000F09AF8641BA4100026A64205D170BDA3
:10EFA80055F8043B98470136EEE755F8043B984777
:10EFB8000136F2E7ACFC0008ACFC0008ACFC000829
:10EFC800B0FC000800000000C1F30A522DE9F84324
:10EFD800A2F2FF36132E0B4607460C46054632DCD6
:10EFE800002E14DA34A3D3E90023F1F7CFF8002276
:10EFF8000023F1F7FFFA38B1002C56DA24F0004468
:10F00800254355D02E4C002523462F4625E02D4A72
:10F0180042FA06F801EA080202431ED026A3D3E901
:10F028000023F1F7B3F800220023F1F7E3FA0028F0
:10F03800EAD0002CBEBF4FF480133341E41824EA11
:10F0480008040025E0E7332E0BDDB6F5806F04D108
:10F058000246F1F79BF807460B4638461946BDE8C5
:10F06800F883A2F213424FF0FF3828FA02F810EAA8
:10F07800080FF2D010A3D3E90023F1F787F8002294
:10F088000023F1F7B7FA0028BED0002C0ADA142EB4
:10F0980001D1013406E0C6F134060123B3401D4412
:10F0A800AF42F6D825EA0805AEE700252C46ABE7BF
:10F0B8004FF00044A8E700BF9C7500883CE4377E09
:10F0C8000000F0BFFFFF0F00F8B500BFF8BC08BC98
:10F0D8009E467047F8B500BFF8BC08BC9E4670470E
:10F0E8000000000001000000020000000000000015
:10F0F8008813000010270000204E00003075000023
:10F10800409C000050C3000060EA0000C0D4010029
:10F1180080A903000053070000EA0637000000003A
:10F128005000000040F709370000000050000000C0
:10F13800C194C10000000000B227000000000000D8
:10F1480000000000000000000000000000000000B7
:10F158000000000099160008AB16000849160008C0
:10F16800AF1600082D1600084516000825647325FB
:10F178003033643A00000000FD1900089D1A0008A9
:10F188000D1A0008A91A00086D1A0008B51A000817
:10F19800000000001D1A0008D5190008A119000870
:10F1A80059190008B1190008C5190008651900089F
:10F1B800691900087D190008251D00084D1D000863
:10F1C800D11C0008BD1C000801000000030000005D
:10F1D800050000000100000001000000060000001A
:10F1E8000A000000200000000200000004000000E7
:10F1F800080000001000000040000000800000002F
:10F2080000010000000200000000000000000000F3
:10F2180000000000000000000100000002000000E3
:10F228000300000004000000A0860100400D030058
:10F23800801A060000350C0040420F0080841E0032
:10F2480000093D0000127A000024F40000366E0127
:10F258000048E801006CDC0200000000000000002B
:10F268000000000000000000040208001010100454
:10F27800101010021010100801000200040006000F
:10F2880008000A000C001000200040008000000167
:10F29800080402040801010101010103070100003B
:10F2A8006572726F723A20526567696F6E20697372
:10F2B800206E6F7420646566696E656420696E20CF
:10F2C800746865204D573A20736574206C6F7261BD
:10F2D80077616E5F636F6E662E68206163636F721D
:10F2E80064696E676C790D0A004D41432072785449
:10F2F800696D654F75740D0A004D4143207478544B
:10F30800696D654F75740D0A004D4143207278444C
:10F318006F6E650D0A004D4143207478446F6E6529
:10F328000D0A00080A0C0D0E10121415181A1B1DD0
:10F338001E2124030502050106020205000006003D
:10F34800000105040400000048E8010048E8010045
:10F3580048E8010048E8010048E8010048E80100E1
:10F3680090D0030000000000030000000201000C20
:10F378000B0A09080707320000000000000102011B
:10F388000000000000020302010000000003040363
:10F39800020100000004050403020100000506053F
:10F3A8000403020100060706050403020107070714
:10F3B8000605040302070702020202020202020211
:10F3C8000202020202020302020202020203040310
:10F3D80002020202020405040302020202050605F3
:10F3E80004030202020607060504030202070707D0
:10F3F8000605040302070733337373F2F2F2F200CF
:10F40800000B357DF2F2F233337373DEDEDEDE524B
:10F41800585F2573206F6E20667265712025642001
:10F42800487A2061742044522025640D0A005258FD
:10F43800206F6E206672657120256420487A2061ED
:10F44800742044522025640D0A005458206F6E2001
:10F458006672657120256420487A206174204452C0
:10F468002025640D0A00310032004D756C74695F07
:10F4780043004D756C74695F500000006EF400081D
:10F4880070F4000878F4000872F4000880F40008AA
:10F498007AF40008C6F8EEF6FFD6DE916002CE5682
:10F4A800E7B54DEC8F1F89FAEFB28EFB41B35F458C
:10F4B8002353E49B75E13D4C6C7EF5836851D1F98B
:10F4C800E2AB622A0895469D30370A2F0E241BDFCF
:10F4D800CD4E7FEA121D583436DCB45BA476B77D76
:10F4E80052DD5E13A6B900C140E379B6D48D6772C8
:10F4F8009498B085BBC54FED869A66118AE904FEDB
:10F50800A078254BA25D80053F2170F16377AF425B
:10F5180020E5FDBF811826C3BE35882E9355FC7A99
:10F52800C8BA32E6C0199EA344543B0B8CC76B285B
:10F53800A7BC16ADDB647414920C48B89FBD43C4D5
:10F548003931D3F2D58B6EDA01B19C49D8ACF3CFFF
:10F55800CAF447106FF04A5C38577397CBA1E83E5E
:10F5680096610D0FE07C71CC9006F71CC26AAE69FB
:10F5780017993A27D9EB2B22D2A907332D3C15C965
:10F5880087AA50A50359091A65D784D082295A1E1B
:10F598007BA86D2CA584998D0DBDB1545003A97D10
:10F5A8001962E69A459D408715EBC90BEC67FDEAA1
:10F5B800BFF7965BC21CAE6A5A41024F5CF434082E
:10F5C8009373533F0C52655E28A10FB509369B3DD6
:10F5D8002669CD9F1B9E742E2DB2EEFBF64D61CE93
:10F5E8007B3E7197F568002C601FC8EDBE46D94B6D
:10F5F800DED4E84A6B2AE516C5D75594CF100681A4
:10F60800F044BAE3F3FEC08AADBC4804DFC17563B9
:10F61800301A0E6D4C14352FE1A2CC3957F28247BF
:10F62800ACE72B95A098D17F667EAB83CA29D33CE3
:10F6380079E21D763B564E1EDB0A6CE45D6EEFA642
:10F64800A8A4378B324359B78C64D2E0B4FA0725A3
:10F65800AF8EE918D5886F7224F1C751237C9C219D
:10F66800DDDC86859042C4AAD8050112A35FF9D0D3
:10F67800915827B93813B333BB7089A7B6229220A3
:10F6880049FF787A8FF88017DA31C6B8C3B0771196
:10F69800CBFCD63A637C777BF26B6FC53001672B66
:10F6A800FED7AB76CA82C97DFA5947F0ADD4A2AF6E
:10F6B8009CA472C0B7FD9326363FF7CC34A5E5F17C
:10F6C80071D8311504C723C31896059A071280E22A
:10F6D800EB27B27509832C1A1B6E5AA0523BD6B37E
:10F6E80029E32F8453D100ED20FCB15B6ACBBE39EE
:10F6F8004A4C58CFD0EFAAFB434D338545F9027FDA
:10F70800503C9FA851A3408F929D38F5BCB6DA2192
:10F7180010FFF3D2CD0C13EC5F974417C4A77E3DBE
:10F72800645D197360814FDC222A908846EEB81414
:10F73800DE5E0BDBE0323A0A4906245CC2D3AC62D7
:10F748009195E479E7C8376D8DD54EA96C56F4EAE2
:10F75800657AAE08BA78252E1CA6B4C6E8DD741FF3
:10F768004BBD8B8A703EB5664803F60E613557B9B6
:10F7780086C11D9EE1F8981169D98E949B1E87E970
:10F78800CE5528DF8CA1890DBFE6426841992D0F1F
:10F79800B054BB162323232323232025732025308D
:10F7A80032583A253032583A253032583A253032D4
:10F7B800583A253032583A253032583A253032589E
:10F7C8003A253032583A253032583A253032583AAC
:10F7D800253032583A253032583A253032583A25B1
:10F7E8003032583A253032583A253032580D0A000E
:10F7F800232323232323204465764555493A202093
:10F8080020202020253032583A253032583A2530E9
:10F8180032583A253032583A253032583A25303263
:10F82800583A253032583A253032580D0A002323E9
:10F8380023232323204170704555493A2020202056
:10F848002020253032583A253032583A253032585F
:10F858003A253032583A253032583A253032583A1B
:10F86800253032583A253032580D0A0023232323F5
:10F87800232320446576416464723A2020202020A6
:10F88800253032583A253032583A253032583A2500
:10F898003032580D0A004170704B65793A202020AB
:10F8A8002020004E776B4B65793A202020202000DD
:10F8B8004E776B534B65793A2020202000417070B9
:10F8C800534B65793A20202020004442496E744BFE
:10F8D80065793A202020004D43526F6F744B65794B
:10F8E8003A2020004D434B454B65793A2020202093
:10F8F800004D43417070534B65795F303A004D437A
:10F908004E776B534B65795F303A0000000000007A
:10F918004150505F9EF80008010000004E574B5FB1
:10F92800ABF80008080000004E574B53B8F8000821
:10F938000900000041505053C5F800080A000000B3
:10F948004442495FD2F800080B0000004D4352546E
:10F95800DFF800080C0000004D434B45ECF80008A8
:10F968000D0000004D434B30F9F800080E00000070
:10F978004D415330F9F800080F0000004D4E533048
:10F9880006F90008100000005A45524FD3F9000844
:10F99800526164696F53656E64204F76657273694E
:10F9A8007A650D0A004952515F52585F54585F54A6
:10F9B800494D454F55540D0A00505245204F4B0DA7
:10F9C8000A0053594E43204F4B0D0A004844522019
:10F9D8004F4B0D0A00484452204B4F0D0A00495224
:10F9E800515F4352435F4552524F520D0A0004057E
:10F9F80006000000841E0000093D0000127A000085
:10FA080024F4000048E8010090D0030020A107007A
:10FA180000000000B128000061510000C3A20000EE
:10FA280002010003E5C70008A9C60008E1C80008EC
:10FA380025C700080DD20008CDC7000839CF000837
:10FA4800B1CD000889C5000849D4000889D200084A
:10FA5800B9C70008A1C6000851C7000829C700088F
:10FA6800E1C60008D7C60008D9C50008D5C50008F2
:10FA7800D3C60008CFC6000879C80008A5C8000882
:10FA8800C5C6000865D5000839C6000801C60008C3
:10FA980035D50008DDC50008A9CB00082DC9000828
:10FAA80081E3000887E30008CDC50008D1C5000838
:10FAB800C01200001F000000A81600001700000078
:10FAC800841C00000F000000E42500001E00000058
:10FAD800B42D000016000000083900000E000000D8
:10FAE8002C4C00001D000000685B000015000000A1
:10FAF800747200000D000000589800001C000000FF
:10FB080034B7000014000000E8E400000C00000016
:10FB1800783101001B000000686E0100130000002E
:10FB280034CA01000B000000286202001A0000001D
:10FB380040DB0200120000003C9303000A000000B2
:10FB4800C0C204001900000060B3050011000000E5
:10FB5800382007000900000020A10700000000006D
:10FB6800040302020101010100000000000000007E
:10FB78003C4E554C4C3E00303132333435363738F4
:10FB8800396162636465666768696A6B6C6D6E6F1C
:10FB9800707172737475767778797A003031323390
:10FBA8003435363738394142434445464748494A4F
:10FBB8004B4C4D4E4F505152535455565758595A15
:04FBC8000000000039
:10FBCC000000000000000000000000000000000029
:10FBDC000000000000000000002B7E151628AED29D
:10FBEC00A6ABF7158809CF4F3C012B7E151628AE16
:10FBFC00D2A6ABF7158809CF4F3C082B7E151628DB
:10FC0C00AED2A6ABF7158809CF4F3C092B7E151643
:10FC1C0028AED2A6ABF7158809CF4F3C0A000000DE
:10FC2C00000000000000000000000000000B0000BD
:10FC3C0000000000000000000000000000000C00AC
:10FC4C000000000000000000000000000000000D9B
:10FC5C000000000000000000000000000000000098
:10FC6C000E0000000000000000000000000000007A
:10FC7C00000F000000000000000000000000000069
:10FC8C000000100000000000000000000000000058
:08FC9C00000000000000000060
:08FCA400340FFF7F0100000096
:04FCAC005D010008EE
:04FCB000390100080E
:10FCB4000200000000000000D50200200D1800081A
:10FCC4003D18000855180008C1180008E11E000876
:10FCD400B91E00081D1E0008E921000800000000EC
:10FCE400452100081D21000871210008EB1D0008B2
:10FCF400E71D0008E91D0008251E0008ED1D000889
:10FD0400F91D0008E92000080000010000000000BF
:10FD1400000000000000000004000000401F00007C
:10FD24003075000000093D00100000005C05002053
:10FD34000000FF0000000000000000005C0500203F
:10FD44000000000000000000FF00000000000000B0
:10FD54005C0500200000000000000000000000001E
:10FD64000000000000000000E000000069680008D6
:10FD740099670008A5670008D16700080000000023
:10FD840000000000C1680008B1670008316C000879
:10FD9400000000000000000000000000000000005F
:10FDA400000E0F0D0109081101000000FF00000002
:08FDB400FFFFFFFFFFFFFFFF4F
:0400000508002411BA
:00000001FF
